:020000040800F2
:1000000000000220A903000849870008558700085E
:100010005D870008658700086D8700080000000004
:1000200000000000000000000000000081870008C0
:1000300075870008000000008D8700080191000806
:10004000F9030008F9030008F9030008F9030008A0
:10005000F9030008F9030008F9030008F903000890
:10006000F9030008F9030008F9030008F903000880
:10007000F9030008F9030008F9030008F903000870
:10008000F9030008F9030008F9030008F903000860
:10009000F9030008F9030008F9030008F903000850
:1000A000F9030008F9030008F9030008F903000840
:1000B000F903000899870008AD870008F9030008D4
:1000C000F9030008F9030008F9030008F903000820
:1000D000F9030008F9030008F9030008F903000810
:1000E000F9030008F9030008F9030008F903000800
:1000F000F9030008F9030008F9030008F9030008F0
:10010000F9030008F9030008F9030008F9030008DF
:10011000F9030008F9030008F9030008F9030008CF
:10012000D1870008F9030008F9030008B98700081F
:10013000F9030008F9030008F9030008F9030008AF
:10014000F9030008F9030008F9030008F90300089F
:10015000F9030008F9030008F9030008F90300088F
:10016000F9030008F9030008F9030008F90300087F
:10017000F9030008F9030008F90300080000000073
:10018000F9030008F9030008F9030008F90300085F
:10019000F9030008F9030008F9030008F90300084F
:1001A000F9030008F9030008F903000880B58EB0D0
:1001B00000AF40F6D803C2F200034BF6BA22CCF6E9
:1001C000DE221A6044F67403C2F200034BF6BA2230
:1001D000CCF6DE221A6040F6D803C2F200033B637D
:1001E00044F67803C2F20003FB623B6BBB6207E09C
:1001F000BB6A4FF000021A60BB6A03F10403BB62E2
:10020000FA6ABB6A9A42F3D840F6D803C2F20003F6
:100210001B68002B06D144F67403C2F200031B686E
:10022000002B00D0FEE740F20003C2F200034BF6C1
:10023000BA22CCF6DE221A6040F6D403C2F20003E2
:100240004BF6BA22CCF6DE221A6042F2C473C0F634
:1002500002037B6240F20003C2F200033B6240F6FD
:10026000D803C2F20003FB613B6ABB610BE07B6A0F
:100270001A68BB691A60BB6903F10403BB617B6A3E
:1002800003F104037B62FA69BB699A42EFD840F23A
:100290000003C2F200031A6845F27863C1F2342306
:1002A0009A420BD140F6D403C2F200031A6840F61A
:1002B000D403C2F200031B689A4200D0FEE70DF09F
:1002C0000DF807F104023B461046194608F076F98E
:1002D00040F20042C0F6000240F20043C0F60003C4
:1002E000D31A4FEAA3037B614FF000033B610BE09D
:1002F00040F20043C0F600033A6953F822309847B1
:100300003B6903F101033B617A693B699A42EFDC87
:1003100040F20042C0F6000240F20043C0F6000383
:10032000D31A4FEAA3037B614FF000033B610BE05C
:1003300040F20043C0F600033A6953F82230984770
:100340003B6903F101033B617A693B699A42EFDC47
:100350007A683B68104619460AF08AF903467B63BF
:1003600040F20042C0F6000240F20043C0F6000333
:10037000D31A4FEAA303FB60FB68BB600DE0BB68C8
:1003800003F1FF3240F20043C0F6000353F822307D
:100390009847BB6803F1FF33BB60BB68002BEEDC02
:1003A000786B08F067F900BF80B500AFFFF7FEFE7D
:1003B00080B400AFFEE700BF80B400AFFEE700BF2F
:1003C00080B400AFFEE700BF80B400AFFEE700BF1F
:1003D00080B400AFFEE700BF80B400AFFEE700BF0F
:1003E00080B400AFFEE700BF80B400AFFEE700BFFF
:1003F00080B400AFFEE700BF80B400AFFEE700BFEF
:1004000080B582B000AF78607B68002B02D14FF0DE
:100410000103B1E07B689B69002B28D07B681A68D8
:100420004FF48053C4F201039A4268D07B681A6883
:100430004FF48843C4F200039A4260D07B681A6884
:100440004FF49043C4F200039A4258D07B681A6874
:100450004FF4A053C4F201039A4250D045F2FC106D
:10046000C0F601004FF0F90108F09CF847E07B6806
:100470001A684FF48053C4F201039A423FD07B685C
:100480001A684FF48843C4F200039A4237D07B685D
:100490001A684FF49043C4F200039A422FD07B684D
:1004A0001A684FF49843C4F200039A4227D07B683D
:1004B0001A684FF4A043C4F200039A421FD07B682D
:1004C0001A684FF4A053C4F201039A4217D07B6814
:1004D0001A684FF4F043C4F200039A420FD07B68CD
:1004E0001A684FF4F843C4F200039A4207D045F269
:1004F000FC10C0F601004FF0FE0108F053F87B68D5
:1005000093F83930DBB2002B02D1786800F03AF86A
:100510007B684FF0020283F839207B681B687A6899
:100520001268D26822F40052DA60786800F0A6F807
:100530007B681B687A681268126922F490421A611B
:100540007B681B687A681268526922F02A025A6135
:100550007B681B687A681268D26842F40052DA60DD
:100560007B684FF0000283F83A207B684FF001026D
:1005700083F839204FF00003184607F10807BD46FD
:1005800080BD00BF80B483B000AF786007F10C0776
:10059000BD4680BC704700BF80B487B000AFF86034
:1005A000B9601346FB804FF000037B61FB6893F852
:1005B0003930DBB27B617B69012B02D07B69222B56
:1005C00054D1BB68002B02D0FB88002B02D14FF026
:1005D00001034DE0FB6893F83830012B02D14FF056
:1005E000020345E0FB684FF0010283F83820FB6806
:1005F000BA681A62FB68FA889A84FB68FA88DA8417
:10060000FB684FF0000283F83A20FB6893F839301A
:10061000DBB2222B05D1FB684FF0320283F8392080
:1006200004E0FB684FF0120283F83920FB681B6876
:10063000FA681268D26842F48072DA60FB681B685C
:10064000FA681268526942F001025A61FB684FF081
:10065000000283F83820FB681B68FA681268D268C9
:1006600042F04002DA604FF0000301E04FF0020375
:10067000184607F11C07BD4680BC7047F0B585B031
:1006800000AF78604FF00003FB607B681A684FF49E
:100690008053C4F201039A423FD07B681A684FF43A
:1006A0008843C4F200039A4237D07B681A684FF43B
:1006B0009043C4F200039A422FD07B681A684FF42B
:1006C0009843C4F200039A4227D07B681A684FF41B
:1006D000A043C4F200039A421FD07B681A684FF40B
:1006E000A053C4F201039A4217D07B681A684FF4F2
:1006F000F043C4F200039A420FD07B681A684FF4AB
:10070000F843C4F200039A4207D045F2FC10C0F649
:10071000010040F2147107F045FF7B685A6843F20C
:10072000A073C0F2A0039A4207D945F2FC10C0F6AC
:10073000010040F2157107F035FF7B689B68002BC4
:100740000CD07B689B68B3F5805F07D045F2FC1046
:10075000C0F6010040F2167107F024FF7B68DB68E9
:10076000002B0CD07B68DB68B3F5005F07D045F247
:10077000FC10C0F6010040F2177107F013FF7B6810
:100780001B69002B11D07B681B69B3F5806F0CD0FF
:100790007B681B69B3F5C06F07D045F2FC10C0F64B
:1007A00001004FF4E36107F0FDFE7B685A694FF6E4
:1007B000F3731340002B03D17B685B69002B07D1D7
:1007C00045F2FC10C0F6010040F2197107F0EAFE94
:1007D0007B689B69002B16D07B689B69B3F5807F93
:1007E00011D07B689B69B3F5007F0CD07B689B6957
:1007F000B3F5407F07D045F2FC10C0F6010040F28F
:100800001A7107F0CFFE7B689B69002B27D07B68AD
:100810001A684FF48053C4F201039A421FD07B68D8
:100820001A684FF48843C4F200039A4217D07B68D9
:100830001A684FF49043C4F200039A420FD07B68C9
:100840001A684FF4A053C4F201039A4207D045F24C
:10085000FC10C0F6010040F21F7107F0A3FE7B6898
:100860001B681B69FB60FB6823F44053FB607B68DB
:10087000DB68FA681343FB607B681B68FA681A61DF
:100880007B681B68DB68FB60FB6823F4164323F07E
:100890000C03FB607B689A687B681B691A437B6862
:1008A0005B691A437B68DB691343FA681343FB6097
:1008B0007B681B68FA68DA607B681B685B69FB60B1
:1008C000FB6823F44073FB607B689B69FA68134301
:1008D000FB607B681B68FA685A617B68DB69B3F56B
:1008E000004F40F0C4807B681A684FF48053C4F214
:1008F00001039A4207D07B681A684FF4A053C4F2F0
:1009000001039A4259D17B681C6802F04DF80246F7
:1009100013464FEA83039B184FEA83029A187B68B9
:100920005B684FEA4303B2FBF3F248F21F53C5F290
:10093000EB13A3FB02134FEA53134FEA031502F024
:1009400033F8024613464FEA83039B184FEA8302AB
:100950009A187B685B684FEA4303B2FBF3F602F038
:1009600023F8024613464FEA83039B184FEA83029B
:100970009A187B685B684FEA4303B2FBF3F248F2D4
:100980001F53C5F2EB13A3FB02134FEA53134FF0AF
:10099000640202FB03F3F31A4FEA031303F132027A
:1009A00048F21F53C5F2EB13A3FB02134FEA531394
:1009B00003F00F032B43A3601CE17B681C6801F06C
:1009C000C9FF024613464FEA83039B184FEA83028E
:1009D0009A187B685B684FEA4303B2FBF3F248F274
:1009E0001F53C5F2EB13A3FB02134FEA53134FEA55
:1009F000031501F0AFFF024613464FEA83039B182D
:100A00004FEA83029A187B685B684FEA4303B2FBA4
:100A1000F3F601F09FFF024613464FEA83039B184B
:100A20004FEA83029A187B685B684FEA4303B2FB84
:100A3000F3F248F21F53C5F2EB13A3FB02134FEA84
:100A400053134FF0640202FB03F3F31A4FEA03134C
:100A500003F1320248F21F53C5F2EB13A3FB02135A
:100A60004FEA531303F00F032B43A360C2E07B68EC
:100A70001A684FF48053C4F201039A4207D07B688E
:100A80001A684FF4A053C4F201039A4259D17B680B
:100A90001C6801F089FF024613464FEA83039B1846
:100AA0004FEA83029A187B685B684FEA8303B2FBC4
:100AB000F3F248F21F53C5F2EB13A3FB02134FEA04
:100AC00053134FEA031501F06FFF024613464FEA36
:100AD00083039B184FEA83029A187B685B684FEA8E
:100AE0008303B2FBF3F601F05FFF024613464FEAC1
:100AF00083039B184FEA83029A187B685B684FEA6E
:100B00008303B2FBF3F248F21F53C5F2EB13A3FBCE
:100B100002134FEA53134FF0640202FB03F3F31A7C
:100B20004FEA031303F1320248F21F53C5F2EB13ED
:100B3000A3FB02134FEA531303F00F032B43A360ED
:100B400058E07B681C6801F005FF024613464FEA37
:100B500083039B184FEA83029A187B685B684FEA0D
:100B60008303B2FBF3F248F21F53C5F2EB13A3FB6E
:100B700002134FEA53134FEA031501F0EBFE02464E
:100B800013464FEA83039B184FEA83029A187B6847
:100B90005B684FEA8303B2FBF3F601F0DBFE02462B
:100BA00013464FEA83039B184FEA83029A187B6827
:100BB0005B684FEA8303B2FBF3F248F21F53C5F2BE
:100BC000EB13A3FB02134FEA53134FF0640202FB33
:100BD00003F3F31A4FEA031303F1320248F21F53EF
:100BE000C5F2EB13A3FB02134FEA531303F00F03F9
:100BF0002B43A36007F11407BD46F0BD80B483B05A
:100C000000AF786007F10C07BD4680BC704700BF9D
:100C100080B483B000AF786007F10C07BD4680BC9C
:100C2000704700BF80B582B000AF78607B68002B52
:100C300002D14FF00103C4E07B681A684FF0000353
:100C4000C4F201039A426CD07B681B68B3F1804FF9
:100C500067D07B681A684FF48063C4F200039A423D
:100C60005FD07B681A684FF40063C4F200039A42B5
:100C700057D07B681A684FF44063C4F200039A426D
:100C80004FD07B681A684FF48053C4F200039A4235
:100C900047D07B681A684FF4A053C4F200039A420D
:100CA0003FD07B681A684FF48063C4F201039A4214
:100CB00037D07B681A684FF48043C4F201039A422C
:100CC0002FD07B681A684FF48843C4F201039A421C
:100CD00027D07B681A684FF49043C4F201039A420C
:100CE0001FD07B681A684FF4C053C4F200039A42C5
:100CF00017D07B681A684FF4E053C4F200039A429D
:100D00000FD07B681A684FF40053C4F200039A4274
:100D100007D045F22C20C0F601004FF0D10107F0BA
:100D200041FC7B689B68002B17D07B689B68102B6D
:100D300013D07B689B68202B0FD07B689B68402B6F
:100D40000BD07B689B68602B07D045F22C20C0F647
:100D500001004FF0D20107F025FC7B681B69002BD6
:100D600011D07B681B69B3F5807F0CD07B681B6951
:100D7000B3F5007F07D045F22C20C0F601004FF0FC
:100D8000D30107F00FFC7B6893F83930DBB2002BFE
:100D900002D1786800F01AF87B684FF0020283F8FD
:100DA00039207B681A687B6803F1040310461946F2
:100DB00000F00AFA7B684FF0010283F839204FF007
:100DC0000003184607F10807BD4680BD80B483B014
:100DD00000AF786007F10C07BD4680BC704700BFCC
:100DE00080B582B000AF78607B681A684FF000036E
:100DF000C4F201039A426CD07B681B68B3F1804F48
:100E000067D07B681A684FF48063C4F200039A428B
:100E10005FD07B681A684FF40063C4F200039A4203
:100E200057D07B681A684FF44063C4F200039A42BB
:100E30004FD07B681A684FF48053C4F200039A4283
:100E400047D07B681A684FF4A053C4F200039A425B
:100E50003FD07B681A684FF48063C4F201039A4262
:100E600037D07B681A684FF48043C4F201039A427A
:100E70002FD07B681A684FF48843C4F201039A426A
:100E800027D07B681A684FF49043C4F201039A425A
:100E90001FD07B681A684FF4C053C4F200039A4213
:100EA00017D07B681A684FF4E053C4F200039A42EB
:100EB0000FD07B681A684FF40053C4F200039A42C3
:100EC00007D045F22C20C0F6010040F25B1107F07C
:100ED00069FB7B681B687A681268D26842F001027D
:100EE000DA607B681B687A681268126842F0010257
:100EF0001A604FF00003184607F10807BD4680BD91
:100F000080B582B000AF78607B681B681B6903F016
:100F10000203002B27D07B681B68DB6803F0020309
:100F2000002B20D07B681B687A681268126922F057
:100F300002021A617B684FF001021A767B681B6817
:100F40009B6903F00303002B03D0786800F01EF9BF
:100F500005E0786800F010F9786800F021F97B6806
:100F60004FF000021A767B681B681B6903F00403CC
:100F7000002B27D07B681B68DB6803F00403002B81
:100F800020D07B681B687A681268126922F004021C
:100F90001A617B684FF002021A767B681B689B69B6
:100FA00003F44073002B03D0786800F0EFF805E0FD
:100FB000786800F0E1F8786800F0F2F87B684FF0AC
:100FC00000021A767B681B681B6903F00803002B7C
:100FD00027D07B681B68DB6803F00803002B20D058
:100FE0007B681B687A681268126922F008021A612D
:100FF0007B684FF004021A767B681B689B6903F0DC
:101000000303002B03D0786800F0C0F805E078688F
:1010100000F0B2F8786800F0C3F87B684FF0000287
:101020001A767B681B681B6903F01003002B27D01E
:101030007B681B68DB6803F01003002B20D07B6803
:101040001B687A681268126922F010021A617B68C4
:101050004FF008021A767B681B689B6903F44073A3
:10106000002B03D0786800F091F805E0786800F074
:1010700083F8786800F094F87B684FF000021A76E5
:101080007B681B681B6903F00103DBB2002B12D0E5
:101090007B681B68DB6803F00103DBB2002B0AD01E
:1010A0007B681B687A681268126922F001021A6173
:1010B00078680AF043FD7B681B681B6903F08003B6
:1010C000002B11D07B681B68DB6803F08003002BCA
:1010D0000AD07B681B687A681268126922F0800265
:1010E0001A617868FFF794FD7B681B681B6903F041
:1010F0004003002B11D07B681B68DB6803F04003C2
:10110000002B0AD07B681B687A681268126922F08B
:1011100040021A61786800F04DF87B681B681B6913
:1011200003F02003002B11D07B681B68DB6803F001
:101130002003002B0AD07B681B687A68126812694A
:1011400022F020021A617868FFF758FD07F10807BE
:10115000BD4680BD80B483B000AF78607B681B68FB
:101160007A681268126922F001021A6107F10C070D
:10117000BD4680BC704700BF80B483B000AF7860CC
:1011800007F10C07BD4680BC704700BF80B483B038
:1011900000AF786007F10C07BD4680BC704700BF08
:1011A00080B483B000AF786007F10C07BD4680BC07
:1011B000704700BF80B483B000AF786007F10C07C0
:1011C000BD4680BC704700BF80B485B000AF78607A
:1011D00039604FF00003FB607B681B68FB607A6836
:1011E0004FF00003C4F201039A421FD07B68B3F1B1
:1011F000804F1BD07A684FF48063C4F200039A4298
:1012000014D07A684FF40063C4F200039A420DD000
:101210007A684FF44063C4F200039A4206D07A68B9
:101220004FF48063C4F201039A4202D14FF00103EC
:1012300001E04FF00003002B08D0FB6823F070039F
:10124000FB603B685B68FA681343FB607A684FF0A9
:101250000003C4F201039A4249D07B68B3F1804F86
:1012600045D07A684FF48063C4F200039A423ED0BE
:101270007A684FF40063C4F200039A4237D07A6868
:101280004FF44063C4F200039A4230D07A684FF4BE
:101290008063C4F201039A4229D07A684FF48043F4
:1012A000C4F201039A4222D07A684FF48843C4F210
:1012B00001039A421BD07A684FF49043C4F20103B1
:1012C0009A4214D07A684FF4C053C4F200039A4291
:1012D0000DD07A684FF4E053C4F200039A4206D06E
:1012E0007A684FF40053C4F200039A4202D14FF0DF
:1012F000010301E04FF00003002B08D0FB6823F44A
:101300004073FB603B68DB68FA681343FB607B68F3
:10131000FA681A603B689A687B68DA623B681A6808
:101320007B689A627A684FF00003C4F201039A4224
:1013300006D07A684FF48063C4F201039A4202D166
:101340004FF0010301E04FF00003002B03D03B6896
:101350001A697B681A637B684FF001025A6107F1D2
:101360001407BD4680BC704780B582B000AF78607E
:101370007B68002B02D14FF0010332E17B685B6890
:10138000002B0CD07B685B68B3F5827F07D045F2F9
:101390005C20C0F601004FF0A50107F003F97B685F
:1013A0009B68002B11D07B689B68B3F5806F0CD0D5
:1013B0007B689B68B3F5004F07D045F25C20C0F610
:1013C00001004FF0A60107F0EDF87B68DB68B3F58C
:1013D000006F0BD07B68DB68002B07D045F25C20E8
:1013E000C0F601004FF0A70107F0DCF87B681B692D
:1013F000002B0BD07B681B69022B07D045F25C20C9
:10140000C0F601004FF0A80107F0CCF87B685B69DB
:10141000002B0BD07B685B69012B07D045F25C2069
:10142000C0F601004FF0A90107F0BCF87B689B698A
:10143000B3F5007F10D07B689B69002B0CD07B68D4
:101440009B69B3F5802F07D045F25C20C0F6010000
:101450004FF0AA0107F0A6F87B68DB69002B23D0C8
:101460007B68DB69082B1FD07B68DB69102B1BD0E6
:101470007B68DB69182B17D07B68DB69202B13D0C6
:101480007B68DB69282B0FD07B68DB69302B0BD0A6
:101490007B68DB69382B07D045F25C20C0F6010081
:1014A0004FF0AB0107F07EF87B681B6A002B0BD076
:1014B0007B681B6A802B07D045F25C20C0F60100D8
:1014C0004FF0AC0107F06EF87B685B6A002B0BD025
:1014D0007B685B6A102B07D045F25C20C0F60100E8
:1014E0004FF0AD0107F05EF87B689B6A002B0CD0D3
:1014F0007B689B6AB3F5005F07D045F25C20C0F6BD
:1015000001004FF0AE0107F04DF87B68DB6A002B5D
:1015100005D07B68DA6A4FF6FF739A4207D945F225
:101520005C20C0F601004FF0AF0107F03BF87B688C
:1015300093F85130DBB2002B02D1786800F056F8F6
:101540007B684FF0020283F851207B681B687A6841
:101550001268126822F040021A607B681B687A6881
:1015600051687A68926811437A68D26811437A6840
:10157000126911437A68526911437A68926902F4D8
:10158000007211437A68D26911437A68126A114372
:101590007A68926A0A431A607B681B687A68926963
:1015A0004FEA124202F004017A68526A0A435A6012
:1015B0007B681B687A68D26A1A617B681B687A68E4
:1015C0001268D26922F40062DA617B684FF000028F
:1015D00083F852207B684FF0010283F851204FF0CE
:1015E0000003184607F10807BD4680BD80B483B0EC
:1015F00000AF786007F10C07BD4680BC704700BFA4
:1016000080B584B000AFF860B9603B601346FB80E2
:10161000FB6893F85130DBB2012B40F04F81BB687F
:10162000002B02D0FB88002B02D14FF0010347E1D1
:10163000FB689B68002B0CD0FB689B68B3F5004FE0
:1016400007D045F25C20C0F601004FF4AE7106F001
:10165000A9FFFB6893F85030012B02D14FF0020331
:101660002EE1FB684FF0010283F85020FB684FF039
:10167000120283F85120FB684FF0000283F85220D9
:10168000FB68BA681A63FB68FA889A86FB68FA886E
:10169000DA86FB684FF00002DA64FB684FF0000264
:1016A0009A64FB684FF000029A87FB684FF00002D3
:1016B000DA87FB689B6AB3F5005F0FD1FB681B6894
:1016C000FA681268126822F400521A60FB681B68FC
:1016D000FA681268126842F400521A60FB689B684C
:1016E000B3F5004F07D1FB681B68FA6812681268EF
:1016F00042F480421A60FB681B681B6803F04003D9
:10170000002B07D1FB681B68FA681268126842F068
:1017100040021A60FB68DB68002B42D1FB681A6844
:10172000FB681B6B1978D16003F10102FB681A6337
:10173000FB68DB8E03F1FF339AB2FB68DA861EE0AA
:10174000F8684FF002014FF000023B6800F0BEF86D
:101750000346002B02D04FF00303B1E0FB681A6888
:10176000FB681B6B1978D16003F10102FB681A63F7
:10177000FB68DB8E03F1FF339AB2FB68DA86FB6805
:10178000DB8E002BDCD1FB689B6AB3F5005F4ED18A
:10179000FB681B68FA681268126842F480521A608B
:1017A00045E0FB681B68FA68126B1288DA60FB6818
:1017B0001B6B03F10202FB681A63FB68DB8E03F10B
:1017C000FF339AB2FB68DA8620E0F8684FF0020136
:1017D0004FF000023B6800F079F80346002B02D07E
:1017E0004FF003036CE0FB681B68FA68126B128809
:1017F000DA60FB681B6B03F10202FB681A63FB688B
:10180000DB8E03F1FF339AB2FB68DA86FB68DB8E6E
:10181000002BDAD1FB689B6AB3F5005F07D1FB6848
:101820001B68FA681268126842F480521A60F868FD
:101830004FF002014FF000023B6800F047F803460A
:10184000002B0CD0FB6893F85230DBB243F020033E
:10185000DAB2FB6883F852204FF0030330E0F868F7
:101860004FF080014FF001023B6800F02FF8034673
:10187000002B0CD0FB6893F85230DBB243F020030E
:10188000DAB2FB6883F852204FF0030318E0FB68DC
:101890009B68002B05D1FB681B68DB68FB681B6835
:1018A0009B68FB684FF0010283F85120FB684FF002
:1018B000000283F850204FF0000301E04FF00203D4
:1018C000184607F11007BD4680BD00BF80B586B041
:1018D00000AFF860B9603B601346FB714FF0000346
:1018E0007B6106F053FE02463B68D3187B61FB79AF
:1018F000002B40F083803BE03B68B3F1FF3F37D0E3
:1019000006F044FE02467B699A4231D3FB681B68AD
:10191000FA681268526822F0E0025A60FB681B689D
:10192000FA681268126822F040021A60FB689B6A2B
:10193000B3F5005F0FD1FB681B68FA681268126884
:1019400022F400521A60FB681B68FA681268126879
:1019500042F400521A60FB684FF0010283F85120F4
:10196000FB684FF0000283F850204FF0030351E072
:10197000FB681B689B681A46BB681A40BB689A42A2
:10198000BAD145E03B68B3F1FF3F38D006F0FEFD29
:1019900002467B699A4232D3FB681B68FA68126878
:1019A000526822F0E0025A60FB681B68FA6812680D
:1019B000126822F040021A60FB689B6AB3F5005F70
:1019C0000FD1FB681B68FA681268126822F4005293
:1019D0001A60FB681B68FA681268126842F40052C9
:1019E0001A60FB684FF0010283F85120FB684FF04A
:1019F000000283F850204FF003030BE000BFFB68A8
:101A00001B689B681A46BB681A40BB689A42B9D0EB
:101A10004FF00003184607F11807BD4680BD00BF10
:101A200080B483B000AF03463960FB7197F907308B
:101A3000002B10DA4FF46D43CEF20003FA7902F076
:101A40000F02A2F104013A68D2B24FEA0212D2B2F6
:101A50005B181A760DE04FF46143CEF2000397F95C
:101A600007103A68D2B24FEA0212D2B25B1883F87A
:101A7000002307F10C07BD4680BC704780B582B0DB
:101A800000AF78607B6803F1FF326FF07F439A42CA
:101A900002D94FF001031DE04EF21003CEF2000315
:101AA0007A6802F1FF325A604FF0FF304FF00F01B9
:101AB000FFF7B6FF4EF21003CEF200034FF0000224
:101AC0009A604EF21003CEF200034FF007021A6044
:101AD0004FF00003184607F10807BD4680BD00BF60
:101AE00090B595B000AF78604FF00003FB647B6861
:101AF0001B680F2B07D945F29C20C0F601004FF45C
:101B00009D7106F04FFD7B681B6803F00103DBB29B
:101B1000002B00F0A6807B685B68002B0FD07B68F1
:101B20005B68012B0BD07B685B68052B07D045F207
:101B30009C20C0F6010040F23F1106F033FD4FF447
:101B40006053C4F202039B6803F00C03042B11D012
:101B50004FF46053C4F202039B6803F00C03082B9C
:101B600018D14FF46053C4F202035B6803F480039E
:101B7000002B0FD04FF46053C4F202031B6803F430
:101B80000033002B6CD07B685B68012B68D04FF072
:101B9000010358E343F60203C4F202034FF00002CC
:101BA0001A7006F0F3FC034603F59C5303F1080397
:101BB000FB6408E006F0EAFC0246FB6C9A4202D3A2
:101BC0004FF003033FE34FF46053C4F202031B687A
:101BD00003F40033002BEDD143F60203C4F20203F9
:101BE0007A685268D2B21A707B685B68012B1BD18D
:101BF00006F0CCFC034603F59C5303F10803FB6499
:101C000008E006F0C3FC0246FB6C9A4202D34FF098
:101C1000030318E34FF46053C4F202031B6803F498
:101C20000033002BEDD01CE006F0B0FC034603F5BA
:101C30009C5303F10803FB6408E006F0A7FC02468E
:101C4000FB6C9A4202D34FF00303FCE24FF4605363
:101C5000C4F202031B6803F40033002BEDD100E053
:101C600000BF7B681B6803F00203002B00F0AE800E
:101C70007B68DB68002B0BD07B68DB68012B07D00F
:101C800045F29C20C0F6010040F27F1106F08AFC6C
:101C90007B681B691F2B07D945F29C20C0F6010009
:101CA0004FF4C07106F07EFC4FF46053C4F202039F
:101CB0009B6803F00C03002B11D04FF46053C4F267
:101CC00002039B6803F00C03082B18D14FF46053F8
:101CD000C4F202035B6803F48003002B0FD14FF4BE
:101CE0006053C4F202031B6803F00203002B6CD0A4
:101CF0007B68DB68012B68D04FF00103A3E27B68AF
:101D0000DB68002B40D04FF00003C4F247234FF0B4
:101D100001021A6006F03AFC034603F16403FB6417
:101D200008E006F033FC0246FB6C9A4202D34FF007
:101D3000030388E24FF46053C4F202031B6803F00C
:101D40000203002BEDD04FF46053C4F202034FF4B2
:101D50006052C4F20202126822F0F8017A68106937
:101D60004FF0F802BA64BA6C92FAA2F47C647A6C0E
:101D70003A643A6CB2FA82F4FC63FA6BD2B200FABB
:101D800002F20A431A6021E04FF00003C4F2472335
:101D90004FF000021A6006F0F9FB034603F16403FA
:101DA000FB6408E006F0F2FB0246FB6C9A4202D3A9
:101DB0004FF0030347E24FF46053C4F202031B6881
:101DC00003F00203002BEDD100E000BF7B681B682D
:101DD00003F00803002B54D07B685B69002B0BD009
:101DE0007B685B69012B07D045F29C20C0F601009F
:101DF0004FF4DC7106F0D6FB7B685B69002B20D0CA
:101E00004FF46863C4F247234FF001021A6006F0F2
:101E1000BDFB034603F16403FB6408E006F0B6FB78
:101E20000246FB6C9A4202D34FF003030BE24FF4DD
:101E30006053C4F202035B6F03F00203002BEDD08A
:101E40001FE04FF46863C4F247234FF000021A60AA
:101E500006F09CFB034603F16403FB6408E006F014
:101E600095FB0246FB6C9A4202D34FF00303EAE172
:101E70004FF46053C4F202035B6F03F00203002BC4
:101E8000EDD17B681B6803F00403002B00F0AA80EF
:101E90007B689B68002B0FD07B689B68012B0BD065
:101EA0007B689B68052B07D045F29C20C0F601009B
:101EB0004FF4F17106F076FB4FF46053C4F2020365
:101EC0004FF46052C4F20202126C42F080521A6463
:101ED0004FF4E043C4F200034FF4E042C4F20002C6
:101EE000126842F480721A6006F050FB034603F158
:101EF0006403FB6408E006F049FB0246FB6C9A426F
:101F000002D34FF003039EE14FF4E043C4F2000319
:101F10001B6803F48073002BEDD043F67003C4F20A
:101F200002034FF000021A7006F030FB034603F57F
:101F30009C5303F10803FB6408E006F027FB02460C
:101F4000FB6C9A4202D34FF003037CE14FF46053E1
:101F5000C4F202031B6F03F00203002BEDD143F622
:101F60007003C4F202037A689268D2B21A707B6876
:101F70009B68012B1BD106F009FB034603F59C531C
:101F800003F10803FB6408E006F000FB0246FB6C6B
:101F90009A4202D34FF0030355E14FF46053C4F269
:101FA00002031B6F03F00203002BEDD01AE006F0D2
:101FB000EDFA034603F59C5303F10803FB6408E0C4
:101FC00006F0E4FA0246FB6C9A4202D34FF0030398
:101FD00039E14FF46053C4F202031B6F03F00203B4
:101FE000002BEDD17B689B69002B0FD07B689B6930
:101FF000012B0BD07B689B69022B07D045F29C20FC
:10200000C0F6010040F2262106F0CCFA7B689B69FD
:10201000002B00F016814FF46053C4F202039B685A
:1020200003F00C03082B00F009817B689B69022BED
:1020300040F0E3807B68DB69002B0CD07B68DB69B8
:10204000B3F5800F07D045F29C20C0F6010040F2A6
:102050002F2106F0A7FA7B681B6A3F2B07D945F2B0
:102060009C20C0F601004FF40C7106F09BFA7B68CF
:102070005B6ABF2B04D97B685B6AB3F5D87F07D94D
:1020800045F29C20C0F6010040F2312106F08AFAA8
:102090007B689B6A022B13D07B689B6A042B0FD052
:1020A0007B689B6A062B0BD07B689B6A082B07D04A
:1020B00045F29C20C0F6010040F2322106F072FA8F
:1020C0007B68DB6A032B03D97B68DB6A0F2B07D99C
:1020D00045F29C20C0F6010040F2332106F062FA7E
:1020E0004FF06003C4F247234FF000021A6006F07D
:1020F0004DFA034603F16403FB6408E006F046FA78
:102100000246FB6C9A4202D34FF003039BE04FF46C
:102110006053C4F202031B6803F00073002BEDD17F
:102120004FF46053C4F202037A68116A7A68506A05
:1021300047F6C072BA63BA6B92FAA2F47C637A6B08
:102140003A633A6BB2FA82F4FC62FA6AD2B200FAEB
:1021500002F211437A68926A4FEA520202F1FF30AA
:102160004FF44032BA62BA6A92FAA2F47C627A6A96
:102170003A623A6AB2FA82F4FC61FA69D2B200FABF
:1021800002F211437A68D26911437A68D06A4FF03B
:102190007062BA61BA6992FAA2F47C617A693A61B2
:1021A0003A69B2FA82F4FC60FA68D2B200FA02F23A
:1021B0000A4342F000525A604FF06003C4F24723D2
:1021C0004FF001021A6006F0E1F9034603F16403DF
:1021D000FB6408E006F0DAF90246FB6C9A4202D38F
:1021E0004FF003032FE04FF46053C4F202031B6867
:1021F00003F00073002BEDD023E04FF06003C4F236
:1022000047234FF000021A6006F0C0F9034603F1BD
:102210006403FB6408E006F0B9F90246FB6C9A42DD
:1022200002D34FF003030EE04FF46053C4F20203F5
:102230001B6803F00073002BEDD102E04FF00103A7
:1022400001E04FF00003184607F15407BD4690BD6A
:1022500080B584B000AF786039604FF00003FB6058
:102260007B681B68002B03D07B681B680F2B07D98A
:1022700045F29C20C0F6010040F2962106F092F94A
:102280003B68002B34D03B68012B31D03B68022BDC
:102290002ED03B68032B2BD03B68042B28D03B6807
:1022A000052B25D03B68062B22D03B68072B1FD07F
:1022B0003B68082B1CD03B68092B19D03B680A2BC4
:1022C00016D03B680B2B13D03B680C2B10D03B680F
:1022D0000D2B0DD03B680E2B0AD03B680F2B07D07F
:1022E00045F29C20C0F6010040F2972106F05AF911
:1022F0004FF47053C4F202031B6803F00F023B68F3
:102300009A4280F0B7804FF47053C4F202033A68E7
:10231000D2B21A704FF47053C4F202031B6803F078
:102320000F023B689A4202D04FF0010315E27B682E
:102330001B6803F00103DBB2002B00F051817B68C6
:102340005B68002B0FD07B685B68012B0BD07B6830
:102350005B68022B07D045F29C20C0F6010040F2DA
:10236000AD2106F01FF97B685B68012B0BD14FF4A0
:102370006053C4F202031B6803F40033002B1ED128
:102380004FF00103E9E17B685B68022B0BD14FF44E
:102390006053C4F202031B6803F00073002B0ED1DC
:1023A0004FF00103D9E14FF46053C4F202031B68FC
:1023B00003F00203002B02D14FF00103CDE14FF4F3
:1023C0006053C4F202034FF46052C4F202029268F6
:1023D00022F003017A6852680A439A6006F0D6F840
:1023E000034603F59C5303F10803FB607B685B68BD
:1023F000012B13D108E006F0C9F80246FB689A42A7
:1024000002D34FF00303A8E14FF46053C4F2020378
:102410009B6803F00C03042BEDD1E1E07B685B6863
:10242000022B1CD108E006F0B1F80246FB689A4284
:1024300002D34FF0030390E14FF46053C4F2020360
:102440009B6803F00C03082BEDD1C9E006F09EF861
:102450000246FB689A4203D34FF003037DE100BFBD
:102460004FF46053C4F202039B6803F00C03002B8B
:10247000ECD1B5E07B681B6803F00103DBB2002BF5
:1024800000F09A807B685B68002B0FD07B685B68EC
:10249000012B0BD07B685B68022B07D045F29C2098
:1024A000C0F6010040F2F52106F07CF87B685B681D
:1024B000012B0BD14FF46053C4F202031B6803F4E9
:1024C0000033002B1ED14FF0010346E17B685B68AF
:1024D000022B0BD14FF46053C4F202031B6803F0CC
:1024E0000073002B0ED14FF0010336E14FF460531F
:1024F000C4F202031B6803F00203002B02D14FF069
:1025000001032AE14FF46053C4F202034FF4605216
:10251000C4F20202926822F003017A6852680A4308
:102520009A6006F033F8034603F59C5303F1080361
:10253000FB607B685B68012B13D108E006F026F88E
:102540000246FB689A4202D34FF0030305E14FF4C1
:102550006053C4F202039B6803F00C03042BEDD11B
:102560002AE07B685B68022B1CD108E006F00EF8BD
:102570000246FB689A4202D34FF00303EDE04FF4AA
:102580006053C4F202039B6803F00C03082BEDD1E7
:1025900012E005F0FBFF0246FB689A4203D34FF0BE
:1025A0000303DAE000BF4FF46053C4F202039B68F8
:1025B00003F00C03002BECD14FF47053C4F2020370
:1025C0003A68D2B21A704FF47053C4F202031B6817
:1025D00003F00F023B689A4202D04FF00103BCE0C7
:1025E0007B681B6803F00203002B3AD07B689B6872
:1025F000002B27D07B689B68802B23D07B689B684F
:10260000902B1FD07B689B68A02B1BD07B689B689E
:10261000B02B17D07B689B68C02B13D07B689B685E
:10262000D02B0FD07B689B68E02B0BD07B689B681E
:10263000F02B07D045F29C20C0F6010040F2453156
:1026400005F0B0FF4FF46053C4F202034FF4605240
:10265000C4F20202926822F0F0017A6892680A439A
:102660009A607B681B6803F00403002B2ED07B6804
:10267000DB68002B1BD07B68DB68B3F5805F16D06E
:102680007B68DB68B3F5A05F11D07B68DB68B3F5CE
:10269000C05F0CD07B68DB68B3F5E05F07D045F224
:1026A0009C20C0F601004FF4537105F07BFF4FF4FE
:1026B0006053C4F202034FF46052C4F20202926803
:1026C00022F4E0517A68D2680A439A607B681B68FA
:1026D00003F00803002B30D07B681B69002B1BD054
:1026E0007B681B69B3F5805F16D07B681B69B3F507
:1026F000A05F11D07B681B69B3F5C05F0CD07B680D
:102700001B69B3F5E05F07D045F29C20C0F60100DD
:1027100040F2533105F046FF4FF46053C4F2020318
:102720004FF46052C4F20202926822F460417A6867
:1027300012694FEAC2020A439A6000F0D7F80246D3
:1027400044F6D353C1F26203A3FB02134FEA93137F
:102750001846FFF793F94FF00003184607F11007EA
:10276000BD4680BD90B494B000AF4FF000037B64D1
:102770004FF00003FB644FF000033B644FF0000395
:10278000BB644FF46053C4F202039B6803F00C0374
:10279000042B0AD0082B0ED0002B40F09A804FF467
:1027A0001053C0F2F403BB6499E04FF45853C0F2E5
:1027B0006E13BB6493E04FF46053C4F202035B6892
:1027C00003F03F037B644FF46053C4F202035B6881
:1027D00003F480024FF48003FB63FB6B93FAA3F4D2
:1027E000BC63BB6B7B637B6BB3FA83F43C633B6B77
:1027F000DBB222FA03F3002B24D04FF45853C0F27B
:102800006E137A6CB3FBF2F24FF46053C4F202031E
:102810005B68194647F6C0730B4047F6C071F96212
:10282000F96A91FAA1F4BC62B96A7962796AB1FA7B
:1028300081F43C62396AC9B223FA01F303FB02F363
:10284000FB6423E04FF41053C0F2F4037A6CB3FB43
:10285000F2F24FF46053C4F202035B68194647F684
:10286000C0730B4047F6C071F961F96991FAA1F4A0
:10287000BC61B96979617969B1FA81F43C613969FE
:10288000C9B223FA01F303FB02F3FB644FF4605374
:10289000C4F202035B6803F440324FF44033FB6040
:1028A000FB6893FAA3F4BC60BB687B607B68B3FAF7
:1028B00083F43C603B68DBB222FA03F303F10103CB
:1028C0004FEA43033B64FA6C3B6CB2FBF3F3BB642B
:1028D00005E04FF41053C0F2F403BB6400BFBB6CBF
:1028E000184607F15007BD4690BC704790B585B0BB
:1028F00000AFFFF737FF02464FF46053C4F2020304
:102900009B6803F0F0014FF0F003FB60FB6893FA63
:10291000A3F4BC60BB687B607B68B3FA83F43C6063
:102920003B68DBB221FA03F145F28C23C0F60103C8
:102930005B5C22FA03F240F20C03C2F200031A605D
:1029400040F20C03C2F200031B68184607F114079B
:10295000BD4690BD90B585B000AFFFF7C7FF0246FA
:102960004FF46053C4F202039B6803F4E0514FF448
:10297000E053FB60FB6893FAA3F4BC60BB687B6028
:102980007B68B3FA83F43C603B68DBB221FA03F165
:1029900045F28C23C0F601035B5C22FA03F3184670
:1029A00007F11407BD4690BD90B585B000AFFFF7A5
:1029B0009DFF02464FF46053C4F202039B6803F488
:1029C00060414FF46043FB60FB6893FAA3F4BC6082
:1029D000BB687B607B68B3FA83F43C603B68DBB226
:1029E00021FA03F145F28C23C0F601035B5C22FA65
:1029F00003F3184607F11407BD4690BD90B587B0A4
:102A000000AF786039604FF000033B614FF0000386
:102A1000FB604FF00003BB603B681B68002B07D1D5
:102A200045F2CC20C0F601004FF0C30105F0BAFD1D
:102A30003B685B68002B4BD03B685B68012B47D041
:102A40003B685B68112B43D03B685B68022B3FD02F
:102A50003B685B68122B3BD03B685A684FF0000321
:102A6000C1F211039A4233D03B685A684FF0000319
:102A7000C1F221039A422BD03B685A684FF0000301
:102A8000C1F231039A4223D03B685A684FF00003E9
:102A9000C1F212039A421BD03B685A684FF0000300
:102AA000C1F222039A4213D03B685A684FF00003E8
:102AB000C1F232039A420BD03B685B68032B07D00C
:102AC00045F2CC20C0F601004FF0C40105F06AFDCC
:102AD0003B689B68002B0FD03B689B68012B0BD099
:102AE0003B689B68022B07D045F2CC20C0F6010062
:102AF0004FF0C50105F056FD4FF000037B61F5E294
:102B00007B694FF0010202FA03F33B613B681A68EC
:102B10003B691340FB60FA683B699A4240F0E282ED
:102B20003B685B68022B04D03B685B68122B40F06B
:102B3000FA803B681B69002B00F0BB803B681B6977
:102B4000092B00F0B6803B681B69002B00F0B180B8
:102B50003B681B69002B00F0AC803B681B69002BB5
:102B600000F0A7803B681B69002B00F0A2803B6847
:102B70001B69012B00F09D803B681B69012B00F055
:102B800098803B681B69022B00F093803B681B69AF
:102B9000022B00F08E803B681B69022B00F08980BD
:102BA0003B681B69032B00F084803B681B69042B86
:102BB0007FD03B681B69042B7BD03B681B69042BCF
:102BC00077D03B681B69052B73D03B681B69052BCD
:102BD0006FD03B681B69092B6BD03B681B69062BC8
:102BE00067D03B681B69092B63D03B681B69072BC7
:102BF0005FD03B681B69072B5BD03B681B69072BC9
:102C000057D03B681B69082B53D03B681B69082BC6
:102C10004FD03B681B69082B4BD03B681B69092BC5
:102C200047D03B681B69092B43D03B681B690A2BC3
:102C30003FD03B681B690A2B3BD03B681B690B2BC1
:102C400037D03B681B690C2B33D03B681B690C2BBE
:102C50002FD03B681B690D2B2BD03B681B690F2BBA
:102C600027D03B681B69052B23D03B681B69052BCC
:102C70001FD03B681B69052B1BD03B681B69082BC9
:102C800017D03B681B69082B13D03B681B690C2BC2
:102C90000FD03B681B69062B0BD03B681B690E2BC2
:102CA00007D045F2CC20C0F601004FF0D60105F068
:102CB00079FC3B681A697B6903F007034FEA8303D9
:102CC00002FA03F3BB607B694FEAD3027B694FEAE8
:102CD000D3017B6801F1080153F8213019467B6963
:102CE00003F007034FEA83034FF00F0000FA03F3EA
:102CF0006FEA030319407B6802F1080243F82210CF
:102D00007B694FEAD3027B694FEAD3017B6801F10B
:102D1000080153F821301946BB6819437B6802F15A
:102D2000080243F822107B681B681A467B694FEA49
:102D300043034FF0030101FA03F36FEA03031A4060
:102D40007B681A607B681B681A463B685B6803F007
:102D500003017B694FEA430301FA03F31A437B68DB
:102D60001A603B685B68012B0BD03B685B68022BE9
:102D700007D03B685B68112B03D03B685B68122B64
:102D80004FD13B68DB68002B13D03B68DB68012B1D
:102D90000FD03B68DB68022B0BD03B68DB68032B52
:102DA00007D045F2CC20C0F601004FF0E60105F057
:102DB000F9FB7B689B681A467B694FEA43034FF037
:102DC000030101FA03F36FEA03031A407B689A6078
:102DD0007B689B681A463B68D9687B694FEA430366
:102DE00001FA03F31A437B689A607B685B681A46B2
:102DF0007B694FF0010101FA03F36FEA03031A4004
:102E00007B685A607B685B681A463B685B6803F0C6
:102E100010034FEA13117B6901FA03F31A437B682D
:102E20005A607B68DB681A467B694FEA43034FF0C0
:102E3000030101FA03F36FEA03031A407B68DA60C7
:102E40007B68DB681A463B6899687B694FEA4303F5
:102E500001FA03F31A437B68DA603B685B6803F0AE
:102E60008053002B00F03E814FF46053C4F2020304
:102E70004FF46052C4F20202526C42F480425A642F
:102E80007B6903F003034FEA83034FF00F0202FA5A
:102E900003F3BB604FF46053C4F201037A694FEA55
:102EA00092004FF46052C4F2010279694FEA910135
:102EB00001F1020152F821201146BA686FEA0202BC
:102EC000114000F1020243F822104FF46053C4F2A3
:102ED00001037A694FEA92004FF46052C4F2010292
:102EE00079694FEA910101F1020152F8212011465E
:102EF0007C684FF00002C4F2020294425CD07C680D
:102F00004FF48062C4F20202944252D07C684FF4C3
:102F10000062C4F20202944248D07C684FF44062DE
:102F2000C4F2020294423ED07C684FF48052C4F254
:102F30000202944234D07C684FF4A052C4F20202E0
:102F400094422AD07C684FF4C052C4F202029442E8
:102F500020D07C684FF4E052C4F20202944216D0B2
:102F60007C684FF40052C4F2020294420CD07C6898
:102F70004FF41052C4F20202944202D14FF00902FF
:102F800001E04FF00A0201E04FF0080201E04FF0CB
:102F9000070201E04FF0060201E04FF0050201E0F8
:102FA0004FF0040201E04FF0030201E04FF0020293
:102FB00001E04FF0010201E04FF000027C6904F0F3
:102FC00003044FEA840402FA04F2114300F10202FE
:102FD00043F822104FF47053C4F201034FF47052BF
:102FE000C4F2010212681146FA686FEA02020A404E
:102FF0001A604FF47053C4F201034FF47052C4F2DC
:10300000010252681146FA686FEA02020A405A60E9
:103010003B685B6803F48033002B0CD04FF4705393
:10302000C4F201034FF47052C4F201021268114657
:10303000FA680A431A603B685B6803F40033002BAC
:103040000CD04FF47053C4F201034FF47052C4F229
:10305000010252681146FA680A435A604FF47053ED
:10306000C4F201034FF47052C4F201029268114697
:10307000FA686FEA02020A409A604FF47053C4F291
:1030800001034FF47052C4F20102D2681146FA688B
:103090006FEA02020A40DA603B685B6803F480135F
:1030A000002B0CD04FF47053C4F201034FF4705254
:1030B000C4F2010292681146FA680A439A603B68BA
:1030C0005B6803F40013002B0CD04FF47053C4F270
:1030D00001034FF47052C4F20102D2681146FA683B
:1030E0000A43DA607B6903F101037B617B690F2B83
:1030F0007FF606AD07F11C07BD4690BD80B584B0D4
:1031000000AF78600B467B807B88012B3CD07B88AE
:10311000022B39D07B88042B36D07B88082B33D008
:103120007B88102B30D07B88202B2DD07B88402BA8
:103130002AD07B88802B27D07B88B3F5807F23D053
:103140007B88B3F5007F1FD07B88B3F5806F1BD0E1
:103150007B88B3F5006F17D07B88B3F5805F13D001
:103160007B88B3F5005F0FD07B88B3F5804F0BD021
:103170007B88B3F5004F07D045F2CC20C0F60100A4
:1031800040F2751105F00EFA7B681B691A467B88C0
:103190001340002B03D04FF00103FB7302E04FF00C
:1031A0000003FB73FB7B184607F11007BD4680BD8B
:1031B00080B582B000AF786013460A467A807B7093
:1031C0007B88012B3CD07B88022B39D07B88042B59
:1031D00036D07B88082B33D07B88102B30D07B886F
:1031E000202B2DD07B88402B2AD07B88802B27D08A
:1031F0007B88B3F5807F23D07B88B3F5007F1FD019
:103200007B88B3F5806F1BD07B88B3F5006F17D038
:103210007B88B3F5805F13D07B88B3F5005F0FD058
:103220007B88B3F5804F0BD07B88B3F5004F07D078
:1032300045F2CC20C0F601004FF4CB7105F0B2F995
:103240007B78002B0AD07B78012B07D045F2CC206D
:10325000C0F6010040F2971105F0A4F97B78002B2D
:1032600003D07B687A881A8302E07B687A885A8365
:1032700007F10807BD4680BD80B584B000AF786017
:103280004FF00003FB607B68002B02D14FF001037D
:1032900009E27B681A6846F21003C4F202039A42FC
:1032A0007FD07B681A6846F22803C4F202039A4270
:1032B00077D07B681A6846F24003C4F202039A4250
:1032C0006FD07B681A6846F25803C4F202039A4230
:1032D00067D07B681A6846F27003C4F202039A4210
:1032E0005FD07B681A6846F28803C4F202039A42F0
:1032F00057D07B681A6846F2A003C4F202039A42D0
:103300004FD07B681A6846F2B803C4F202039A42AF
:1033100047D07B681A6846F21043C4F202039A420F
:103320003FD07B681A6846F22843C4F202039A42EF
:1033300037D07B681A6846F24043C4F202039A42CF
:103340002FD07B681A6846F25843C4F202039A42AF
:1033500027D07B681A6846F27043C4F202039A428F
:103360001FD07B681A6846F28843C4F202039A426F
:1033700017D07B681A6846F2A043C4F202039A424F
:103380000FD07B681A6846F2B843C4F202039A422F
:1033900007D045F2FC20C0F601004FF0B50105F062
:1033A00001F97B685B68002B2AD07B685B68B3F10E
:1033B000007F25D07B685B68B3F1806F20D07B688D
:1033C0005B68B3F1C06F1BD07B685B68B3F1006FC3
:1033D00016D07B685B68B3F1206F11D07B685B68A7
:1033E000B3F1406F0CD07B685B68B3F1606F07D0BE
:1033F00045F2FC20C0F601004FF0B60105F0D2F80E
:103400007B689B68002B0FD07B689B68402B0BD0A0
:103410007B689B68802B07D045F2FC20C0F601003A
:103420004FF0B70105F0BEF87B68DB68B3F5007FAD
:103430000BD07B68DB68002B07D045F2FC20C0F680
:1034400001004FF0B80105F0ADF87B681B69B3F5DA
:10345000806F0BD07B681B69002B07D045F2FC20E6
:10346000C0F601004FF0B90105F09CF87B685B697C
:10347000002B11D07B685B69B3F5006F0CD07B68C3
:103480005B69B3F5805F07D045F2FC20C0F6010010
:103490004FF0BA0105F086F87B689B69002B11D0CC
:1034A0007B689B69B3F5005F0CD07B689B69B3F5C3
:1034B000804F07D045F2FC20C0F601004FF0BB0161
:1034C00005F070F87B68DB69002B10D07B68DB6946
:1034D000B3F5807F0BD07B68DB69202B07D045F2EA
:1034E000FC20C0F601004FF0BC0105F05BF87B68E2
:1034F0001B6A002B16D07B681B6AB3F5803F11D086
:103500007B681B6AB3F5003F0CD07B681B6AB3F580
:10351000403F07D045F2FC20C0F601004FF0BD014E
:1035200005F040F87B685B6A002B0BD07B685B6A18
:10353000042B07D045F2FC20C0F601004FF0BE017D
:1035400005F030F87B685B6A002B4DD07B689B6A86
:10355000002B13D07B689B6A012B0FD07B689B6A82
:10356000022B0BD07B689B6A032B07D045F2FC2013
:10357000C0F601004FF0C30105F014F87B68DB6A68
:10358000002B16D07B68DB6AB3F5000F11D07B6887
:10359000DB6AB3F1807F0CD07B68DB6AB3F1C07F5C
:1035A00007D045F2FC20C0F601004FF0C40104F042
:1035B000F9FF7B681B6B002B16D07B681B6BB3F588
:1035C000001F11D07B681B6BB3F5800F0CD07B689C
:1035D0001B6BB3F5C00F07D045F2FC20C0F601000D
:1035E0004FF0C50104F0DEFF7B684FF0020283F864
:1035F00035207B681B681B68FB60FA6848F23F0354
:10360000CFF214031340FB607B685A687B689B68A9
:103610001A437B68DB681A437B681B691A437B6823
:103620005B691A437B689B691A437B68DB691A43B1
:103630007B681B6A1343FA681343FB607B685B6A11
:10364000042B07D17B68DA6A7B681B6B1343FA682B
:103650001343FB607B681B68FA681A607B681B6811
:103660005B69FB60FB6823F00703FB607B685B6AB8
:10367000FA681343FB607B685B6A042B04D17B68A8
:103680009B6AFA681343FB607B681B68FA685A619F
:103690007B684FF00002DA647B684FF0010283F828
:1036A00035204FF00003184607F11007BD4680BDD6
:1036B00080B582B000AF78607B681B681A4646F21E
:1036C0005843C4F202039A4240F293804FF4C84335
:1036D000C4F202035B681A467B68196846F210035D
:1036E000C4F2020399427BD07B68196846F210430A
:1036F000C4F20203994270D07B68196846F27003E5
:10370000C4F20203994265D07B68196846F270439F
:10371000C4F2020399425AD07B68196846F2280322
:10372000C4F2020399424FD07B68196846F22843DD
:10373000C4F20203994244D07B68196846F28803B8
:10374000C4F20203994239D07B68196846F2884373
:10375000C4F2020399422ED07B68196846F24003F6
:10376000C4F20203994223D07B68196846F24043B1
:10377000C4F20203994218D07B68196846F2A0038C
:10378000C4F2020399420DD07B68196846F2A04347
:10379000C4F20203994202D14FF4002301E04FF03A
:1037A000007301E04FF4002301E04FF4002301E037
:1037B0004FF4002301E04FF4007301E04FF4007375
:1037C00001E04FF4007301E04FF4007301E04FF0AB
:1037D000080301E04FF0080301E04FF0080301E0A7
:1037E0004FF008031340002B0CBF00230123DBB272
:1037F000CBE17B681B681A4646F2B803C4F20203A9
:103800009A4240F293804FF4C843C4F202031B680B
:103810001A467B68196846F21003C4F20203994203
:103820007BD07B68196846F21043C4F202039942C8
:1038300070D07B68196846F27003C4F202039942A3
:1038400065D07B68196846F27043C4F2020399425E
:103850005AD07B68196846F22803C4F202039942E1
:103860004FD07B68196846F22843C4F2020399429C
:1038700044D07B68196846F28803C4F20203994277
:1038800039D07B68196846F28843C4F20203994232
:103890002ED07B68196846F24003C4F202039942B5
:1038A00023D07B68196846F24043C4F20203994270
:1038B00018D07B68196846F2A003C4F2020399424B
:1038C0000DD07B68196846F2A043C4F20203994206
:1038D00002D14FF4002301E04FF0007301E04FF4F8
:1038E000002301E04FF4002301E04FF4002301E046
:1038F0004FF4007301E04FF4007301E04FF40073E4
:1039000001E04FF4007301E04FF0080301E04FF0D5
:10391000080301E04FF0080301E04FF008031340F3
:10392000002B0CBF00230123DBB22EE17B681B6858
:103930001A4646F25803C4F202039A4240F29380B8
:103940004FF4C043C4F202035B681A467B681968EF
:1039500046F21003C4F2020399427BD07B681968D7
:1039600046F21043C4F20203994270D07B68196892
:1039700046F27003C4F20203994265D07B6819686D
:1039800046F27043C4F2020399425AD07B68196828
:1039900046F22803C4F2020399424FD07B681968AB
:1039A00046F22843C4F20203994244D07B68196866
:1039B00046F28803C4F20203994239D07B68196841
:1039C00046F28843C4F2020399422ED07B681968FC
:1039D00046F24003C4F20203994223D07B6819687F
:1039E00046F24043C4F20203994218D07B6819683A
:1039F00046F2A003C4F2020399420DD07B68196815
:103A000046F2A043C4F20203994202D14FF40023CC
:103A100001E04FF0007301E04FF4002301E04FF4A8
:103A2000002301E04FF4002301E04FF4007301E0B4
:103A30004FF4007301E04FF4007301E04FF40073A2
:103A400001E04FF0080301E04FF0080301E04FF000
:103A5000080301E04FF008031340002B0CBF0023C4
:103A60000123DBB291E04FF4C043C4F202031B68B0
:103A70001A467B68196846F21003C4F202039942A1
:103A80007BD07B68196846F21043C4F20203994266
:103A900070D07B68196846F27003C4F20203994241
:103AA00065D07B68196846F27043C4F202039942FC
:103AB0005AD07B68196846F22803C4F2020399427F
:103AC0004FD07B68196846F22843C4F2020399423A
:103AD00044D07B68196846F28803C4F20203994215
:103AE00039D07B68196846F28843C4F202039942D0
:103AF0002ED07B68196846F24003C4F20203994253
:103B000023D07B68196846F24043C4F2020399420D
:103B100018D07B68196846F2A003C4F202039942E8
:103B20000DD07B68196846F2A043C4F202039942A3
:103B300002D14FF4002301E04FF0007301E04FF495
:103B4000002301E04FF4002301E04FF4002301E0E3
:103B50004FF4007301E04FF4007301E04FF4007381
:103B600001E04FF4007301E04FF0080301E04FF073
:103B7000080301E04FF0080301E04FF00803134091
:103B8000002B0CBF00230123DBB2002B00F091823D
:103B90007B681B681B6803F00403002B00F089821C
:103BA0007B681B687A681268126822F004021A6047
:103BB0007B681B681A4646F25843C4F202039A42D5
:103BC00040F293804FF4C843C4F202034FF4C8425A
:103BD000C4F20202D26811467A68106846F21002F6
:103BE000C4F2020290427BD07A68106846F210421A
:103BF000C4F20202904270D07A68106846F27002F5
:103C0000C4F20202904265D07A68106846F27042AF
:103C1000C4F2020290425AD07A68106846F2280232
:103C2000C4F2020290424FD07A68106846F22842ED
:103C3000C4F20202904244D07A68106846F28802C8
:103C4000C4F20202904239D07A68106846F2884283
:103C5000C4F2020290422ED07A68106846F2400206
:103C6000C4F20202904223D07A68106846F24042C1
:103C7000C4F20202904218D07A68106846F2A0029C
:103C8000C4F2020290420DD07A68106846F2A04257
:103C9000C4F20202904202D14FF4002201E04FF040
:103CA000007201E04FF4002201E04FF4002201E035
:103CB0004FF4002201E04FF4007201E04FF4007273
:103CC00001E04FF4007201E04FF4007201E04FF0A8
:103CD000080201E04FF0080201E04FF0080201E0A5
:103CE0004FF008020A43DA60CBE17B681B681A4692
:103CF00046F2B803C4F202039A4240F293804FF4B2
:103D0000C843C4F202034FF4C842C4F202029268EC
:103D100011467A68106846F21002C4F2020290421C
:103D20007BD07A68106846F21042C4F202029042D8
:103D300070D07A68106846F27002C4F202029042B3
:103D400065D07A68106846F27042C4F2020290426E
:103D50005AD07A68106846F22802C4F202029042F1
:103D60004FD07A68106846F22842C4F202029042AC
:103D700044D07A68106846F28802C4F20202904287
:103D800039D07A68106846F28842C4F20202904242
:103D90002ED07A68106846F24002C4F202029042C5
:103DA00023D07A68106846F24042C4F20202904280
:103DB00018D07A68106846F2A002C4F2020290425B
:103DC0000DD07A68106846F2A042C4F20202904216
:103DD00002D14FF4002201E04FF0007201E04FF4F5
:103DE000002201E04FF4002201E04FF4002201E044
:103DF0004FF4007201E04FF4007201E04FF40072E2
:103E000001E04FF4007201E04FF0080201E04FF0D2
:103E1000080201E04FF0080201E04FF008020A43F7
:103E20009A602EE17B681B681A4646F25803C4F27A
:103E300002039A4240F293804FF4C043C4F202035B
:103E40004FF4C042C4F20202D26811467A68106888
:103E500046F21002C4F2020290427BD07A681068E7
:103E600046F21042C4F20202904270D07A681068A2
:103E700046F27002C4F20202904265D07A6810687D
:103E800046F27042C4F2020290425AD07A68106838
:103E900046F22802C4F2020290424FD07A681068BB
:103EA00046F22842C4F20202904244D07A68106876
:103EB00046F28802C4F20202904239D07A68106851
:103EC00046F28842C4F2020290422ED07A6810680C
:103ED00046F24002C4F20202904223D07A6810688F
:103EE00046F24042C4F20202904218D07A6810684A
:103EF00046F2A002C4F2020290420DD07A68106825
:103F000046F2A042C4F20202904202D14FF40022D3
:103F100001E04FF0007201E04FF4002201E04FF4A5
:103F2000002201E04FF4002201E04FF4007201E0B2
:103F30004FF4007201E04FF4007201E04FF40072A0
:103F400001E04FF0080201E04FF0080201E04FF0FD
:103F5000080201E04FF008020A43DA6091E04FF4F2
:103F6000C043C4F202034FF4C042C4F2020292689A
:103F700011467A68106846F21002C4F202029042BA
:103F80007BD07A68106846F21042C4F20202904276
:103F900070D07A68106846F27002C4F20202904251
:103FA00065D07A68106846F27042C4F2020290420C
:103FB0005AD07A68106846F22802C4F2020290428F
:103FC0004FD07A68106846F22842C4F2020290424A
:103FD00044D07A68106846F28802C4F20202904225
:103FE00039D07A68106846F28842C4F202029042E0
:103FF0002ED07A68106846F24002C4F20202904263
:1040000023D07A68106846F24042C4F2020290421D
:1040100018D07A68106846F2A002C4F202029042F8
:104020000DD07A68106846F2A042C4F202029042B3
:1040300002D14FF4002201E04FF0007201E04FF492
:10404000002201E04FF4002201E04FF4002201E0E1
:104050004FF4007201E04FF4007201E04FF400727F
:1040600001E04FF4007201E04FF0080201E04FF070
:10407000080201E04FF0080201E04FF008020A4395
:104080009A607B68DB6C43F001027B68DA647B68D2
:104090004FF0040283F835207B684FF0000283F86C
:1040A00034207B689B6C002B03D07B689B6C78680A
:1040B00098477B681B681A4646F25843C4F20203CD
:1040C0009A4240F29C804FF4C843C4F202035B68FA
:1040D0001A467B68196846F21003C4F2020399423B
:1040E00000F082807B68196846F21043C4F2020334
:1040F000994274D07B68196846F27003C4F20203D7
:10410000994267D07B68196846F27043C4F2020393
:1041100099425AD07B68196846F22803C4F2020318
:1041200099424FD07B68196846F22843C4F20203D3
:10413000994244D07B68196846F28803C4F20203AE
:10414000994239D07B68196846F28843C4F2020369
:1041500099422ED07B68196846F24003C4F20203EC
:10416000994223D07B68196846F24043C4F20203A7
:10417000994218D07B68196846F2A003C4F2020382
:1041800099420DD07B68196846F2A043C4F202033D
:10419000994202D14FF4803301E04FF4800301E0F3
:1041A0004FF4803301E04FF4803301E04FF480336B
:1041B00001E04FF0400301E04FF0400301E04FF019
:1041C000400301E04FF0400303E04FF00103C0F271
:1041D000800303E04FF00103C0F2800303E04FF0DF
:1041E0000103C0F2800303E04FF00103C0F280033B
:1041F0001340002B0CBF00230123DBB2E6E17B68F8
:104200001B681A4646F2B803C4F202039A4240F20F
:104210009C804FF4C843C4F202031B681A467B68B3
:10422000196846F21003C4F20203994200F082803A
:104230007B68196846F21043C4F20203994274D0B5
:104240007B68196846F27003C4F20203994267D092
:104250007B68196846F27043C4F2020399425AD04F
:104260007B68196846F22803C4F2020399424FD0D2
:104270007B68196846F22843C4F20203994244D08D
:104280007B68196846F28803C4F20203994239D068
:104290007B68196846F28843C4F2020399422ED023
:1042A0007B68196846F24003C4F20203994223D0A6
:1042B0007B68196846F24043C4F20203994218D061
:1042C0007B68196846F2A003C4F2020399420DD03C
:1042D0007B68196846F2A043C4F20203994202D1F6
:1042E0004FF4803301E04FF4800301E04FF480335A
:1042F00001E04FF4803301E04FF4803301E04FF0F0
:10430000400301E04FF0400301E04FF0400301E0C3
:104310004FF0400303E04FF00103C0F2800303E0DD
:104320004FF00103C0F2800303E04FF00103C0F23D
:10433000800303E04FF00103C0F280031340002B21
:104340000CBF00230123DBB240E17B681B681A46E7
:1043500046F25803C4F202039A4240F29C804FF4A2
:10436000C043C4F202035B681A467B68196846F2D0
:104370001003C4F20203994200F082807B6819683E
:1043800046F21043C4F20203994274D07B68196864
:1043900046F27003C4F20203994267D07B68196841
:1043A00046F27043C4F2020399425AD07B681968FE
:1043B00046F22803C4F2020399424FD07B68196881
:1043C00046F22843C4F20203994244D07B6819683C
:1043D00046F28803C4F20203994239D07B68196817
:1043E00046F28843C4F2020399422ED07B681968D2
:1043F00046F24003C4F20203994223D07B68196855
:1044000046F24043C4F20203994218D07B6819680F
:1044100046F2A003C4F2020399420DD07B681968EA
:1044200046F2A043C4F20203994202D14FF4803312
:1044300001E04FF4800301E04FF4803301E04FF4DA
:10444000803301E04FF4803301E04FF0400301E09E
:104450004FF0400301E04FF0400301E04FF0400314
:1044600003E04FF00103C0F2800303E04FF00103CB
:10447000C0F2800303E04FF00103C0F2800303E0C9
:104480004FF00103C0F280031340002B0CBF002348
:104490000123DBB29AE04FF4C043C4F202031B686D
:1044A0001A467B68196846F21003C4F20203994267
:1044B00000F082807B68196846F21043C4F2020360
:1044C000994274D07B68196846F27003C4F2020303
:1044D000994267D07B68196846F27043C4F20203C0
:1044E00099425AD07B68196846F22803C4F2020345
:1044F00099424FD07B68196846F22843C4F2020300
:10450000994244D07B68196846F28803C4F20203DA
:10451000994239D07B68196846F28843C4F2020395
:1045200099422ED07B68196846F24003C4F2020318
:10453000994223D07B68196846F24043C4F20203D3
:10454000994218D07B68196846F2A003C4F20203AE
:1045500099420DD07B68196846F2A043C4F2020369
:10456000994202D14FF4803301E04FF4800301E01F
:104570004FF4803301E04FF4803301E04FF4803397
:1045800001E04FF0400301E04FF0400301E04FF045
:10459000400301E04FF0400303E04FF00103C0F29D
:1045A000800303E04FF00103C0F2800303E04FF00B
:1045B0000103C0F2800303E04FF00103C0F2800367
:1045C0001340002B0CBF00230123DBB2002B00F0B3
:1045D000B5827B681B685B6903F08003002B00F0E9
:1045E000AD827B681B687A681268526922F080028B
:1045F0005A617B681B681A4646F25843C4F20203AC
:104600009A4240F29C804FF4C842C4F202024FF436
:10461000C843C4F20203DB6819467B68186846F297
:104620001003C4F20203984200F082807B6818688D
:1046300046F21043C4F20203984274D07B681868B3
:1046400046F27003C4F20203984267D07B68186890
:1046500046F27043C4F2020398425AD07B6818684D
:1046600046F22803C4F2020398424FD07B681868D0
:1046700046F22843C4F20203984244D07B6818688B
:1046800046F28803C4F20203984239D07B68186866
:1046900046F28843C4F2020398422ED07B68186821
:1046A00046F24003C4F20203984223D07B681868A4
:1046B00046F24043C4F20203984218D07B6818685F
:1046C00046F2A003C4F2020398420DD07B6818683A
:1046D00046F2A043C4F20203984202D14FF4803361
:1046E00001E04FF4800301E04FF4803301E04FF428
:1046F000803301E04FF4803301E04FF0400301E0EC
:104700004FF0400301E04FF0400301E04FF0400361
:1047100003E04FF00103C0F2800303E04FF0010318
:10472000C0F2800303E04FF00103C0F2800303E016
:104730004FF00103C0F280030B43D360E6E17B68D6
:104740001B681A4646F2B803C4F202039A4240F2CA
:104750009C804FF4C842C4F202024FF4C843C4F232
:1047600002039B6819467B68186846F21003C4F27E
:104770000203984200F082807B68186846F210437A
:10478000C4F20203984274D07B68186846F2700342
:10479000C4F20203984267D07B68186846F27043FF
:1047A000C4F2020398425AD07B68186846F2280384
:1047B000C4F2020398424FD07B68186846F228433F
:1047C000C4F20203984244D07B68186846F288031A
:1047D000C4F20203984239D07B68186846F28843D5
:1047E000C4F2020398422ED07B68186846F2400358
:1047F000C4F20203984223D07B68186846F2404313
:10480000C4F20203984218D07B68186846F2A003ED
:10481000C4F2020398420DD07B68186846F2A043A8
:10482000C4F20203984202D14FF4803301E04FF406
:10483000800301E04FF4803301E04FF4803301E066
:104840004FF4803301E04FF0400301E04FF04003AC
:1048500001E04FF0400301E04FF0400303E04FF070
:104860000103C0F2800303E04FF00103C0F28003B4
:1048700003E04FF00103C0F2800303E04FF00103B7
:10488000C0F280030B43936040E17B681B681A46CB
:1048900046F25803C4F202039A4240F29C804FF45D
:1048A000C042C4F202024FF4C043C4F20203DB6808
:1048B00019467B68186846F21003C4F20203984256
:1048C00000F082807B68186846F21043C4F202034D
:1048D000984274D07B68186846F27003C4F20203F1
:1048E000984267D07B68186846F27043C4F20203AE
:1048F00098425AD07B68186846F22803C4F2020333
:1049000098424FD07B68186846F22843C4F20203ED
:10491000984244D07B68186846F28803C4F20203C8
:10492000984239D07B68186846F28843C4F2020383
:1049300098422ED07B68186846F24003C4F2020306
:10494000984223D07B68186846F24043C4F20203C1
:10495000984218D07B68186846F2A003C4F202039C
:1049600098420DD07B68186846F2A043C4F2020357
:10497000984202D14FF4803301E04FF4800301E00C
:104980004FF4803301E04FF4803301E04FF4803383
:1049900001E04FF0400301E04FF0400301E04FF031
:1049A000400301E04FF0400303E04FF00103C0F289
:1049B000800303E04FF00103C0F2800303E04FF0F7
:1049C0000103C0F2800303E04FF00103C0F2800353
:1049D0000B43D3609AE04FF4C042C4F202024FF49A
:1049E000C043C4F202039B6819467B68186846F20C
:1049F0001003C4F20203984200F082807B681868BA
:104A000046F21043C4F20203984274D07B681868DF
:104A100046F27003C4F20203984267D07B681868BC
:104A200046F27043C4F2020398425AD07B68186879
:104A300046F22803C4F2020398424FD07B681868FC
:104A400046F22843C4F20203984244D07B681868B7
:104A500046F28803C4F20203984239D07B68186892
:104A600046F28843C4F2020398422ED07B6818684D
:104A700046F24003C4F20203984223D07B681868D0
:104A800046F24043C4F20203984218D07B6818688B
:104A900046F2A003C4F2020398420DD07B68186866
:104AA00046F2A043C4F20203984202D14FF480338D
:104AB00001E04FF4800301E04FF4803301E04FF454
:104AC000803301E04FF4803301E04FF0400301E018
:104AD0004FF0400301E04FF0400301E04FF040038E
:104AE00003E04FF00103C0F2800303E04FF0010345
:104AF000C0F2800303E04FF00103C0F2800303E043
:104B00004FF00103C0F280030B4393607B68DB6CC2
:104B100043F002027B68DA647B684FF0040283F89A
:104B200035207B684FF0000283F834207B689B6C53
:104B3000002B03D07B689B6C786898477B681B6868
:104B40001A4646F25843C4F202039A4240F29C804D
:104B50004FF4C843C4F202035B681A467B681968C5
:104B600046F21003C4F20203994200F082807B688F
:104B7000196846F21043C4F20203994274D07B686C
:104B8000196846F27003C4F20203994267D07B6849
:104B9000196846F27043C4F2020399425AD07B6806
:104BA000196846F22803C4F2020399424FD07B6889
:104BB000196846F22843C4F20203994244D07B6844
:104BC000196846F28803C4F20203994239D07B681F
:104BD000196846F28843C4F2020399422ED07B68DA
:104BE000196846F24003C4F20203994223D07B685D
:104BF000196846F24043C4F20203994218D07B6818
:104C0000196846F2A003C4F2020399420DD07B68F2
:104C1000196846F2A043C4F20203994202D14FF44C
:104C2000802301E04FF0807301E04FF4802301E026
:104C30004FF4802301E04FF4802301E04FF48073B0
:104C400001E04FF4807301E04FF4807301E04FF412
:104C5000807303E04FF00403C0F2800303E04FF0E1
:104C60000403C0F2800303E04FF00403C0F28003AA
:104C700003E04FF00403C0F280031340002B0CBF8D
:104C800000230123DBB2E6E17B681B681A4646F28B
:104C9000B803C4F202039A4240F29C804FF4C84326
:104CA000C4F202031B681A467B68196846F21003B7
:104CB000C4F20203994200F082807B68196846F2D0
:104CC0001043C4F20203994274D07B68196846F21B
:104CD0007003C4F20203994267D07B68196846F2F8
:104CE0007043C4F2020399425AD07B68196846F2B5
:104CF0002803C4F2020399424FD07B68196846F238
:104D00002843C4F20203994244D07B68196846F2F2
:104D10008803C4F20203994239D07B68196846F2CD
:104D20008843C4F2020399422ED07B68196846F288
:104D30004003C4F20203994223D07B68196846F20B
:104D40004043C4F20203994218D07B68196846F2C6
:104D5000A003C4F2020399420DD07B68196846F2A1
:104D6000A043C4F20203994202D14FF4802301E030
:104D70004FF0807301E04FF4802301E04FF4802373
:104D800001E04FF4802301E04FF4807301E04FF421
:104D9000807301E04FF4807301E04FF4807303E00F
:104DA0004FF00403C0F2800303E04FF00403C0F2AD
:104DB000800303E04FF00403C0F2800303E04FF0F0
:104DC0000403C0F280031340002B0CBF0023012317
:104DD000DBB240E17B681B681A4646F25803C4F216
:104DE00002039A4240F29C804FF4C043C4F2020393
:104DF0005B681A467B68196846F21003C4F2020326
:104E0000994200F082807B68196846F21043C4F230
:104E10000203994274D07B68196846F27003C4F2A9
:104E20000203994267D07B68196846F27043C4F266
:104E3000020399425AD07B68196846F22803C4F2EB
:104E4000020399424FD07B68196846F22843C4F2A6
:104E50000203994244D07B68196846F28803C4F281
:104E60000203994239D07B68196846F28843C4F23C
:104E7000020399422ED07B68196846F24003C4F2BF
:104E80000203994223D07B68196846F24043C4F27A
:104E90000203994218D07B68196846F2A003C4F255
:104EA000020399420DD07B68196846F2A043C4F210
:104EB0000203994202D14FF4802301E04FF0807346
:104EC00001E04FF4802301E04FF4802301E04FF430
:104ED000802301E04FF4807301E04FF4807301E020
:104EE0004FF4807301E04FF4807303E04FF004034C
:104EF000C0F2800303E04FF00403C0F2800303E03C
:104F00004FF00403C0F2800303E04FF00403C0F24B
:104F100080031340002B0CBF00230123DBB29AE077
:104F20004FF4C043C4F202031B681A467B68196839
:104F300046F21003C4F20203994200F082807B68BB
:104F4000196846F21043C4F20203994274D07B6898
:104F5000196846F27003C4F20203994267D07B6875
:104F6000196846F27043C4F2020399425AD07B6832
:104F7000196846F22803C4F2020399424FD07B68B5
:104F8000196846F22843C4F20203994244D07B6870
:104F9000196846F28803C4F20203994239D07B684B
:104FA000196846F28843C4F2020399422ED07B6806
:104FB000196846F24003C4F20203994223D07B6889
:104FC000196846F24043C4F20203994218D07B6844
:104FD000196846F2A003C4F2020399420DD07B681F
:104FE000196846F2A043C4F20203994202D14FF479
:104FF000802301E04FF0807301E04FF4802301E053
:105000004FF4802301E04FF4802301E04FF48073DC
:1050100001E04FF4807301E04FF4807301E04FF43E
:10502000807303E04FF00403C0F2800303E04FF00D
:105030000403C0F2800303E04FF00403C0F28003D6
:1050400003E04FF00403C0F280031340002B0CBFB9
:1050500000230123DBB2002B00F0B5827B681B68C4
:105060001B6803F00203002B00F0AD827B681B6815
:105070007A681268126822F002021A607B681B6864
:105080001A4646F25843C4F202039A4240F29C8008
:105090004FF4C842C4F202024FF4C843C4F2020300
:1050A000DB6819467B68186846F21003C4F20203F5
:1050B000984200F082807B68186846F21043C4F280
:1050C0000203984274D07B68186846F27003C4F2F9
:1050D0000203984267D07B68186846F27043C4F2B6
:1050E000020398425AD07B68186846F22803C4F23B
:1050F000020398424FD07B68186846F22843C4F2F6
:105100000203984244D07B68186846F28803C4F2D0
:105110000203984239D07B68186846F28843C4F28B
:10512000020398422ED07B68186846F24003C4F20E
:105130000203984223D07B68186846F24043C4F2C9
:105140000203984218D07B68186846F2A003C4F2A4
:10515000020398420DD07B68186846F2A043C4F25F
:105160000203984202D14FF4802301E04FF0807394
:1051700001E04FF4802301E04FF4802301E04FF47D
:10518000802301E04FF4807301E04FF4807301E06D
:105190004FF4807301E04FF4807303E04FF0040399
:1051A000C0F2800303E04FF00403C0F2800303E089
:1051B0004FF00403C0F2800303E04FF00403C0F299
:1051C00080030B43D360E6E17B681B681A4646F216
:1051D000B803C4F202039A4240F29C804FF4C842E2
:1051E000C4F202024FF4C843C4F202039B6819469A
:1051F0007B68186846F21003C4F20203984200F07C
:1052000082807B68186846F21043C4F20203984219
:1052100074D07B68186846F27003C4F202039842A7
:1052200067D07B68186846F27043C4F20203984264
:105230005AD07B68186846F22803C4F202039842E9
:105240004FD07B68186846F22843C4F202039842A4
:1052500044D07B68186846F28803C4F2020398427F
:1052600039D07B68186846F28843C4F2020398423A
:105270002ED07B68186846F24003C4F202039842BD
:1052800023D07B68186846F24043C4F20203984278
:1052900018D07B68186846F2A003C4F20203984253
:1052A0000DD07B68186846F2A043C4F2020398420E
:1052B00002D14FF4802301E04FF0807301E04FF4FE
:1052C000802301E04FF4802301E04FF4802301E0CC
:1052D0004FF4807301E04FF4807301E04FF480736A
:1052E00001E04FF4807303E04FF00403C0F2800349
:1052F00003E04FF00403C0F2800303E04FF0040327
:10530000C0F2800303E04FF00403C0F280030B43BC
:10531000936040E17B681B681A4646F25803C4F26A
:1053200002039A4240F29C804FF4C042C4F202024F
:105330004FF4C043C4F20203DB6819467B68186867
:1053400046F21003C4F20203984200F082807B68A8
:10535000186846F21043C4F20203984274D07B6886
:10536000186846F27003C4F20203984267D07B6863
:10537000186846F27043C4F2020398425AD07B6820
:10538000186846F22803C4F2020398424FD07B68A3
:10539000186846F22843C4F20203984244D07B685E
:1053A000186846F28803C4F20203984239D07B6839
:1053B000186846F28843C4F2020398422ED07B68F4
:1053C000186846F24003C4F20203984223D07B6877
:1053D000186846F24043C4F20203984218D07B6832
:1053E000186846F2A003C4F2020398420DD07B680D
:1053F000186846F2A043C4F20203984202D14FF467
:10540000802301E04FF0807301E04FF4802301E03E
:105410004FF4802301E04FF4802301E04FF48073C8
:1054200001E04FF4807301E04FF4807301E04FF42A
:10543000807303E04FF00403C0F2800303E04FF0F9
:105440000403C0F2800303E04FF00403C0F28003C2
:1054500003E04FF00403C0F280030B43D3609AE0F3
:105460004FF4C042C4F202024FF4C043C4F202033C
:105470009B6819467B68186846F21003C4F2020361
:10548000984200F082807B68186846F21043C4F2AC
:105490000203984274D07B68186846F27003C4F225
:1054A0000203984267D07B68186846F27043C4F2E2
:1054B000020398425AD07B68186846F22803C4F267
:1054C000020398424FD07B68186846F22843C4F222
:1054D0000203984244D07B68186846F28803C4F2FD
:1054E0000203984239D07B68186846F28843C4F2B8
:1054F000020398422ED07B68186846F24003C4F23B
:105500000203984223D07B68186846F24043C4F2F5
:105510000203984218D07B68186846F2A003C4F2D0
:10552000020398420DD07B68186846F2A043C4F28B
:105530000203984202D14FF4802301E04FF08073C0
:1055400001E04FF4802301E04FF4802301E04FF4A9
:10555000802301E04FF4807301E04FF4807301E099
:105560004FF4807301E04FF4807303E04FF00403C5
:10557000C0F2800303E04FF00403C0F2800303E0B5
:105580004FF00403C0F2800303E04FF00403C0F2C5
:1055900080030B4393607B68DB6C43F004027B6801
:1055A000DA647B684FF0040283F835207B684FF0A3
:1055B000000283F834207B689B6C002B03D07B684F
:1055C0009B6C786898477B681B681A4646F258437C
:1055D000C4F202039A4240F293804FF4C843C4F2EB
:1055E00002035B681A467B68196846F21003C4F22E
:1055F000020399427BD07B68196846F21043C4F2DB
:105600000203994270D07B68196846F27003C4F2B5
:105610000203994265D07B68196846F27043C4F270
:10562000020399425AD07B68196846F22803C4F2F3
:10563000020399424FD07B68196846F22843C4F2AE
:105640000203994244D07B68196846F28803C4F289
:105650000203994239D07B68196846F28843C4F244
:10566000020399422ED07B68196846F24003C4F2C7
:105670000203994223D07B68196846F24043C4F282
:105680000203994218D07B68196846F2A003C4F25D
:10569000020399420DD07B68196846F2A043C4F218
:1056A0000203994202D14FF4801301E04FF080636E
:1056B00001E04FF4801301E04FF4801301E04FF458
:1056C000801301E04FF4806301E04FF4806301E058
:1056D0004FF4806301E04FF4806301E04FF010036A
:1056E00001E04FF0100301E04FF0100301E04FF034
:1056F00010031340002B0CBF00230123DBB2CBE1CE
:105700007B681B681A4646F2B803C4F202039A4249
:1057100040F293804FF4C843C4F202031B681A4658
:105720007B68196846F21003C4F2020399427BD0E9
:105730007B68196846F21043C4F20203994270D0A4
:105740007B68196846F27003C4F20203994265D07F
:105750007B68196846F27043C4F2020399425AD03A
:105760007B68196846F22803C4F2020399424FD0BD
:105770007B68196846F22843C4F20203994244D078
:105780007B68196846F28803C4F20203994239D053
:105790007B68196846F28843C4F2020399422ED00E
:1057A0007B68196846F24003C4F20203994223D091
:1057B0007B68196846F24043C4F20203994218D04C
:1057C0007B68196846F2A003C4F2020399420DD027
:1057D0007B68196846F2A043C4F20203994202D1E1
:1057E0004FF4801301E04FF0806301E04FF4801329
:1057F00001E04FF4801301E04FF4801301E04FF417
:10580000806301E04FF4806301E04FF4806301E0C6
:105810004FF4806301E04FF0100301E04FF01003FC
:1058200001E04FF0100301E04FF010031340002B94
:105830000CBF00230123DBB22EE17B681B681A46F4
:1058400046F25803C4F202039A4240F293804FF4A6
:10585000C043C4F202035B681A467B68196846F2CB
:105860001003C4F2020399427BD07B68196846F2A8
:105870001043C4F20203994270D07B68196846F263
:105880007003C4F20203994265D07B68196846F23E
:105890007043C4F2020399425AD07B68196846F2F9
:1058A0002803C4F2020399424FD07B68196846F27C
:1058B0002843C4F20203994244D07B68196846F237
:1058C0008803C4F20203994239D07B68196846F212
:1058D0008843C4F2020399422ED07B68196846F2CD
:1058E0004003C4F20203994223D07B68196846F250
:1058F0004043C4F20203994218D07B68196846F20B
:10590000A003C4F2020399420DD07B68196846F2E5
:10591000A043C4F20203994202D14FF4801301E084
:105920004FF0806301E04FF4801301E04FF48013E7
:1059300001E04FF4801301E04FF4806301E04FF485
:10594000806301E04FF4806301E04FF4806301E085
:105950004FF0100301E04FF0100301E04FF010038F
:1059600001E04FF010031340002B0CBF0023012374
:10597000DBB291E04FF4C043C4F202031B681A4645
:105980007B68196846F21003C4F2020399427BD087
:105990007B68196846F21043C4F20203994270D042
:1059A0007B68196846F27003C4F20203994265D01D
:1059B0007B68196846F27043C4F2020399425AD0D8
:1059C0007B68196846F22803C4F2020399424FD05B
:1059D0007B68196846F22843C4F20203994244D016
:1059E0007B68196846F28803C4F20203994239D0F1
:1059F0007B68196846F28843C4F2020399422ED0AC
:105A00007B68196846F24003C4F20203994223D02E
:105A10007B68196846F24043C4F20203994218D0E9
:105A20007B68196846F2A003C4F2020399420DD0C4
:105A30007B68196846F2A043C4F20203994202D17E
:105A40004FF4801301E04FF0806301E04FF48013C6
:105A500001E04FF4801301E04FF4801301E04FF4B4
:105A6000806301E04FF4806301E04FF4806301E064
:105A70004FF4806301E04FF0100301E04FF010039A
:105A800001E04FF0100301E04FF010031340002B32
:105A90000CBF00230123DBB2002B00F019857B68CB
:105AA0001B681B6803F00803002B00F011857B685E
:105AB0001B681B6803F48023002B00F084827B6842
:105AC0001B681A4646F25843C4F202039A4240F257
:105AD00093804FF4C843C4F202034FF4C842C4F2A7
:105AE0000202D26811467A68106846F21002C4F2C7
:105AF000020290427BD07A68106846F21042C4F2EB
:105B00000202904270D07A68106846F27002C4F2C5
:105B10000202904265D07A68106846F27042C4F280
:105B2000020290425AD07A68106846F22802C4F203
:105B3000020290424FD07A68106846F22842C4F2BE
:105B40000202904244D07A68106846F28802C4F299
:105B50000202904239D07A68106846F28842C4F254
:105B6000020290422ED07A68106846F24002C4F2D7
:105B70000202904223D07A68106846F24042C4F292
:105B80000202904218D07A68106846F2A002C4F26D
:105B9000020290420DD07A68106846F2A042C4F228
:105BA0000202904202D14FF4801201E04FF0806275
:105BB00001E04FF4801201E04FF4801201E04FF455
:105BC000801201E04FF4806201E04FF4806201E056
:105BD0004FF4806201E04FF4806201E04FF0100268
:105BE00001E04FF0100201E04FF0100201E04FF031
:105BF00010020A43DA60CBE17B681B681A4646F262
:105C0000B803C4F202039A4240F293804FF4C843AF
:105C1000C4F202034FF4C842C4F202029268114671
:105C20007A68106846F21002C4F2020290427BD0F9
:105C30007A68106846F21042C4F20202904270D0B4
:105C40007A68106846F27002C4F20202904265D08F
:105C50007A68106846F27042C4F2020290425AD04A
:105C60007A68106846F22802C4F2020290424FD0CD
:105C70007A68106846F22842C4F20202904244D088
:105C80007A68106846F28802C4F20202904239D063
:105C90007A68106846F28842C4F2020290422ED01E
:105CA0007A68106846F24002C4F20202904223D0A1
:105CB0007A68106846F24042C4F20202904218D05C
:105CC0007A68106846F2A002C4F2020290420DD037
:105CD0007A68106846F2A042C4F20202904202D1F1
:105CE0004FF4801201E04FF0806201E04FF4801227
:105CF00001E04FF4801201E04FF4801201E04FF414
:105D0000806201E04FF4806201E04FF4806201E0C4
:105D10004FF4806201E04FF0100201E04FF01002FA
:105D200001E04FF0100201E04FF010020A439A60C8
:105D30002EE17B681B681A4646F25803C4F2020340
:105D40009A4240F293804FF4C043C4F202034FF4EE
:105D5000C042C4F20202D26811467A68106846F264
:105D60001002C4F2020290427BD07A68106846F2B8
:105D70001042C4F20202904270D07A68106846F273
:105D80007002C4F20202904265D07A68106846F24E
:105D90007042C4F2020290425AD07A68106846F209
:105DA0002802C4F2020290424FD07A68106846F28C
:105DB0002842C4F20202904244D07A68106846F247
:105DC0008802C4F20202904239D07A68106846F222
:105DD0008842C4F2020290422ED07A68106846F2DD
:105DE0004002C4F20202904223D07A68106846F260
:105DF0004042C4F20202904218D07A68106846F21B
:105E0000A002C4F2020290420DD07A68106846F2F5
:105E1000A042C4F20202904202D14FF4801201E08B
:105E20004FF0806201E04FF4801201E04FF48012E5
:105E300001E04FF4801201E04FF4806201E04FF482
:105E4000806201E04FF4806201E04FF4806201E083
:105E50004FF0100201E04FF0100201E04FF010028D
:105E600001E04FF010020A43DA6091E04FF4C043C2
:105E7000C4F202034FF4C042C4F202029268114617
:105E80007A68106846F21002C4F2020290427BD097
:105E90007A68106846F21042C4F20202904270D052
:105EA0007A68106846F27002C4F20202904265D02D
:105EB0007A68106846F27042C4F2020290425AD0E8
:105EC0007A68106846F22802C4F2020290424FD06B
:105ED0007A68106846F22842C4F20202904244D026
:105EE0007A68106846F28802C4F20202904239D001
:105EF0007A68106846F28842C4F2020290422ED0BC
:105F00007A68106846F24002C4F20202904223D03E
:105F10007A68106846F24042C4F20202904218D0F9
:105F20007A68106846F2A002C4F2020290420DD0D4
:105F30007A68106846F2A042C4F20202904202D18E
:105F40004FF4801201E04FF0806201E04FF48012C4
:105F500001E04FF4801201E04FF4801201E04FF4B1
:105F6000806201E04FF4806201E04FF4806201E062
:105F70004FF4806201E04FF0100201E04FF0100298
:105F800001E04FF0100201E04FF010020A439A6066
:105F90007B681B681B6803F40023002B05D17B681A
:105FA0004FF0310283F835208AE27B681B681B685A
:105FB00003F40023002B00F083827B684FF0410242
:105FC00083F835207CE27B681B681B6803F48073D0
:105FD000002B07D17B681B687A681268126822F070
:105FE00008021A607B681B681A4646F25843C4F2DE
:105FF00002039A4240F293804FF4C843C4F2020372
:106000004FF4C842C4F20202D26811467A6810689E
:1060100046F21002C4F2020290427BD07A68106805
:1060200046F21042C4F20202904270D07A681068C0
:1060300046F27002C4F20202904265D07A6810689B
:1060400046F27042C4F2020290425AD07A68106856
:1060500046F22802C4F2020290424FD07A681068D9
:1060600046F22842C4F20202904244D07A68106894
:1060700046F28802C4F20202904239D07A6810686F
:1060800046F28842C4F2020290422ED07A6810682A
:1060900046F24002C4F20202904223D07A681068AD
:1060A00046F24042C4F20202904218D07A68106868
:1060B00046F2A002C4F2020290420DD07A68106843
:1060C00046F2A042C4F20202904202D14FF4801282
:1060D00001E04FF0806201E04FF4801201E04FF4E4
:1060E000801201E04FF4801201E04FF4806201E081
:1060F0004FF4806201E04FF4806201E04FF480626F
:1061000001E04FF0100201E04FF0100201E04FF00B
:10611000100201E04FF010020A43DA60CBE17B6825
:106120001B681A4646F2B803C4F202039A4240F2D0
:1061300093804FF4C843C4F202034FF4C842C4F240
:106140000202926811467A68106846F21002C4F2A0
:10615000020290427BD07A68106846F21042C4F284
:106160000202904270D07A68106846F27002C4F25F
:106170000202904265D07A68106846F27042C4F21A
:10618000020290425AD07A68106846F22802C4F29D
:10619000020290424FD07A68106846F22842C4F258
:1061A0000202904244D07A68106846F28802C4F233
:1061B0000202904239D07A68106846F28842C4F2EE
:1061C000020290422ED07A68106846F24002C4F271
:1061D0000202904223D07A68106846F24042C4F22C
:1061E0000202904218D07A68106846F2A002C4F207
:1061F000020290420DD07A68106846F2A042C4F2C2
:106200000202904202D14FF4801201E04FF080620E
:1062100001E04FF4801201E04FF4801201E04FF4EE
:10622000801201E04FF4806201E04FF4806201E0EF
:106230004FF4806201E04FF4806201E04FF0100201
:1062400001E04FF0100201E04FF0100201E04FF0CA
:1062500010020A439A602EE17B681B681A4646F2D8
:106260005803C4F202039A4240F293804FF4C043B1
:10627000C4F202034FF4C042C4F20202D2681146D3
:106280007A68106846F21002C4F2020290427BD093
:106290007A68106846F21042C4F20202904270D04E
:1062A0007A68106846F27002C4F20202904265D029
:1062B0007A68106846F27042C4F2020290425AD0E4
:1062C0007A68106846F22802C4F2020290424FD067
:1062D0007A68106846F22842C4F20202904244D022
:1062E0007A68106846F28802C4F20202904239D0FD
:1062F0007A68106846F28842C4F2020290422ED0B8
:106300007A68106846F24002C4F20202904223D03A
:106310007A68106846F24042C4F20202904218D0F5
:106320007A68106846F2A002C4F2020290420DD0D0
:106330007A68106846F2A042C4F20202904202D18A
:106340004FF4801201E04FF0806201E04FF48012C0
:1063500001E04FF4801201E04FF4801201E04FF4AD
:10636000806201E04FF4806201E04FF4806201E05E
:106370004FF4806201E04FF0100201E04FF0100294
:1063800001E04FF0100201E04FF010020A43DA6022
:1063900091E04FF4C043C4F202034FF4C042C4F290
:1063A0000202926811467A68106846F21002C4F23E
:1063B000020290427BD07A68106846F21042C4F222
:1063C0000202904270D07A68106846F27002C4F2FD
:1063D0000202904265D07A68106846F27042C4F2B8
:1063E000020290425AD07A68106846F22802C4F23B
:1063F000020290424FD07A68106846F22842C4F2F6
:106400000202904244D07A68106846F28802C4F2D0
:106410000202904239D07A68106846F28842C4F28B
:10642000020290422ED07A68106846F24002C4F20E
:106430000202904223D07A68106846F24042C4F2C9
:106440000202904218D07A68106846F2A002C4F2A4
:10645000020290420DD07A68106846F2A042C4F25F
:106460000202904202D14FF4801201E04FF08062AC
:1064700001E04FF4801201E04FF4801201E04FF48C
:10648000801201E04FF4806201E04FF4806201E08D
:106490004FF4806201E04FF4806201E04FF010029F
:1064A00001E04FF0100201E04FF0100201E04FF068
:1064B00010020A439A607B684FF0310283F835205E
:1064C0007B681B6C002B03D07B681B6C786898473B
:1064D0007B681B681A4646F25843C4F202039A428C
:1064E00040F293804FF4C843C4F202035B681A463B
:1064F0007B68196846F21003C4F2020399427BD00C
:106500007B68196846F21043C4F20203994270D0C6
:106510007B68196846F27003C4F20203994265D0A1
:106520007B68196846F27043C4F2020399425AD05C
:106530007B68196846F22803C4F2020399424FD0DF
:106540007B68196846F22843C4F20203994244D09A
:106550007B68196846F28803C4F20203994239D075
:106560007B68196846F28843C4F2020399422ED030
:106570007B68196846F24003C4F20203994223D0B3
:106580007B68196846F24043C4F20203994218D06E
:106590007B68196846F2A003C4F2020399420DD049
:1065A0007B68196846F2A043C4F20203994202D103
:1065B0004FF4001301E04FF0006301E04FF40013CB
:1065C00001E04FF4001301E04FF4001301E04FF439
:1065D000006301E04FF4006301E04FF4006301E069
:1065E0004FF4006301E04FF0200301E04FF020037F
:1065F00001E04FF0200301E04FF020031340002B97
:106600000CBF00230123DBB2CBE17B681B681A4679
:1066100046F2B803C4F202039A4240F293804FF468
:10662000C843C4F202031B681A467B68196846F225
:106630001003C4F2020399427BD07B68196846F2CA
:106640001043C4F20203994270D07B68196846F285
:106650007003C4F20203994265D07B68196846F260
:106660007043C4F2020399425AD07B68196846F21B
:106670002803C4F2020399424FD07B68196846F29E
:106680002843C4F20203994244D07B68196846F259
:106690008803C4F20203994239D07B68196846F234
:1066A0008843C4F2020399422ED07B68196846F2EF
:1066B0004003C4F20203994223D07B68196846F272
:1066C0004043C4F20203994218D07B68196846F22D
:1066D000A003C4F2020399420DD07B68196846F208
:1066E000A043C4F20203994202D14FF4001301E027
:1066F0004FF0006301E04FF4001301E04FF400138A
:1067000001E04FF4001301E04FF4006301E04FF4A7
:10671000006301E04FF4006301E04FF4006301E027
:106720004FF0200301E04FF0200301E04FF0200381
:1067300001E04FF020031340002B0CBF0023012386
:10674000DBB22EE17B681B681A4646F25803C4F29E
:1067500002039A4240F293804FF4C043C4F2020312
:106760005B681A467B68196846F21003C4F202039C
:1067700099427BD07B68196846F21043C4F2020349
:10678000994270D07B68196846F27003C4F2020324
:10679000994265D07B68196846F27043C4F20203DF
:1067A00099425AD07B68196846F22803C4F2020362
:1067B00099424FD07B68196846F22843C4F202031D
:1067C000994244D07B68196846F28803C4F20203F8
:1067D000994239D07B68196846F28843C4F20203B3
:1067E00099422ED07B68196846F24003C4F2020336
:1067F000994223D07B68196846F24043C4F20203F1
:10680000994218D07B68196846F2A003C4F20203CB
:1068100099420DD07B68196846F2A043C4F2020386
:10682000994202D14FF4001301E04FF0006301E000
:106830004FF4001301E04FF4001301E04FF4001394
:1068400001E04FF4006301E04FF4006301E04FF416
:10685000006301E04FF4006301E04FF0200301E02A
:106860004FF0200301E04FF0200301E04FF0200340
:106870001340002B0CBF00230123DBB291E04FF447
:10688000C043C4F202031B681A467B68196846F2CB
:106890001003C4F2020399427BD07B68196846F268
:1068A0001043C4F20203994270D07B68196846F223
:1068B0007003C4F20203994265D07B68196846F2FE
:1068C0007043C4F2020399425AD07B68196846F2B9
:1068D0002803C4F2020399424FD07B68196846F23C
:1068E0002843C4F20203994244D07B68196846F2F7
:1068F0008803C4F20203994239D07B68196846F2D2
:106900008843C4F2020399422ED07B68196846F28C
:106910004003C4F20203994223D07B68196846F20F
:106920004043C4F20203994218D07B68196846F2CA
:10693000A003C4F2020399420DD07B68196846F2A5
:10694000A043C4F20203994202D14FF4001301E0C4
:106950004FF0006301E04FF4001301E04FF4001327
:1069600001E04FF4001301E04FF4006301E04FF445
:10697000006301E04FF4006301E04FF4006301E0C5
:106980004FF0200301E04FF0200301E04FF020031F
:1069900001E04FF020031340002B0CBF0023012324
:1069A000DBB2002B00F02B857B681B681B6803F0B3
:1069B0001003002B00F023857B681B681B6803F421
:1069C0008023002B00F08C827B681B681A4646F2FD
:1069D0005843C4F202039A4240F293804FF4C843F2
:1069E000C4F202034FF4C842C4F20202D268114654
:1069F0007A68106846F21002C4F2020290427BD01C
:106A00007A68106846F21042C4F20202904270D0D6
:106A10007A68106846F27002C4F20202904265D0B1
:106A20007A68106846F27042C4F2020290425AD06C
:106A30007A68106846F22802C4F2020290424FD0EF
:106A40007A68106846F22842C4F20202904244D0AA
:106A50007A68106846F28802C4F20202904239D085
:106A60007A68106846F28842C4F2020290422ED040
:106A70007A68106846F24002C4F20202904223D0C3
:106A80007A68106846F24042C4F20202904218D07E
:106A90007A68106846F2A002C4F2020290420DD059
:106AA0007A68106846F2A042C4F20202904202D113
:106AB0004FF4001201E04FF0006201E04FF40012C9
:106AC00001E04FF4001201E04FF4001201E04FF436
:106AD000006201E04FF4006201E04FF4006201E067
:106AE0004FF4006201E04FF0200201E04FF020027D
:106AF00001E04FF0200201E04FF020020A43DA608B
:106B0000CBE17B681B681A4646F2B803C4F2020365
:106B10009A4240F293804FF4C843C4F202034FF408
:106B2000C842C4F20202926811467A68106846F2BE
:106B30001002C4F2020290427BD07A68106846F2DA
:106B40001042C4F20202904270D07A68106846F295
:106B50007002C4F20202904265D07A68106846F270
:106B60007042C4F2020290425AD07A68106846F22B
:106B70002802C4F2020290424FD07A68106846F2AE
:106B80002842C4F20202904244D07A68106846F269
:106B90008802C4F20202904239D07A68106846F244
:106BA0008842C4F2020290422ED07A68106846F2FF
:106BB0004002C4F20202904223D07A68106846F282
:106BC0004042C4F20202904218D07A68106846F23D
:106BD000A002C4F2020290420DD07A68106846F218
:106BE000A042C4F20202904202D14FF4001201E02E
:106BF0004FF0006201E04FF4001201E04FF4001288
:106C000001E04FF4001201E04FF4006201E04FF4A4
:106C1000006201E04FF4006201E04FF4006201E025
:106C20004FF0200201E04FF0200201E04FF020027F
:106C300001E04FF020020A439A602EE17B681B6856
:106C40001A4646F25803C4F202039A4240F2938075
:106C50004FF4C043C4F202034FF4C042C4F2020234
:106C6000D26811467A68106846F21002C4F2020235
:106C700090427BD07A68106846F21042C4F2020259
:106C8000904270D07A68106846F27002C4F2020234
:106C9000904265D07A68106846F27042C4F20202EF
:106CA00090425AD07A68106846F22802C4F2020272
:106CB00090424FD07A68106846F22842C4F202022D
:106CC000904244D07A68106846F28802C4F2020208
:106CD000904239D07A68106846F28842C4F20202C3
:106CE00090422ED07A68106846F24002C4F2020246
:106CF000904223D07A68106846F24042C4F2020201
:106D0000904218D07A68106846F2A002C4F20202DB
:106D100090420DD07A68106846F2A042C4F2020296
:106D2000904202D14FF4001201E04FF0006201E006
:106D30004FF4001201E04FF4001201E04FF4001292
:106D400001E04FF4006201E04FF4006201E04FF413
:106D5000006201E04FF4006201E04FF0200201E028
:106D60004FF0200201E04FF0200201E04FF020023E
:106D70000A43DA6091E04FF4C043C4F202034FF4D7
:106D8000C042C4F20202926811467A68106846F264
:106D90001002C4F2020290427BD07A68106846F278
:106DA0001042C4F20202904270D07A68106846F233
:106DB0007002C4F20202904265D07A68106846F20E
:106DC0007042C4F2020290425AD07A68106846F2C9
:106DD0002802C4F2020290424FD07A68106846F24C
:106DE0002842C4F20202904244D07A68106846F207
:106DF0008802C4F20202904239D07A68106846F2E2
:106E00008842C4F2020290422ED07A68106846F29C
:106E10004002C4F20202904223D07A68106846F21F
:106E20004042C4F20202904218D07A68106846F2DA
:106E3000A002C4F2020290420DD07A68106846F2B5
:106E4000A042C4F20202904202D14FF4001201E0CB
:106E50004FF0006201E04FF4001201E04FF4001225
:106E600001E04FF4001201E04FF4006201E04FF442
:106E7000006201E04FF4006201E04FF4006201E0C3
:106E80004FF0200201E04FF0200201E04FF020021D
:106E900001E04FF020020A439A607B681B681B6880
:106EA00003F40023002B09D17B685B6C002B00F0FE
:106EB000A6827B685B6C78689847A0E27B681B6859
:106EC0001B6803F40023002B00F099827B68DB6BC6
:106ED000002B00F094827B68DB6B786898478EE229
:106EE0007B681B681B6803F48073002B07D17B68E9
:106EF0001B687A681268126822F010021A607B68B8
:106F00001B681A4646F25843C4F202039A4240F202
:106F100093804FF4C843C4F202034FF4C842C4F252
:106F20000202D26811467A68106846F21002C4F272
:106F3000020290427BD07A68106846F21042C4F296
:106F40000202904270D07A68106846F27002C4F271
:106F50000202904265D07A68106846F27042C4F22C
:106F6000020290425AD07A68106846F22802C4F2AF
:106F7000020290424FD07A68106846F22842C4F26A
:106F80000202904244D07A68106846F28802C4F245
:106F90000202904239D07A68106846F28842C4F200
:106FA000020290422ED07A68106846F24002C4F283
:106FB0000202904223D07A68106846F24042C4F23E
:106FC0000202904218D07A68106846F2A002C4F219
:106FD000020290420DD07A68106846F2A042C4F2D4
:106FE0000202904202D14FF4001201E04FF0006221
:106FF00001E04FF4001201E04FF4001201E04FF401
:10700000001201E04FF4006201E04FF4006201E081
:107010004FF4006201E04FF4006201E04FF0200203
:1070200001E04FF0200201E04FF0200201E04FF0BC
:1070300020020A43DA60CBE17B681B681A4646F2FD
:10704000B803C4F202039A4240F293804FF4C8435B
:10705000C4F202034FF4C842C4F20202926811461D
:107060007A68106846F21002C4F2020290427BD0A5
:107070007A68106846F21042C4F20202904270D060
:107080007A68106846F27002C4F20202904265D03B
:107090007A68106846F27042C4F2020290425AD0F6
:1070A0007A68106846F22802C4F2020290424FD079
:1070B0007A68106846F22842C4F20202904244D034
:1070C0007A68106846F28802C4F20202904239D00F
:1070D0007A68106846F28842C4F2020290422ED0CA
:1070E0007A68106846F24002C4F20202904223D04D
:1070F0007A68106846F24042C4F20202904218D008
:107100007A68106846F2A002C4F2020290420DD0E2
:107110007A68106846F2A042C4F20202904202D19C
:107120004FF4001201E04FF0006201E04FF4001252
:1071300001E04FF4001201E04FF4001201E04FF4BF
:10714000006201E04FF4006201E04FF4006201E0F0
:107150004FF4006201E04FF0200201E04FF0200206
:1071600001E04FF0200201E04FF020020A439A6054
:107170002EE17B681B681A4646F25803C4F20203EC
:107180009A4240F293804FF4C043C4F202034FF49A
:10719000C042C4F20202D26811467A68106846F210
:1071A0001002C4F2020290427BD07A68106846F264
:1071B0001042C4F20202904270D07A68106846F21F
:1071C0007002C4F20202904265D07A68106846F2FA
:1071D0007042C4F2020290425AD07A68106846F2B5
:1071E0002802C4F2020290424FD07A68106846F238
:1071F0002842C4F20202904244D07A68106846F2F3
:107200008802C4F20202904239D07A68106846F2CD
:107210008842C4F2020290422ED07A68106846F288
:107220004002C4F20202904223D07A68106846F20B
:107230004042C4F20202904218D07A68106846F2C6
:10724000A002C4F2020290420DD07A68106846F2A1
:10725000A042C4F20202904202D14FF4001201E0B7
:107260004FF0006201E04FF4001201E04FF4001211
:1072700001E04FF4001201E04FF4006201E04FF42E
:10728000006201E04FF4006201E04FF4006201E0AF
:107290004FF0200201E04FF0200201E04FF0200209
:1072A00001E04FF020020A43DA6091E04FF4C0435E
:1072B000C4F202034FF4C042C4F2020292681146C3
:1072C0007A68106846F21002C4F2020290427BD043
:1072D0007A68106846F21042C4F20202904270D0FE
:1072E0007A68106846F27002C4F20202904265D0D9
:1072F0007A68106846F27042C4F2020290425AD094
:107300007A68106846F22802C4F2020290424FD016
:107310007A68106846F22842C4F20202904244D0D1
:107320007A68106846F28802C4F20202904239D0AC
:107330007A68106846F28842C4F2020290422ED067
:107340007A68106846F24002C4F20202904223D0EA
:107350007A68106846F24042C4F20202904218D0A5
:107360007A68106846F2A002C4F2020290420DD080
:107370007A68106846F2A042C4F20202904202D13A
:107380004FF4001201E04FF0006201E04FF40012F0
:1073900001E04FF4001201E04FF4001201E04FF45D
:1073A000006201E04FF4006201E04FF4006201E08E
:1073B0004FF4006201E04FF0200201E04FF02002A4
:1073C00001E04FF0200201E04FF020020A439A60F2
:1073D0007B68DB6C1A467B68DA647B684FF01102CD
:1073E00083F835207B684FF0000283F834207B68F7
:1073F000DB6B002B03D07B68DB6B7868984707F169
:107400000807BD4680BD00BF80B582B000AF786080
:107410007B68002B02D14FF0010325E07B681A68DE
:107420004FF4E843C4F200039A4207D045F22C30EF
:10743000C0F601004FF0E80101F0B4F87B681B7959
:10744000DBB2002B02D1786800F014F87B684FF0B3
:1074500002021A717B684FF000021A617B684FF0DC
:1074600001021A714FF00003184607F10807BD46E4
:1074700080BD00BF80B483B000AF786007F10C0717
:10748000BD4680BC704700BF80B584B000AF786057
:1074900039604FF00003FB604FF00003BB603B68B6
:1074A000002B0AD03B68102B07D045F22C30C0F6D9
:1074B000010040F26B1101F075F87B685B79012BDC
:1074C00002D14FF0020358E07B684FF001025A717D
:1074D0007B684FF002021A717B681B687A68126839
:1074E000126811463A684FF0010000FA02F20A43AE
:1074F0001A603B68002B1AD17B681B681B6803F07D
:107500000403FB607B681B681B6803F03803BB60E7
:10751000FB68042B27D1BB68382B24D17B681B6800
:107520007A681268526842F001025A601BE07B6878
:107530001B681B6803F48023FB607B681B681B6867
:1075400003F46013BB60FB68B3F5802F0BD1BB68FD
:10755000B3F5601F07D17B681B687A6812685268B0
:1075600042F002025A607B684FF001021A717B6898
:107570004FF000025A714FF00003184607F1100750
:10758000BD4680BD80B586B000AFF860B9607A6056
:107590004FF000037B614FF000033B61BB681B6849
:1075A000002B27D0BB681B68242B23D0BB681B682B
:1075B0000C2B1FD0BB681B68142B1BD0BB681B682F
:1075C0001C2B17D0BB681B68042B13D0BB681B682F
:1075D0002C2B0FD0BB681B68342B0BD0BB681B68EF
:1075E0003C2B07D045F22C30C0F6010040F2F321CD
:1075F00000F0D8FFBB685B68002B0BD0BB685B68F2
:10760000022B07D045F22C30C0F601004FF43D713B
:1076100000F0C8FFBB681B68002B27D0BB681B6845
:10762000242B23D0BB681B680C2B1FD0BB681B68A6
:10763000142B1BD0BB681B681C2B17D0BB681B68A6
:10764000042B13D0BB681B682C2B0FD0BB681B68A6
:10765000342B0BD0BB681B683C2B07D045F22C3079
:10766000C0F6010040F2F52100F09CFF7B68002B82
:107670000AD07B68102B07D045F22C30C0F60100F1
:1076800040F2F62100F08EFFFB685B79012B02D1FE
:107690004FF0020347E0FB684FF001025A71FB68AC
:1076A0004FF002021A714FF4E843C4F200031B6862
:1076B0007B617B6840F6FE7202FA03F36FEA030314
:1076C0007A6913407B61BB681A68BB685B681343C7
:1076D0003B617B683A6902FA03F37A6913437B6181
:1076E0004FF4E843C4F200037A691A604FF4E843A8
:1076F000C4F200034FF4E842C4F2000212681146DB
:107700007A684FF0C00000FA02F26FEA02020A4003
:107710001A60FB684FF001021A71FB684FF000021B
:107720005A714FF00003184607F11807BD4680BD97
:1077300080B586B000AFF860B9607A603B604FF00A
:1077400000037B61BB68002B0AD0BB68102B07D0FD
:1077500045F22C30C0F601004FF44B7100F022FFCF
:107760007B68002B0DD07B68042B0AD07B68082B2C
:1077700007D045F22C30C0F6010040F22D3100F068
:1077800011FF3A684FF6F0739A4207D945F22C3050
:10779000C0F6010040F22E3100F004FFFB681B68C8
:1077A0007B61BB68002B06D17A697B68D31803F133
:1077B00008037B6105E07A697B68D31803F1140341
:1077C0007B617B693A681A604FF00003184607F145
:1077D0001807BD4680BD00BF80B485B000AF78609B
:1077E0007B6803F00703FB604FF46D43CEF20003A8
:1077F000DB68BB60BA684FF6FF031340BB60FB68F1
:107800004FEA0322BB68134343F0BE6343F42023D3
:10781000BB604FF46D43CEF20003BA68DA6007F143
:107820001407BD4680BC704780B400AF4FF46D4371
:10783000CEF20003DB6803F4E0634FEA132318463B
:10784000BD4680BC704700BF80B483B000AF034624
:10785000FB714FF46143CEF2000397F907204FEA22
:107860005212F97901F01F014FF0010000FA01F105
:1078700043F8221007F10C07BD4680BC704700BFDB
:1078800080B483B000AF03463960FB7197F90730CD
:10789000002B10DA4FF46D43CEF20003FA7902F0B8
:1078A0000F02A2F104013A68D2B24FEA0212D2B238
:1078B0005B181A760DE04FF46143CEF2000397F99E
:1078C00007103A68D2B24FEA0212D2B25B1883F8BC
:1078D000002307F10C07BD4680BC704780B489B017
:1078E00000AFF860B9607A60FB6803F00703FB61E2
:1078F000FB69C3F10703042B28BF0423BB61FB69A9
:1079000003F10403062B03D9FB69A3F1030301E090
:107910004FF000037B61BB694FF0010202FA03F3F1
:1079200003F1FF331A46BB681A407B6902FA03F27F
:107930007B694FF0010101FA03F303F1FF331946AC
:107940007B680B401343184607F12407BD4680BCF3
:10795000704700BF80B582B000AF78607B6803F1EC
:10796000FF326FF07F439A4202D94FF001031DE0CE
:107970004EF21003CEF200037A6802F1FF325A6031
:107980004FF0FF304FF00F01FFF77AFF4EF2100378
:10799000CEF200034FF000029A604EF21003CEF2D6
:1079A00000034FF007021A604FF00003184607F17A
:1079B0000807BD4680BD00BF80B582B000AF7860CB
:1079C0007B68072B13D07B68062B10D07B68052BB8
:1079D0000DD07B68042B0AD07B68032B07D045F2BF
:1079E0005C30C0F601004FF0BA0100F0DBFD7868B2
:1079F000FFF7F2FE07F10807BD4680BD80B586B0EF
:107A000000AF0346B9607A60FB734FF000037B61FF
:107A10007B680F2B07D945F25C30C0F601004FF0B0
:107A2000D20100F0BFFDBB680F2B07D945F25C30D7
:107A3000C0F601004FF0D30100F0B4FDFFF7F4FEF3
:107A400003467B617869B9687A68FFF747FF0346A8
:107A500097F90F2010461946FFF712FF07F1180794
:107A6000BD4680BD80B582B000AF0346FB7197F97B
:107A700007301846FFF7E8FE07F10807BD4680BD4E
:107A800080B582B000AF78607868FFF763FF034687
:107A9000184607F10807BD4680BD00BF80B582B01B
:107AA00000AF78607B68002B02D14FF001035DE1ED
:107AB0007B681A684FF40053C4F201039A4217D04E
:107AC0007B681A684FF40453C4F201039A420FD042
:107AD0007B681A684FF40853C4F201039A4207D036
:107AE00045F29030C0F601004FF0D70100F05AFD8A
:107AF0007B685B68002B16D07B685B68B3F5803FC2
:107B000011D07B685B68B3F5003F0CD07B685B6885
:107B1000B3F5403F07D045F29030C0F601004FF07A
:107B2000D80100F03FFD7B689B68002B16D07B6876
:107B30009B68B3F1807F11D07B689B68B3F1007FB5
:107B40000CD07B689B68B3F1407F07D045F2903042
:107B5000C0F601004FF0D90100F024FD7B681B69DD
:107B6000002B0BD07B681B69012B07D045F29030AE
:107B7000C0F601004FF0DA0100F014FD7B689B694C
:107B8000002B0BD07B689B69012B07D045F290300E
:107B9000C0F601004FF0DB0100F004FD7B68DB6AFA
:107BA000002B16D07B68DB6AB3F1805F11D07B6855
:107BB000DB6AB3F1005F0CD07B68DB6AB3F1405F36
:107BC00007D045F29030C0F601004FF0DC0100F024
:107BD000E9FC7B681B6B002B52D07B681B6BB3F1FD
:107BE000807F4DD07B681B6BB3F1007F48D07B68F2
:107BF0001B6BB3F1407F43D07B681B6BB3F1806F8D
:107C00003ED07B681B6BB3F1A06F39D07B681B6BD8
:107C1000B3F1C06F34D07B681B6BB3F1E06F2FD032
:107C20007B681B6BB3F1006F2AD07B681B6BB3F1D1
:107C3000106F25D07B681B6BB3F1206F20D07B6861
:107C40001B6BB3F1306F1BD07B681B6BB3F1406FC4
:107C500016D07B681B6BB3F1506F11D07B681B6B28
:107C6000B3F1606F0CD07B681B6BB3F1706F07D002
:107C700045F29030C0F601004FF0DD0100F092FCBB
:107C80007B68DB68002B0CD07B68DB68B3F5006F8A
:107C900007D045F29030C0F601004FF0DE0100F051
:107CA00081FC7B681B6A002B03D07B681B6A102B4E
:107CB00007D945F29030C0F601004FF0DF0100F027
:107CC00071FC7B68DB69002B0BD07B68DB69012BC7
:107CD00007D045F29030C0F601004FF0E00100F00F
:107CE00061FC7B685B69012B0FD07B685B69002BB3
:107CF0000BD07B685B69022B07D045F29030C0F651
:107D000001004FF0E10100F04DFC7B685B6A002B45
:107D10000BD07B685B6A012B07D045F29030C0F630
:107D200001004FF0E20100F03DFC7B6893F83D302C
:107D3000DBB2002B02D1786800F01EF87B684FF0B0
:107D4000020283F83D20786800F0DAFA7B684FF091
:107D500000021A647B684FF0010283F83D207B68C3
:107D60004FF0000283F83C204FF00003184607F163
:107D70000807BD4680BD00BF80B483B000AF786007
:107D800007F10C07BD4680BC704700BF80B584B0CA
:107D900000AF78604FF00003FB817B689B69002B8C
:107DA0000BD07B689B69012B07D045F29030C0F661
:107DB00001004FF4B37100F0F5FB7B68DB6A002B28
:107DC00016D07B68DB6AB3F1805F11D07B68DB6A19
:107DD000B3F1005F0CD07B68DB6AB3F1405F07D082
:107DE00045F29030C0F6010040F2671100F0DAFB76
:107DF0007B6893F83C30012B02D14FF002035FE027
:107E00007B684FF0010283F83C207B6893F83D309B
:107E1000DBB2222B05D17B684FF0320283F83D2084
:107E200004E07B684FF0120283F83D207B681B68FA
:107E30009B6803F00103002B11D17B681B687A68F3
:107E40001268926842F001029A6004E000BFFB8968
:107E500003F10103FB81FB89B3F5077FF6D94FF4EA
:107E60000C53C4F201035B6803F01F03002B0CD119
:107E70007B68DB6A002B1CD17B681B687A68126800
:107E8000926842F080429A6013E07B681A684FF46F
:107E90000053C4F201039A420BD17B68DB6A002BCA
:107EA00007D17B681B687A681268926842F080424A
:107EB0009A607B684FF0000283F83C204FF000038B
:107EC000184607F11007BD4680BD00BF80B584B0DD
:107ED00000AF7860396000F059FB02463B68D31868
:107EE000FB6016E03B68B3F1FF3F12D000F04EFBA1
:107EF0000246FB689A420CD37B684FF0030283F87A
:107F00003D207B684FF0000283F83C204FF00303D4
:107F100019E07B681B681B6803F00203002BE1D0AB
:107F20007B6893F83D30DBB2252B05D17B684FF0A1
:107F3000350283F83D2004E07B684FF0150283F89A
:107F40003D204FF00003184607F11007BD4680BDE5
:107F500080B483B000AF78607B681B68DB6C184628
:107F600007F10C07BD4680BC704700BF90B583B0D9
:107F700000AF786039603B681B68002B4FD03B68CE
:107F80001B68012B4BD03B681B68022B47D03B681A
:107F90001B68032B43D03B681B68042B3FD03B6816
:107FA0001B68052B3BD03B681B68062B37D03B6812
:107FB0001B68072B33D03B681B68082B2FD03B680E
:107FC0001B68092B2BD03B681B680A2B27D03B680A
:107FD0001B680B2B23D03B681B680C2B1FD03B6806
:107FE0001B680D2B1BD03B681B680E2B17D03B6802
:107FF0001B680F2B13D03B681B68102B0FD03B68FE
:108000001B68112B0BD03B681B68122B07D045F265
:108010009030C0F6010040F2DE3100F0C3FA3B6858
:108020005B68002B03D03B685B68102B07D945F2D7
:108030009030C0F6010040F2DF3100F0B3FA3B6847
:108040009B68002B23D03B689B68012B1FD03B68AB
:108050009B68022B1BD03B689B68032B17D03B68A7
:108060009B68042B13D03B689B68052B0FD03B68A3
:108070009B68062B0BD03B689B68072B07D045F20B
:108080009030C0F601004FF4787100F08BFA7B68F5
:1080900093F83C30012B02D14FF002031CE17B68C6
:1080A0004FF0010283F83C203B681B68092B2AD95A
:1080B0007B6819687B681B68DB6818463B681A6830
:1080C00013464FEA43039B18A3F11E034FF0070228
:1080D00002FA03F36FEA03030340CB607B6819687D
:1080E0007B681B68DB6818463B689C683B681A68BD
:1080F00013464FEA43039B18A3F11E0304FA03F34C
:108100000343CB6025E07B6819687B681B681B69AB
:1081100018463B681A6813464FEA43039B184FF012
:10812000070202FA03F36FEA030303400B617B6863
:1081300019687B681B681B6918463B689C683B682C
:108140001A6813464FEA43039B1804FA03F30343E8
:108150000B613B685B68062B2AD87B6819687B68D3
:108160001B685B6B18463B685A6813464FEA8303EB
:108170009B18A3F105034FF01F0202FA03F36FEA05
:10818000030303404B637B6819687B681B685B6B68
:1081900018463B681C683B685A6813464FEA8303DD
:1081A0009B18A3F1050304FA03F303434B6358E060
:1081B0003B685B680C2B2AD87B6819687B681B6856
:1081C0001B6B18463B685A6813464FEA83039B189B
:1081D000A3F123034FF01F0202FA03F36FEA030334
:1081E00003400B637B6819687B681B681B6B184630
:1081F0003B681C683B685A6813464FEA83039B1828
:10820000A3F1230304FA03F303430B6329E07B6820
:1082100019687B681B68DB6A18463B685A68134616
:108220004FEA83039B18A3F141034FF01F0202FAA8
:1082300003F36FEA03030340CB627B6819687B6832
:108240001B68DB6A18463B681C683B685A68134623
:108250004FEA83039B18A3F1410304FA03F303439A
:10826000CB627B681A684FF40053C4F201039A4250
:108270000FD13B681B68122B0BD14FF40C53C4F287
:1082800001034FF40C52C4F20102526842F480021E
:108290005A607B681A684FF40053C4F201039A4293
:1082A00013D13B681B68102B03D03B681B68112B54
:1082B0000BD14FF40C53C4F201034FF40C52C4F22F
:1082C0000102526842F400025A607B684FF00002DB
:1082D00083F83C204FF00003184607F10C07BD4619
:1082E00090BD00BF80B483B000AF78607B6893F826
:1082F0003D30DBB2184607F10C07BD4680BC704725
:1083000080B582B000AF78604FF40C53C4F2010323
:108310004FF40C52C4F20102526822F440325A6007
:108320004FF40C53C4F201034FF40C52C4F2010297
:10833000526811467A6852680A435A607B681B6823
:108340007A681268526822F480725A607B681B68EF
:108350007A681268526811467A6812694FEA0222F6
:108360000A435A607B681B687A681268526822F078
:1083700040725A607B681B687A68126852681146BE
:108380007A6892680A435A607B681B687A68126848
:10839000926822F400629A607B681B687A681268AF
:1083A000926811467A68D2680A439A607B681B68B3
:1083B0007A681268926822F070629A607B681B6823
:1083C0007A681268926811467A68126B0A439A605A
:1083D0007B681B687A681268926822F040529A6043
:1083E0007B681B687A681268926811467A68D26A5C
:1083F0000A439A607B681B687A681268926822F068
:1084000002029A607B681B687A681268926811465B
:108410007A6892694FEA42020A439A607B685B6A13
:10842000002B2ED07B689B6A002B03D07B689B6A55
:10843000082B07D945F29030C0F601004FF498613F
:1084400000F0B0F87B681B687A681268526842F4E2
:1084500000625A607B681B687A681268526822F46E
:1084600060425A607B681B687A68126852681146DD
:108470007A68926A02F1FF324FEA42320A435A6046
:1084800007E07B681B687A681268526822F4006211
:108490005A607B681B687A681268D26A22F470029C
:1084A000DA627B681B687A681268D26A11467A6859
:1084B000126A02F1FF324FEA02520A43DA627B6823
:1084C0001B687A681268926822F400729A607B686E
:1084D0001B687A681268926811467A68D2694FEA16
:1084E00042220A439A607B681B687A681268926825
:1084F00022F480629A607B681B687A6812689268CE
:1085000011467A6852694FEA82220A439A6007F15B
:108510000807BD4680BD00BF80B500AF4FF4705363
:10852000C4F202034FF47052C4F20202126842F421
:1085300000721A604FF47053C4F202034FF4705289
:10854000C4F20202126842F480621A604FF470535F
:10855000C4F202034FF47052C4F20202126842F4F1
:1085600080721A604FF47A50FFF78AFA4FF00300D6
:10857000FFF722FA00F004F84FF00003184680BD20
:1085800080B400AFBD4680BC704700BF80B400AF70
:1085900040F6DC03C2F200031B681846BD4680BCEF
:1085A000704700BF80B584B000AF7860396045F295
:1085B0000443C0F60103FB6000F062F880B483B0AE
:1085C00000AF786039607B684FF001021A603A684A
:1085D00040F20403C2F20003136007F10C07BD462A
:1085E00080BC704780B584B000AF786040F6E4038B
:1085F000C2F200031B68002B08D140F6E403C2F26C
:10860000000344F67802C2F200021A6040F6E40366
:10861000C2F200031B68FB607B6803F1030323F0D5
:1086200003037B6040F6E403C2F200031A687B6830
:10863000D2184FF60043C2F201039A4208D909F05A
:1086400081F803464FF00C021A604FF0FF330CE044
:1086500040F6E403C2F200031A687B68D21840F6C1
:10866000E403C2F200031A60FB68184607F1100722
:10867000BD4680BD80B483B000AF7860FEE700BF28
:1086800080B582B000AF45F23043C0F601037B6095
:108690004FF00100FFF7EEFF80B400AF4FF46D43E1
:1086A000CEF200034FF46D42CEF20002D2F88820E1
:1086B00042F47002C3F888204FF46053C4F20203FE
:1086C0004FF46052C4F20202126842F001021A60D2
:1086D0004FF46053C4F202034FF000029A604FF46B
:1086E0006053C4F202034FF46052C4F202021268F3
:1086F00022F0847222F480321A604FF46053C4F284
:10870000020343F21002C2F200425A604FF4605377
:10871000C4F202034FF46052C4F20202126822F45F
:1087200080221A604FF46053C4F202034FF000023B
:10873000DA604FF46D43CEF200034FF000629A60AE
:10874000BD4680BC704700BF80B400AFBD4680BC52
:10875000704700BF80B400AFFEE700BF80B400AF39
:10876000FEE700BF80B400AFFEE700BF80B400AFFB
:10877000FEE700BF80B400AFBD4680BC704700BFBD
:1087800080B400AFBD4680BC704700BF80B400AF6E
:10879000BD4680BC704700BF80B500AF40F68C304E
:1087A000C2F20000F8F7ACFB80BD00BF80B500AF9F
:1087B00002F098FD80BD00BF80B500AF40F62833C1
:1087C000C2F200031B6C1846FAF772FF80BD00BFAF
:1087D00080B500AF40F62833C2F200035B6C184648
:1087E000FAF766FF80BD00BF80B590B000AF40F6DD
:1087F0002830C2F20000F8F7F9FE4FF46053C4F2DB
:1088000002034FF46052C4F20202526C42F48052EE
:108810005A6449F2F073C0F601039B883B604FF045
:108820000203FB604FF002037B604FF005033B61E6
:108830004FF00003BB6049F2F073C0F601031A6801
:108840003B4610461946FAF7D9F849F2E073C0F6EC
:1088500001039B883B604FF00203FB604FF0020373
:108860007B604FF00003BB604FF005033B6149F2B2
:10887000E073C0F601031A683B4610461946FAF742
:10888000BDF849F2E873C0F601039B883B604FF0E6
:108890000203FB604FF000037B604FF00103BB60FD
:1088A0004FF005033B6149F2E873C0F601031A6813
:1088B0003B4610461946FAF7A1F849F29073C0F604
:1088C00001039B883B604FF00203FB604FF0010304
:1088D0007B604FF00003BB604FF000033B6149F247
:1088E0009073C0F601031A683B4610461946FAF722
:1088F00085F849F29073C0F601031A6849F2907343
:10890000C0F601039B88104619464FF00102FAF7A2
:108910004FFC40F62833C2F200034FF44052C4F239
:1089200001021A6040F62833C2F200034FF0000241
:108930009A6040F62833C2F200034FF482725A6004
:1089400040F62833C2F200034FF00002DA6040F62E
:108950002833C2F200034FF002021A6140F62833B6
:10896000C2F200034FF001025A6140F62833C2F20E
:1089700000034FF400729A6140F62833C2F20003FC
:108980004FF00002DA6140F62833C2F200034FF0E4
:1089900000021A6240F62833C2F200034FF00002D0
:1089A0009A6240F62833C2F200034FF000025A6286
:1089B00040F62833C2F200034FF00702DA6240F6B5
:1089C0002830C2F20000F8F7CFFC07F14007BD469F
:1089D00080BD00BF84B080B500AF07F1080C8CE803
:1089E0000F003B6E1B884FEA13239BB2DAB240F6AE
:1089F000E803C2F200031A703B6E1B88DAB240F63D
:108A0000E803C2F200035A7040F62830C2F20000B8
:108A100040F6E801C2F200014FF002024FF00103FC
:108A2000F8F7EEFDBD46BDE8804004B0704700BFDA
:108A300080B582B000AF87ED010A3860D7ED017ACA
:108A4000F5EEC07AF1EE10FAD4BF00230123DBB2B9
:108A5000002B0BD097ED010A07F0BEFDF0EE407A37
:108A60003B68C3ED007A4FF0000304E03B68054A21
:108A70001A604FF0FF035BB2184607F10807BD46C6
:108A800080BD00BF0000000080B592B000AF4FF481
:108A90006053C4F202034FF46052C4F20202126C3B
:108AA00042F080521A644FF4E043C4F200034FF4E2
:108AB000E042C4F20002126842F440421A604FF0F1
:108AC00001037B604FF00103BB604FF00203FB61C9
:108AD0004FF480033B624FF00F037B624FF0D203F1
:108AE000BB624FF00203FB624FF007033B6307F1E9
:108AF00004031846F8F7F4FF4FF00D037B634FF0C3
:108B00000203BB634FF00003FB634FF4A0533B64CD
:108B10004FF480537B6407F1340318464FF005018E
:108B2000F9F796FB07F14807BD4680BD80B48DB0CC
:108B300000AFF860B9607A604FF064037B85BB6872
:108B4000022B00F39B804FF00003FB627CE0BB68CC
:108B5000012B27D0022B45D0002B71D17A68FB68FE
:108B6000D318C3F50072FB6A9A4210DA7B68C3F52A
:108B70000072FB6A9A420ADD40F62843C2F2000303
:108B8000FA6A4FEA82029B183F4A1A6058E040F6A0
:108B90002843C2F20003FA6A4FEA82029B183B4A5A
:108BA0001A604DE0FA6A7B689A4210DD7A68FB68C9
:108BB000D218FB6A9A420ADD40F62843C2F200034B
:108BC000FA6A4FEA82029B182F4A1A6038E040F690
:108BD0002843C2F20003FA6A4FEA82029B182B4A2A
:108BE0001A602DE07A68FB68D318C3F50072FB6A3F
:108BF0009A4205DA7B68C3F50072FB6A9A4209DC87
:108C0000FA6A7B689A4210DD7A68FB68D218FB6AC0
:108C10009A420ADD40F62843C2F20003FA6A4FEA9C
:108C200082029B18184A1A6009E040F62843C2F2F3
:108C30000003FA6A4FEA82029B18144A1A6000BFC6
:108C4000FB6A03F10103FB62FA6A40F2FF139A42E6
:108C50007FF77DAF40F62843C2F2000303F580633F
:108C60000A4A1A6040F62843C2F2000303F5FE6385
:108C700003F10C03054A1A6000BF00E000BF07F1D2
:108C80003407BD4680BC70470000803F00000000F4
:108C900080B485B000AF786039604FF00003FB60AE
:108CA0007DE0FB684FEA4302FB684FEAC303796843
:108CB000CB1893ED007AFB684FEA430140F6284356
:108CC000C2F200034FEA81015B18D3ED007A27EE70
:108CD000277AFB684FEAC30303F104037968CB18D2
:108CE000D3ED006AFB684FEA430303F1010140F64C
:108CF0002843C2F200034FEA81015B18D3ED007AEA
:108D000066EEA77A77EE677A43F62C53C2F2000339
:108D10004FEA82029B18C3ED007AFB684FEA4303D7
:108D200003F10102FB684FEAC30303F1040379680E
:108D3000CB1893ED007AFB684FEA430303F101017E
:108D400040F62843C2F200034FEA81015B18D3EDDD
:108D5000007A27EE277AFB684FEAC3037968CB18BD
:108D6000D3ED006AFB684FEA430140F62843C2F2A4
:108D700000034FEA81015B18D3ED007A66EEA77A13
:108D800077EE277A43F62C53C2F200034FEA8202B1
:108D90009B18C3ED007AFB6803F10103FB60FB68DD
:108DA000FF2B7FF77EAF4FF00003FB6032E03B68A4
:108DB0004FEA4302FB68D318BB60FB68002B06DA5E
:108DC000FB684FEA83037A68D318174A1A60FA6877
:108DD00040F2FF139A4206DDFB684FEA83037A688C
:108DE000D318114A1A60FB684FEA83037A68D218D5
:108DF0003B684FEA4301FB68C91843F62C53C2F2A3
:108E000000034FEA81015B181B681360FB6803F1E4
:108E10000103FB60FA6840F2FF139A42C7DD07F1D5
:108E20001407BD4680BC70470000000080B400AF4E
:108E30004FF46053C4F202034FF46052C4F20202D2
:108E4000126B42F001021A634FF46053C4F2020342
:108E50004FF46052C4F20202126B42F002021A6333
:108E60004FF46053C4F202034FF46052C4F20202A2
:108E7000126B42F004021A634FF46053C4F202030F
:108E80004FF46052C4F20202126B42F008021A63FD
:108E90004FF46053C4F202034FF46052C4F2020272
:108EA000126B42F010021A634FF46053C4F20203D3
:108EB0004FF46052C4F20202126B42F400121A63C1
:108EC0004FF46053C4F202034FF46052C4F2020242
:108ED000126B42F480021A63BD4680BC704700BF2B
:108EE00080B582B000AF786040F65413C2F2000340
:108EF00046F28842C4F202021A6040F65413C2F2EB
:108F000000034FF0C0625A6040F65413C2F20003EF
:108F10004FF040029A6040F65413C2F200034FF043
:108F20000002DA6040F65413C2F200034FF480628C
:108F30001A6140F65413C2F200034FF000025A6166
:108F400040F65413C2F200034FF000029A6140F65B
:108F50005413C2F200034FF00002DA6140F65413DA
:108F6000C2F200034FF000021A6240F65413C2F23C
:108F700000034FF000025A6240F65413C2F200039D
:108F80004FF003029A6240F65413C2F200034FF40A
:108F90000002DA6240F65413C2F200034FF40012EA
:108FA0001A6340F65410C2F20000FAF765F97A68C5
:108FB00040F65413C2F20003136440F65413C2F295
:108FC00000037A689A6340F6A413C2F2000346F2E3
:108FD0004042C4F202021A6040F6A413C2F2000337
:108FE0004FF0C0625A6040F6A413C2F200034FF083
:108FF00000029A6040F6A413C2F200034FF0000290
:10900000DA6040F6A413C2F200034FF480621A61E2
:1090100040F6A413C2F200034FF000025A6140F67A
:10902000A413C2F200034FF000029A6140F6A413A9
:10903000C2F200034FF00002DA6140F6A413C2F25C
:1090400000034FF400321A6240F6A413C2F2000388
:109050004FF000025A6240F6A413C2F200034FF030
:1090600003029A6240F6A413C2F200034FF4000216
:10907000DA6240F6A413C2F200034FF400121A633E
:1090800040F6A410C2F20000FAF7F6F87A6840F64B
:10909000A413C2F20003536440F6A413C2F2000307
:1090A0007A689A634FF00F004FF000014FF0010211
:1090B000FEF7A4FC4FF03B00FEF7D4FC4FF0380065
:1090C0004FF000014FF00002FEF798FC4FF038001F
:1090D000FEF7C8FC07F10807BD4680BD80B400AFAD
:1090E00040F65013C2F200031B6803F1010240F680
:1090F0005013C2F200031A60BD4680BC704700BF27
:1091000080B500AF40F6F003C2F20003D3E90001DE
:109110004FF001024FF00003801841EB030140F6CD
:10912000F003C2F20003C3E9000104F0B5F949F20B
:10913000B513C0F60003984740F6D023C2F20003EF
:109140001B68002B0BD040F6D023C2F200031B6833
:1091500003F1FF3240F6D023C2F200031A6080BD53
:1091600080B400AF41F23843C2F200034FF0000276
:109170001A6040F62443C2F200034FF000021A6066
:1091800042F26043C2F200034FF07F021A6041F2E4
:109190003C43C2F200034FF000021A6044F6500351
:1091A000C2F200034FF064021A601846BD4680BC4C
:1091B000704700BF98B500AF40F61813C2F2000325
:1091C0001B78002B40F0F58049F60003C0F6010340
:1091D0001A6849F60003C0F601039B881046194639
:1091E000F9F78CFF03464FEA430449F2F873C0F6DF
:1091F00001031A6849F2F873C0F601039B88104610
:109200001946F9F77BFF0346E21840F62443C2F201
:1092100000031A6040F62443C2F200031A6841F2C8
:109220003843C2F200031B689A4200F0B88041F252
:109230003843C2F200031B68002B06D140F62443DA
:10924000C2F200031B68012B29D041F23843C2F25D
:1092500000031B68012B06D140F62443C2F2000331
:109260001B68032B1BD041F23843C2F200031B687A
:10927000032B06D140F62443C2F200031B68022BE5
:109280000DD041F23843C2F200031B68022B09D112
:1092900040F62443C2F200031B68002B02D14FF0BA
:1092A000010201E04FF0000243F6A843C2F20003BE
:1092B0001A6049F60803C0F601031A6849F6080364
:1092C000C0F601039B8810461946F9F717FF0346BD
:1092D000002B44D143F6A843C2F200031B68002BC5
:1092E0000DD040F6FC03C2F200031B8803F101031A
:1092F0009AB240F6FC03C2F200031A800CE040F67A
:10930000FC03C2F200031B8803F1FF339AB240F65C
:10931000FC03C2F200031A8040F6FC03C2F2000311
:109320001B884FEA53039AB240F6FA03C2F20003D5
:109330001A8040F6FA03C2F200031A8840F21803BA
:10934000C2F200031B88B2FBF3F103FB01F3D31A53
:109350009AB240F6FA03C2F200031A801FE043F605
:10936000A843C2F200031B68002B0CD044F6540340
:10937000C2F200031B6803F1010244F65403C2F277
:1093800000031A600BE044F65403C2F200031B68AA
:1093900003F1FF3244F65403C2F200031A6040F6B0
:1093A0002443C2F200031A6841F23843C2F20003B8
:1093B0001A6098BD0000000098B500AF40F68133F8
:1093C000C2F200031B78002B00F02A8740F68A3394
:1093D000C2F200031B88642B09D14FF00000C4F2D5
:1093E00002004FF480714FF00102F9F7E1FE03F043
:1093F000D1FE40F62C13C2F200031B68012B00F0D3
:109400002282022B00F04284002B40F0688640F656
:109410001013C2F200031B68002B62D140F68A339E
:10942000C2F200031B884FEA430440F67E33C2F2C7
:1094300000031B889BB21A4640F23003C2F20003BD
:109440001B68D31A184607F029FB02460B46104644
:1094500019460FF2C443D3E9002307F0AFFC0246DC
:109460000B461046194607F041FE024642F6A84355
:10947000C2F200034FEA84015B181A6040F68A3397
:10948000C2F200031B884FEA430303F1010440F6D4
:10949000CC23C2F200031B889BB21A4640F22C0375
:1094A000C2F200031B68D31A184607F0F7FA024607
:1094B0000B46104619460FF26043D3E9002307F02C
:1094C0007DFC02460B461046194607F00FFE024689
:1094D00042F6A843C2F200034FEA84015B181A6007
:1094E0005FE040F68A33C2F200031B884FEA430470
:1094F00040F62C23C2F200031B889BB21A4640F2AE
:109500002803C2F200031B68D31A184607F0C6FAF4
:1095100002460B4610461946FFA3D3E9002307F085
:109520004DFC02460B461046194607F0DFFD024689
:1095300042F6A843C2F200034FEA84015B181A60A6
:1095400040F68A33C2F200031B884FEA430303F15B
:10955000010440F62C23C2F200031B889BB21A467A
:1095600040F22803C2F200031B68D31A184607F022
:1095700095FA02460B4610461946E7A3D3E90023A5
:1095800007F01CFC02460B461046194607F0AEFDDC
:10959000024642F6A843C2F200034FEA84015B1878
:1095A0001A6040F62C23C2F200031B889AB240F6E0
:1095B000F803C2F200031B889A420AD940F62C2312
:1095C000C2F200031B889AB240F6F803C2F200030D
:1095D0001A8040F6CC23C2F200031B889AB240F6F0
:1095E000F803C2F200031B889A420AD940F6CC2342
:1095F000C2F200031B889AB240F6F803C2F20003DD
:109600001A8040F68A33C2F200031B884FEA4302F5
:1096100041F24043C2F200034FEA82029B1893EDED
:10962000007A40F60813C2F20003D3ED007AB4EEDC
:10963000E77AF1EE10FAD4BF00230123DBB2002B4E
:1096400013D040F68A33C2F200031B884FEA43026C
:1096500041F24043C2F200034FEA82029B181A68AB
:1096600040F60813C2F200031A6040F68A33C2F2D1
:1096700000031B884FEA430303F1010241F2404318
:10968000C2F200034FEA82029B1893ED007A40F683
:109690000813C2F20003D3ED007AB4EEE77AF1EEDC
:1096A00010FAD4BF00230123DBB2002B15D040F603
:1096B0008A33C2F200031B884FEA430303F101021D
:1096C00041F24043C2F200034FEA82029B181A683B
:1096D00040F60813C2F200031A6040F68A33C2F261
:1096E00000031B884FEA430241F24043C2F20003E9
:1096F0004FEA82029B1893ED007ADFED897A27EE1C
:10970000277A40F21003C2F20003D3ED007A27EE6D
:10971000277ADFED847A77EE277AFCEEE77A17EE88
:10972000903A9BB2184602F0A3FA40F68A33C2F28E
:1097300000031B884FEA430303F1010241F2404357
:10974000C2F200034FEA82029B1893ED007ADFED2C
:10975000747A27EE277A40F21003C2F20003D3EDA9
:10976000007A27EE277ADFED6F7A77EE277AFCEE24
:10977000E77A17EE903A9BB2184602F093FA40F659
:109780008A33C2F200031B881A4640F21403C2F265
:1097900000031B88C3F1FF039A42C0F29B8440F68A
:1097A0008A33C2F200031B881A4640F21403C2F245
:1097B00000031B88A3F58073D3184FEA430140F6DA
:1097C0008A33C2F200031B884FEA430242F6A843E1
:1097D000C2F200034FEA82029B181A6844F2305327
:1097E000C2F200034FEA81015B181A6040F68A3327
:1097F000C2F200031B881A4640F21403C2F20003AF
:109800001B88A3F58073D3184FEA430303F10101CA
:1098100040F68A33C2F200031B884FEA430303F188
:10982000010242F6A843C2F200034FEA82029B18EB
:109830001A6844F23053C2F200034FEA81015B1808
:109840001A6000F047BC40F61013C2F200031B6818
:10985000002B69D140F68A33C2F200031B884FEA1D
:10986000430440F67E33C2F200031B889BB21A46C3
:1098700040F23003C2F200031B68D31A184607F007
:109880000DF902460B461046194623A3D3E90023DF
:1098900007F094FA02460B461046194607F026FCDC
:1098A000024641F24043C2F200034FEA84015B18D2
:1098B0001A6040F68A33C2F200031B884FEA430362
:1098C00003F1010440F6CC23C2F200031B889BB2D3
:1098D0001A4640F22C03C2F200031B68D31A184642
:1098E00007F0DCF802460B46104619460AA3D3E9F6
:1098F000002307F063FA02460B461046194607F0AC
:10990000F5FB024641F24043C2F200034FEA8401F4
:109910005B181A6069E000BF000000000000B04062
:10992000000080450000004540F68A33C2F2000383
:109930001B884FEA430440F62C23C2F200031B8825
:109940009BB21A4640F22803C2F200031B68D31AE6
:10995000184607F0A3F802460B46104619460FF2C8
:109960000043D3E9002307F029FA02460B461046CC
:10997000194607F0BBFB024641F24043C2F2000326
:109980004FEA84015B181A6040F68A33C2F2000382
:109990001B884FEA430303F1010440F62C23C2F273
:1099A00000031B889BB21A4640F22803C2F2000350
:1099B0001B68D31A184607F071F802460B4610468A
:1099C0001946E7A3D3E9002307F0F8F902460B464E
:1099D0001046194607F08AFB024641F24043C2F2A4
:1099E00000034FEA84015B181A6040F62C23C2F290
:1099F00000031B889AB240F6F803C2F200031B88EA
:109A00009A420AD940F62C23C2F200031B889AB26C
:109A100040F6F803C2F200031A8040F6CC23C2F2EB
:109A200000031B889AB240F6F803C2F200031B88B9
:109A30009A420AD940F6CC23C2F200031B889AB29C
:109A400040F6F803C2F200031A8040F68A33C2F2ED
:109A500000031B884FEA430241F66043C2F2000351
:109A60004FEA82029B1893ED007A40F60813C2F287
:109A70000003D3ED007AB4EEE77AF1EE10FAD4BF2A
:109A800000230123DBB2002B13D040F68A33C2F24D
:109A900000031B884FEA430241F66043C2F2000311
:109AA0004FEA82029B181A6840F60813C2F20003BC
:109AB0001A6040F68A33C2F200031B884FEA430360
:109AC00003F1010241F66043C2F200034FEA820251
:109AD0009B1893ED007A40F60813C2F20003D3ED11
:109AE000007AB4EEE77AF1EE10FAD4BF0023012336
:109AF000DBB2002B15D040F68A33C2F200031B887C
:109B00004FEA430303F1010241F66043C2F200034E
:109B10004FEA82029B181A6840F60813C2F200034B
:109B20001A6040F68A33C2F200031B884FEA4302F0
:109B300041F66043C2F200034FEA82029B1893EDA4
:109B4000007ADFED897A27EE277A40F21003C2F21D
:109B50000003D3ED007A27EE277ADFED847A77EEE3
:109B6000277AFCEEE77A17EE903A9BB2184602F09D
:109B70007FF840F68A33C2F200031B884FEA4303A2
:109B800003F1010241F66043C2F200034FEA820290
:109B90009B1893ED007ADFED747A27EE277A40F276
:109BA0001003C2F20003D3ED007A27EE277ADFED2F
:109BB0006F7A77EE277AFCEEE77A17EE903A9BB24F
:109BC000184602F06FF840F68A33C2F200031B8891
:109BD0001A4640F21403C2F200031B88C3F1FF03CC
:109BE0009A42C0F2798240F68A33C2F200031B889F
:109BF0001A4640F21403C2F200031B88A3F58073D7
:109C0000D3184FEA430140F68A33C2F200031B889F
:109C10004FEA430241F24043C2F200034FEA82029C
:109C20009B181A6844F23053C2F200034FEA8101D4
:109C30005B181A6040F68A33C2F200031B881A468A
:109C400040F21403C2F200031B88A3F58073D318FB
:109C50004FEA430303F1010140F68A33C2F20003E5
:109C60001B884FEA430303F1010241F24043C2F271
:109C700000034FEA82029B181A6844F23053C2F282
:109C800000034FEA81015B181A6025E240F61013C9
:109C9000C2F200031B68002B6AD140F68A33C2F27D
:109CA00000031B884FEA430440F67E33C2F20003F0
:109CB0001B889BB21A4640F23003C2F200031B68B5
:109CC000D31A184606F0EAFE02460B46104619461D
:109CD00023A3D3E9002307F071F802460B46104690
:109CE000194607F003FA024641F66043C2F2000348
:109CF0004FEA84015B181A6040F68A33C2F200030F
:109D00001B884FEA430303F1010440F6CC23C2F25F
:109D100000031B889BB21A4640F22C03C2F20003D8
:109D20001B68D31A184606F0B9FE02460B461046C9
:109D300019460BA3D3E9002307F040F802460B466F
:109D40001046194607F0D2F9024641F66043C2F2C6
:109D500000034FEA84015B181A606BE0AFF30080E8
:109D6000000000000000B0400000804500000045F9
:109D700040F68A33C2F200031B884FEA430440F6E0
:109D80002C23C2F200031B889BB21A4640F2280320
:109D9000C2F200031B68D31A184606F07FFE024683
:109DA0000B46104619460FF29043D3E9002307F003
:109DB00005F802460B461046194607F097F9024689
:109DC00041F66043C2F200034FEA84015B181A6057
:109DD00040F68A33C2F200031B884FEA430303F1C3
:109DE000010440F62C23C2F200031B889BB21A46E2
:109DF00040F22803C2F200031B68D31A184606F08B
:109E00004DFE02460B46104619460FF22C43D3E98D
:109E1000002306F0D3FF02460B461046194607F012
:109E200065F9024641F66043C2F200034FEA84013D
:109E30005B181A6040F62C23C2F200031B889AB20A
:109E400040F6F803C2F200031B889A420AD940F692
:109E50002C23C2F200031B889AB240F6F803C2F228
:109E600000031A8040F6CC23C2F200031B889AB28A
:109E700040F6F803C2F200031B889A420AD940F662
:109E8000CC23C2F200031B889AB240F6F803C2F258
:109E900000031A8040F68A33C2F200031B884FEA9F
:109EA000430242F6A843C2F200034FEA82029B1823
:109EB00093ED007A40F60813C2F20003D3ED007A66
:109EC000B4EEE77AF1EE10FAD4BF00230123DBB23F
:109ED000002B13D040F68A33C2F200031B884FEAEE
:109EE000430242F6A843C2F200034FEA82029B18E3
:109EF0001A6840F60813C2F200031A6040F68A336B
:109F0000C2F200031B884FEA430303F1010242F649
:109F1000A843C2F200034FEA82029B1893ED007A35
:109F200040F60813C2F20003D3ED007AB4EEE77AEC
:109F3000F1EE10FAD4BF00230123DBB2002B15D0C1
:109F400040F68A33C2F200031B884FEA430303F151
:109F5000010242F6A843C2F200034FEA82029B18B4
:109F60001A6840F60813C2F200031A6040F68A33FA
:109F7000C2F200031B884FEA430242F6A843C2F232
:109F800000034FEA82029B1893ED007ADFEDA87A76
:109F900027EE277A40F21003C2F20003D3ED007AD5
:109FA00027EE277ADFEDA37A77EE277AFCEEE77AC1
:109FB00017EE903A9BB2184601F05AFE40F68A33EB
:109FC000C2F200031B884FEA430303F1010242F689
:109FD000A843C2F200034FEA82029B1893ED007A75
:109FE000DFED937A27EE277A40F21003C2F20003E6
:109FF000D3ED007A27EE277ADFED8E7A77EE277A97
:10A00000FCEEE77A17EE903A9BB2184601F04AFE52
:10A0100040F68A33C2F200031B881A4640F214034A
:10A02000C2F200031B88C3F1FF039A4256DB40F6DD
:10A030008A33C2F200031B881A4640F21403C2F2AC
:10A0400000031B88A3F58073D3184FEA430140F641
:10A050008A33C2F200031B884FEA430241F6604391
:10A06000C2F200034FEA82029B181A6844F230538E
:10A07000C2F200034FEA81015B181A6040F68A338E
:10A08000C2F200031B881A4640F21403C2F2000316
:10A090001B88A3F58073D3184FEA430303F1010132
:10A0A00040F68A33C2F200031B884FEA430303F1F0
:10A0B000010241F66043C2F200034FEA82029B189C
:10A0C0001A6844F23053C2F200034FEA81015B1870
:10A0D0001A6003E000BF02E000BF00E000BF40F6EE
:10A0E0000813C2F200031B68184606F0E9FC02469A
:10A0F0000B46104619464CA3D3E9002306F034FD65
:10A1000002460B461046194606F0F0FF024640F69E
:10A110000813C2F200031A6040F68A33C2F2000349
:10A120001B8803F101039AB240F68A33C2F200039E
:10A130001A8040F68A33C2F200031B88FF2B6DD9C8
:10A140004FF00000C4F202004FF480714FF00002A3
:10A15000F9F72EF840F62133C2F200034FF0010266
:10A160001A7040F21403C2F200031A8840F68A33D0
:10A17000C2F200031A8040F62C13C2F200031B68DF
:10A18000012B1BD0022B31D0002B47D140F61C13E2
:10A19000C2F200034FF001021A6040F62C13C2F223
:10A1A00000034FF001021A604AF24123C0F6000397
:10A1B00041F24040C2F2000098472FE040F62013E1
:10A1C000C2F200034FF001021A6040F62C13C2F2F3
:10A1D00000034FF002021A604AF24123C0F6000366
:10A1E00041F66040C2F20000984717E040F62413A1
:10A1F000C2F200034FF001021A6040F62C13C2F2C3
:10A2000000034FF000021A604AF24123C0F6000337
:10A2100042F6A840C2F20000984700BF03F018F8C9
:10A2200098BD00BFAFF300801EA7E8482EFFEF3FA8
:10A230000000804500000045000000000000B04024
:10A2400080B485B000AF78604FF00003FB8112E06E
:10A25000FB894FEA83037A68D218F98944F23053B4
:10A26000C2F200034FEA81015B181B681360FB898F
:10A2700003F10103FB81FA8940F21403C2F20003E7
:10A280001B884FEA43039A42E2DB0AE0FB894FEA6C
:10A2900083037A68D318084A1A60FB8903F1010323
:10A2A000FB81FA8940F2FF139A42EFD907F11407B4
:10A2B000BD4680BC704700BF0000000080B584B080
:10A2C00000AF02460B46FA71BB7149F6B803C0F6FF
:10A2D00001031A6849F6B803C0F601039B881046CB
:10A2E00019464FF00002F8F763FF49F6B003C0F6D5
:10A2F00001031A6849F6B003C0F601039B881046B3
:10A3000019464FF00002F8F753FF49F6A803C0F6CC
:10A3100001031A6849F6A803C0F601039B8810469A
:10A3200019464FF00002F8F743FF49F6A803C0F6BC
:10A3300001031A6849F6A803C0F601039B8810467A
:10A3400019464FF00102F8F733FF4FF00003FB739B
:10A350003CE049F6B003C0F60103196849F6B003C2
:10A36000C0F601039A88F879FB7BC3F1070340FA32
:10A3700003F3DBB203F00103DBB2084611461A46D1
:10A38000F8F716FF49F6A803C0F601031A6849F664
:10A39000A803C0F601039B88104619464FF000023F
:10A3A000F8F706FF49F6A803C0F601031A6849F654
:10A3B000A803C0F601039B88104619464FF001021E
:10A3C000F8F7F6FEFB7B03F10103FB73FB7B072B26
:10A3D000BFD949F6B803C0F601031A6849F6B803B5
:10A3E000C0F601039B88104619464FF00102F8F7AA
:10A3F000DFFE49F6B803C0F601031A6849F6B80350
:10A40000C0F601039B88104619464FF00002F8F78A
:10A41000CFFE49F6B003C0F601031A6849F6B0034F
:10A42000C0F601039B88104619464FF00102F8F769
:10A43000BFFE49F6A803C0F601031A6849F6A8034F
:10A44000C0F601039B88104619464FF00002F8F74A
:10A45000AFFE49F6A803C0F601031A6849F6A8033F
:10A46000C0F601039B88104619464FF00102F8F729
:10A470009FFE4FF00003FB733CE049F6B003C0F6CB
:10A480000103196849F6B003C0F601039A88B87948
:10A49000FB7BC3F1070340FA03F3DBB203F00103D4
:10A4A000DBB2084611461A46F8F782FE49F6A803C1
:10A4B000C0F601031A6849F6A803C0F601039B8899
:10A4C000104619464FF00002F8F772FE49F6A8034D
:10A4D000C0F601031A6849F6A803C0F601039B8879
:10A4E000104619464FF00102F8F762FEFB7B03F1BC
:10A4F0000103FB73FB7B072BBFD949F6B803C0F6FA
:10A5000001031A6849F6B803C0F601039B88104698
:10A5100019464FF00102F8F74BFE07F11007BD4650
:10A5200080BD00BF80B500AF4FF46053C4F202039A
:10A530004FF46052C4F20202126B42F002021A633C
:10A540004FF46053C4F202034FF46052C4F20202AB
:10A55000526C42F010025A6443F61453C2F20003E4
:10A560004FF040021A6043F61453C2F200034FF05A
:10A5700002025A6043F61453C2F200034FF0000285
:10A580009A6043F61453C2F200034FF00202DA60FD
:10A5900043F61453C2F200034FF007021A614FF45E
:10A5A0008060C4F2020043F61451C2F20001F8F7D1
:10A5B00025FA43F61453C2F200034FF080021A60EA
:10A5C00043F61453C2F200034FF007021A614FF42E
:10A5D0008060C4F2020043F61451C2F20001F8F7A1
:10A5E0000DFA4FF025004FF000014FF00102FDF78A
:10A5F00005FA4FF02500FDF735FA42F26843C2F242
:10A6000000034FF48052C4F201021A6042F2684320
:10A61000C2F200034FF416525A6042F26843C2F28B
:10A6200000034FF000029A6042F26843C2F2000356
:10A630004FF00002DA6042F26843C2F200034FF0CA
:10A6400000021A6142F26843C2F200034FF00002B6
:10A650009A6142F26843C2F200034FF00C025A6161
:10A6600042F26840C2F20000F5F7CAFE80BD00BFAA
:10A6700080B586B000AF78603960FDF74DFFFEF71A
:10A6800003FA45F24443C0F60103FB6045F2584328
:10A69000C0F60103BB60FEF7C9FB01F035FBFEF716
:10A6A000A3F840F62830C2F20000FEF719FC02F0D1
:10A6B000DFFE02F009FF4FF00000C4F202004FF489
:10A6C00080714FF00102F8F773FD40F22003C2F2EF
:10A6D00000031B881AB240F60413C2F200031B8861
:10A6E0001BB2D11A40F60613C2F200031B781A46B9
:10A6F00040F60413C2F200031B881BB20846114641
:10A700001A46FEF713FA4BF65133C0F6000398478A
:10A71000FEF726FD02F0C6FF4FF0010003F0AEFC8D
:10A720004FF0000003F03AFD4FF0030004F0CCF8C6
:10A730004FF0010004F0F6F84FF6FF704FF0000103
:10A7400004F0D8F84FF000004FF078014FF0C80245
:10A7500003F052FC02F096FA40F68133C2F2000395
:10A760004FF001021A7002F073FD4BF6DD13C0F6D4
:10A77000000398474FF000024FF00003C7E904239D
:10A780004AF64903C0F600034FF0010098474FF026
:10A7900080004FF08001FFF791FDFFF7C3FE42F20A
:10A7A0006840C2F2000040F23401C2F200014FF0F2
:10A7B0001002F5F7F1FEF2E780B586B000AF7860E1
:10A7C00039601F4B3B614FF000037B6119E07B69EF
:10A7D0004FEA83037A68D31893ED007A7B694FEAD6
:10A7E00083037A68D318D3ED007A67EE277A97ED62
:10A7F000047A77EE277AC7ED047A7B6903F10103C7
:10A800007B617A693B689A42E1DB3B6807EE103A6C
:10A81000F8EEC77A97ED047AC7EE277AC7ED047A87
:10A8200007F10C0397ED040A1846FEF701F9FB68DF
:10A8300007EE903AB0EE670A07F11807BD4680BDF3
:10A84000000000000000000090B589B004AF03468E
:10A85000FB7140F61813C2F200034FF001021A70A8
:10A86000FB79002B74D04FF00C0300934FF6FF736D
:10A8700001934FF096004FF05A0145F27C42C0F62A
:10A8800001024FF0280303F001FE4FF0880300930C
:10A890004FF0720301934FF6FF7302934FF07E0067
:10A8A0004FF077014FF088024FF07C0303F094FCE7
:10A8B0004FF00C0300934FF6FF7301934FF0960097
:10A8C0004FF0880147F2B862C0F601024FF02F0343
:10A8D00003F0DCFD4BF2D974C0F600044FF02E00FB
:10A8E0004FF0AE014FF06C024FF6FF73A0474BF2F2
:10A8F000D974C0F600044FF02E004FF0EE014FF077
:10A900006C024FF6FF73A0474FF00A0300934FF617
:10A91000FF7301934FF08E004FF0A20148F64C32C6
:10A92000C0F601024FF09B0303F0B0FD4FF02E0381
:10A9300000934FF6FF73019340F211104FF0C001E6
:10A9400047F62032C0F601024FF02D0303F09EFDC2
:10A9500040F21C03C2F200031B6840F64010C2F232
:10A96000000045F26C41C0F601011A4606F032FFC4
:10A9700040F64013C2F200031A7840F24803C2F2D4
:10A9800000031B7852B25BB29A421CD1FB79002BB8
:10A9900019D140F6FA03C2F200031A8840F21603F6
:10A9A000C2F200031B889A4229D040F6FA03C2F291
:10A9B00000031B88002B06D040F21603C2F20003EE
:10A9C0001B88002B1BD14BF2D974C0F6000440F653
:10A9D0004013C2F200031B785AB240F6FA03C2F2E7
:10A9E00000031B88002B02D14FF4784301E04FF69F
:10A9F000FF7310464FF08E014FF06C02A04740F6F7
:10AA00004013C2F200035A7840F24803C2F2000336
:10AA10005B7852B25BB29A4223D141F64043C2F214
:10AA200000031B78002B1CD1FB79002B19D140F6B9
:10AA3000FA03C2F200031A8840F21603C2F20003BE
:10AA40001B889A4229D040F6FA03C2F200031B8801
:10AA5000002B06D040F21603C2F200031B88002B25
:10AA60001BD14BF2D974C0F6000440F64013C2F279
:10AA700000035B785AB240F6FA03C2F200031B8867
:10AA8000002B02D14FF4784301E04FF6FF731046DC
:10AA90004FF09E014FF06C02A04740F64013C2F207
:10AAA00000039A7840F24803C2F200039B7852B246
:10AAB0005BB29A421CD1FB79002B19D140F6FA0304
:10AAC000C2F200031A8840F21603C2F200031B8888
:10AAD0009A4229D040F6FA03C2F200031B88012BE8
:10AAE00006D040F21603C2F200031B88012B1BD1D3
:10AAF0004BF2D974C0F6000440F64013C2F20003D2
:10AB00009B785AB240F6FA03C2F200031B88012B6D
:10AB100002D14FF4784301E04FF6FF7310464FF037
:10AB2000BE014FF06C02A04740F64013C2F2000392
:10AB3000DA7840F24803C2F20003DB7852B25BB22B
:10AB40009A421CD1FB79002B19D140F6FA03C2F2CC
:10AB500000031A8840F21603C2F200031B889A42CF
:10AB600029D040F6FA03C2F200031B88022B06D05C
:10AB700040F21603C2F200031B88022B1BD14BF2DA
:10AB8000D974C0F6000440F64013C2F20003DB782B
:10AB90005AB240F6FA03C2F200031B88022B02D11C
:10ABA0004FF4784301E04FF6FF7310464FF0CE01AB
:10ABB0004FF06C02A04740F64013C2F200031A792E
:10ABC00040F24803C2F200031B7952B25BB29A42D0
:10ABD0001CD1FB79002B19D140F6FA03C2F2000315
:10ABE0001A8840F21603C2F200031B889A4229D049
:10ABF00040F6FA03C2F200031B88032B06D040F292
:10AC00001603C2F200031B88032B1BD14BF2D9742D
:10AC1000C0F6000440F64013C2F200031B795AB29A
:10AC200040F6FA03C2F200031B88032B02D14FF453
:10AC3000784301E04FF6FF7310464FF0DE014FF00E
:10AC40006C02A04740F64013C2F200035A7940F26A
:10AC50004803C2F200035B7952B25BB29A421CD144
:10AC6000FB79002B19D140F6FA03C2F200031A88CF
:10AC700040F21603C2F200031B889A4229D040F624
:10AC8000FA03C2F200031B88042B06D040F216031D
:10AC9000C2F200031B88042B1BD14BF2D974C0F6FF
:10ACA000000440F64013C2F200035B795AB240F64A
:10ACB000FA03C2F200031B88042B02D14FF478433D
:10ACC00001E04FF6FF7310464FF0FE014FF06C02AB
:10ACD000A04740F64013C2F200039A7940F24803BD
:10ACE000C2F200039B7952B25BB29A421CD1FB794B
:10ACF000002B19D140F6FA03C2F200031A8840F281
:10AD00001603C2F200031B889A4229D040F6FA03C8
:10AD1000C2F200031B88052B06D040F21603C2F2D4
:10AD200000031B88052B1BD14BF2D974C0F600041D
:10AD300040F64013C2F200039B795AB240F6FA0380
:10AD4000C2F200031B88052B02D14FF4784301E0C7
:10AD50004FF6FF7310464FF487714FF06C02A04717
:10AD600040F64013C2F20003DA7940F24803C2F21F
:10AD70000003DB7952B25BB29A421CD1FB79002B03
:10AD800019D140F6FA03C2F200031A8840F2160302
:10AD9000C2F200031B889A4229D040F6FA03C2F29D
:10ADA00000031B88062B06D040F21603C2F20003F4
:10ADB0001B88062B1BD14BF2D974C0F6000440F659
:10ADC0004013C2F20003DB795AB240F6FA03C2F232
:10ADD00000031B88062B02D14FF4784301E04FF6A5
:10ADE000FF7310464FF48F714FF06C02A04740F292
:10ADF0001C03C2F200031A6840F60013C2F20003FB
:10AE00001A6040F24800C2F2000040F64011C2F25F
:10AE1000000106F007FD40F60413C2F200031A8891
:10AE200040F22403C2F200031B8812B21BB29A4202
:10AE30001ED1FB79002B1BD140F6FA03C2F20003AE
:10AE40001A8840F21603C2F200031B889A4200F0EF
:10AE5000998040F6FA03C2F200031B88072B07D043
:10AE600040F21603C2F200031B88072B40F08A80D1
:10AE700040F60413C2F200031B881AB213464FEACD
:10AE800083039B184FEAC30340F64010C2F2000050
:10AE900045F27041C0F601011A4606F09BFC4FF0E6
:10AEA000020003F011FD40F6FA03C2F200031B8812
:10AEB000072B02D14FF4784301E04FF6FF73184699
:10AEC0004FF0000103F016FD4FF0C8004FF087016E
:10AED00003F0E2FC4FF00003FB600EE040F640138D
:10AEE000C2F20003FA689B181B78DBB2184603F025
:10AEF00057FBFB6803F10103FB60FB68032BEDDDEF
:10AF00004FF0000300934FF079004FF078014FF0BD
:10AF100003024FF0640303F01DF940F60413C2F27C
:10AF200000031B881BB24FEAD372D3184FEA6303A6
:10AF30009BB21BB203F1780240F22003C2F200037D
:10AF40001B8819B240F60413C2F200031B881BB21F
:10AF5000CB1A4FEAD371CB184FEA63034FF6FF7158
:10AF600000914FF0790011464FF0030203F0F2F820
:10AF700040F60413C2F200031A8840F22403C2F21E
:10AF800000031A8040F22003C2F200031A8840F244
:10AF90002203C2F200031B8812B21BB29A421ED1D6
:10AFA000FB79002B1BD140F6FA03C2F200031A888A
:10AFB00040F21603C2F200031B889A4200F0998007
:10AFC00040F6FA03C2F200031B88082B07D040F2B8
:10AFD0001603C2F200031B88082B40F08A8040F25F
:10AFE0002003C2F200031B881AB213464FEA830300
:10AFF0009B184FEAC30340F64010C2F2000045F22E
:10B000007441C0F601011A4606F0E4FB4FF002005D
:10B0100003F05AFC40F6FA03C2F200031B88082B27
:10B0200002D14FF4784301E04FF6FF7318464FF01A
:10B03000000103F05FFC40F209104FF0870103F0BC
:10B040002BFC4FF00003BB600EE040F64013C2F251
:10B050000003BA689B181B78DBB2184603F0A0FA0D
:10B06000BB6803F10103BB60BB68032BEDDD4FF050
:10B07000000300934FF079004FF078014FF0030286
:10B080004FF0640303F066F840F60413C2F20003C5
:10B090001B881BB24FEAD372D3184FEA63039BB2EB
:10B0A0001BB203F1780240F22003C2F200031B88B6
:10B0B00019B240F60413C2F200031B881BB2CB1A6C
:10B0C0004FEAD371CB184FEA63034FF6FF7100913B
:10B0D0004FF0790011464FF0030203F03BF840F2C5
:10B0E0002003C2F200031A8840F22203C2F20003D6
:10B0F0001A8040F60613C2F200031A7840F22603C3
:10B10000C2F200031B789A421CD1FB79002B19D1A3
:10B1100040F6FA03C2F200031A8840F21603C2F2A4
:10B1200000031B889A4279D040F6FA03C2F200036A
:10B130001B88092B06D040F21603C2F200031B88BD
:10B14000092B6BD140F60613C2F200031B78012BCA
:10B1500020D0022B3BD0002B56D140F6FA03C2F28E
:10B1600000031B88092B02D14FF4784301E04FF60E
:10B17000FF734FF00902009201934FF0C4004FF0AB
:10B180005B0145F63C02C0F601024FF01C0303F0E0
:10B190007DF939E040F6FA03C2F200031B88092B5F
:10B1A00002D14FF4784301E04FF6FF734FF00902EC
:10B1B000009201934FF0C4004FF05B0145F634223A
:10B1C000C0F601024FF01C0303F060F91CE040F6EA
:10B1D000FA03C2F200031B88092B02D14FF4784313
:10B1E00001E04FF6FF734FF00902009201934FF018
:10B1F000C4004FF05B0145F62C42C0F601024FF04F
:10B200001C0303F043F900BF40F60613C2F200032B
:10B210001A7840F22603C2F200031A7040F21003BB
:10B22000C2F200031B68184605F04AFC02460B46B2
:10B230001046194612A3D3E9002305F095FC0246F7
:10B240000B461046194610A3D3E9002305F0F4FE7F
:10B250000346002B09D140F6FA03C2F200031A8814
:10B2600040F21603C2F200031A8040F61813C2F22D
:10B2700000034FF000021A7007F11407BD4690BD9D
:10B28000AE47E17A14AEEF3F00000000000000007E
:10B2900080B485B000AF786039604FF00003FB6088
:10B2A0000AE0FB684FEA83033A68D3180B4A1A6036
:10B2B000FB6803F10103FB60FA6840F2FF139A4256
:10B2C000EFDD7B684FEA83033A68D318044A1A60BB
:10B2D00007F11407BD4680BC704700BF00000000A6
:10B2E0000000803F80B588B000AF40F62133C2F245
:10B2F00000031B78DBB2002B00F0648240F61C13C5
:10B30000C2F200031B68012B40F0FE8040F61413CC
:10B31000C2F200031B68002B78D13B4618464FF45D
:10B3200080714FF000024FF0010303F00BFB3B462E
:10B33000184642F6A841C2F2000104F0FFFE40F6B2
:10B340001013C2F200031B68002B25D140F628130E
:10B35000C2F200031B78012B1ED04FF00003FB83C9
:10B3600015E0F98BFA8B42F6A843C2F200034FEACC
:10B3700082029B181A6842F2A443C2F200034FEA09
:10B3800081015B181A60FB8B03F10103FB83FA8BCD
:10B3900040F2FF139A42E4D940F60C13C2F20003C4
:10B3A0001B6842F6A840C2F200001946FDF770FC87
:10B3B00040F61013C2F200031B68012B32D140F695
:10B3C0002813C2F200031B78012B2BD04FF000038F
:10B3D000BB8315E0B98BBA8B42F6A843C2F20003D7
:10B3E0004FEA82029B181A6842F2A443C2F2000399
:10B3F0004FEA81015B181A60BB8B03F10103BB8329
:10B40000BA8B40F2FF139A42E4D90BE040F61413D2
:10B41000C2F200031B68184642F6A841C2F20001BE
:10B42000FFF736FF3B4618464FF480714FF001029C
:10B430004FF0010303F086FA3B46184642F6A84156
:10B44000C2F2000104F07AFE40F60613C2F20003D5
:10B450001B78022B40D142F6A840C2F2000043F212
:10B46000A841C2F200014FF4807204F0D3FF4FF004
:10B4700000037B832DE07B8B4FEA43017A8B43F201
:10B48000A843C2F200034FEA82029B181A6842F6F0
:10B49000A843C2F200034FEA81015B181A607B8B5C
:10B4A0004FEA430303F101017A8B43F2A843C2F24E
:10B4B00000034FEA82029B181A6842F6A843C2F2C0
:10B4C00000034FEA81015B181A607B8B03F10103D3
:10B4D0007B837B8BFF2BCED942F6A840C2F20000C3
:10B4E0004FF40071FFF768F9F0EE407A40F6301340
:10B4F000C2F20003C3ED007A40F61C13C2F200034F
:10B500004FF000021A6056E140F62013C2F2000329
:10B510001B68012B40F0A48040F61413C2F2000314
:10B520001B68002B1ED13B4618464FF480714FF02C
:10B5300000024FF0010303F005FA3B46184641F2C2
:10B540004041C2F2000104F0F9FD40F60C13C2F2D2
:10B5500000031B6841F24040C2F200001946FDF7AB
:10B5600097FB0BE040F61413C2F200031B68184669
:10B5700041F24041C2F20001FFF78AFE3B46184605
:10B580004FF480714FF001024FF0010303F0DAF93C
:10B590003B46184641F24041C2F2000104F0CEFDA4
:10B5A00040F60613C2F200031B78022B40D141F291
:10B5B0004040C2F2000043F2A841C2F200014FF441
:10B5C000807204F027FF4FF000033B832DE03B8B9C
:10B5D0004FEA43013A8B43F2A843C2F200034FEA19
:10B5E00082029B181A6841F24043C2F200034FEAFC
:10B5F00081015B181A603B8B4FEA430303F10101A1
:10B600003A8B43F2A843C2F200034FEA82029B182E
:10B610001A6841F24043C2F200034FEA81015B180D
:10B620001A603B8B03F101033B833B8BFF2BCED98D
:10B6300041F24040C2F200004FF40071FFF7BCF845
:10B64000F0EE407A40F63013C2F20003C3ED007A08
:10B6500040F62013C2F200034FF000021A60AAE085
:10B6600040F62413C2F200031B68012B40F0A380B4
:10B6700040F61413C2F200031B68002B1ED13B4698
:10B6800018464FF480714FF000024FF0010303F0B1
:10B6900059F93B46184641F66041C2F2000104F0F8
:10B6A0004DFD40F60C13C2F200031B6841F66040EA
:10B6B000C2F200001946FDF7EBFA0BE040F6141356
:10B6C000C2F200031B68184641F66041C2F2000155
:10B6D000FFF7DEFD3B4618464FF480714FF0010244
:10B6E0004FF0010303F02EF93B46184641F6604146
:10B6F000C2F2000104F022FD40F60613C2F200037C
:10B700001B78022B40D141F66040C2F2000043F2A8
:10B71000A841C2F200014FF4807204F07BFE4FF0AA
:10B720000003FB822DE0FB8A4FEA4301FA8A43F2D1
:10B73000A843C2F200034FEA82029B181A6841F63E
:10B740006043C2F200034FEA81015B181A60FB8A72
:10B750004FEA430303F10101FA8A43F2A843C2F21C
:10B7600000034FEA82029B181A6841F66043C2F256
:10B7700000034FEA81015B181A60FB8A03F10103A1
:10B78000FB82FB8AFF2BCED941F66040C2F200005B
:10B790004FF40071FFF710F8F0EE407A40F63013E6
:10B7A000C2F20003C3ED007A40F62413C2F2000394
:10B7B0004FF000021A6040F62133C2F200034FF04E
:10B7C00000021A7040F6D420C2F20000F5F7C2FC65
:10B7D00007F12007BD4680BD80B584B002AFF87187
:10B7E000B9807A803B8097F90730A3F12E030B2BA9
:10B7F00000F2E28001A252F823F000BF2DB8000849
:10B80000B9B9000895B9000851B8000875B8000822
:10B8100099B80008BDB80008E1B8000805B90008EB
:10B8200029B900084DB9000871B90008BA887B88A9
:10B8300039884FF01300009001911046194645F6E3
:10B840002462C0F601024FF00F0302F01FFEC0E0B9
:10B85000BA887B8839884FF0130000900191104618
:10B86000194646F26002C0F601024FF00F0302F0E3
:10B870000DFEAEE0BA887B8839884FF01300009047
:10B8800001911046194646F29C22C0F601024FF083
:10B890000F0302F0FBFD9CE0BA887B8839884FF0EB
:10B8A0001300009001911046194646F2D842C0F6A6
:10B8B00001024FF00F0302F0E9FD8AE0BA887B88AD
:10B8C00039884FF01300009001911046194646F256
:10B8D0001472C0F601024FF00F0302F0D7FD78E0BA
:10B8E000BA887B8839884FF0130000900191104688
:10B8F000194646F65012C0F601024FF00F0302F04F
:10B90000C5FD66E0BA887B8839884FF01300009047
:10B9100001911046194646F68C32C0F601024FF0EE
:10B920000F0302F0B3FD54E0BA887B8839884FF0EA
:10B930001300009001911046194646F6C852C0F611
:10B9400001024FF00F0302F0A1FD42E0BA887B88AC
:10B9500039884FF01300009001911046194647F2C4
:10B960000402C0F601024FF00F0302F08FFD30E039
:10B97000BA887B8839884FF01300009001911046F7
:10B98000194647F24022C0F601024FF00F0302F0C1
:10B990007DFD1EE0BA887B8839884FF01300009047
:10B9A00001911046194647F27C42C0F601024FF061
:10B9B0000F0302F06BFD0CE0BA887B884FF00001AA
:10B9C0000091104619464FF00F024FF0130302F09A
:10B9D000C1FB07F10807BD4680BD00BF80B500AFC1
:10B9E00040F20C03C2F200031A684DF62913C6F2A6
:10B9F0004263A3FB02134FEA136303F1FF3240F6E5
:10BA00003413C2F200031A604FF46053C4F202030D
:10BA10004FF46052C4F20202126C42F002021A6445
:10BA200040F68C33C2F200034FF48062C4F200028D
:10BA30001A6040F68C33C2F200034FF000029A60A5
:10BA400040F68C33C2F2000340F21A42DA6040F64C
:10BA50003413C2F200031A6840F68C33C2F20003BA
:10BA60005A6040F68C33C2F200034FF000021A61B4
:10BA700040F68C30C2F20000F5F7D4F840F68C3076
:10BA8000C2F20000F5F7ACF94FF01D004FF00001D5
:10BA90004FF00102FBF7B2FF4FF01D00FBF7E2FF92
:10BAA0004FF46053C4F202034FF46052C4F2020236
:10BAB000126C42F004021A6440F6D423C2F200036E
:10BAC0004FF40062C4F200021A6040F6D423C2F2BE
:10BAD00000034FF000029A6040F6D423C2F2000344
:10BAE00040F21A42DA6040F63413C2F200031A68D8
:10BAF00040F6D423C2F200035A6040F6D423C2F2C7
:10BB000000034FF000021A6140F6D420C2F2000098
:10BB1000F5F788F840F6D420C2F20000F5F760F996
:10BB20004FF01E004FF002014FF00402FBF766FFDA
:10BB30004FF01E00FBF796FF80BD00BF80B582B0BE
:10BB400000AF7860FDF738FC07F10807BD4680BDFF
:10BB500080B500AF4FF46053C4F202034FF460525B
:10BB6000C4F20202126C42F000521A6443F600530F
:10BB7000C2F200034FF4E842C4F200021A6043F636
:10BB80000050C2F20000FBF73FFC0346002B01D03F
:10BB9000FDF7A4FA40F63813C2F200034FF000029A
:10BBA0001A6040F63813C2F200034FF000025A60E8
:10BBB00043F60050C2F2000040F63811C2F2000114
:10BBC0004FF00002FBF7DEFC0346002B01D0FDF72F
:10BBD00085FA43F60050C2F2000040F63811C2F276
:10BBE00000014FF01002FBF7CDFC0346002B01D003
:10BBF000FDF774FA43F60050C2F200004FF0000166
:10BC00004FF000024FF08803FBF792FD0346002B34
:10BC100001D0FDF763FA43F60050C2F200004FF086
:10BC200010014FF000024FF08803FBF781FD03463F
:10BC3000002B01D0FDF752FA43F60050C2F200008B
:10BC40004FF00001FBF720FC0346002B01D0FDF76D
:10BC500045FA43F60050C2F200004FF01001FBF726
:10BC600013FC0346002B01D0FDF738FA80BD00BF5E
:10BC700080B582B000AF0346FB80FB884FEA0353D8
:10BC80004FEA1353FB80FB8843F60050C2F20000DA
:10BC90004FF000014FF00002FBF74AFD07F10807E3
:10BCA000BD4680BD80B582B000AF0346FB80FB88F7
:10BCB0004FEA03534FEA1353FB80FB8843F60050CF
:10BCC000C2F200004FF010014FF00002FBF730FD10
:10BCD00007F10807BD4680BD80B483B000AF78602F
:10BCE00040F6D023C2F200037A681A6000BF40F623
:10BCF000D023C2F200031B68002BF8D107F10C0718
:10BD0000BD4680BC704700BF80B586B000AF49F229
:10BD10006873C0F601039B887B604FF002033B61B0
:10BD20004FF00203BB604FF00203FB604FF00103D2
:10BD30007B6149F26873C0F601031A6807F10403D6
:10BD400010461946F6F75AFE49F27073C0F6010321
:10BD50009B887B604FF002033B614FF00203BB60A6
:10BD60004FF00203FB604FF001037B6149F27073F7
:10BD7000C0F601031A6807F1040310461946F6F7E6
:10BD80003DFE49F28073C0F601039B887B604FF053
:10BD900002033B614FF00103BB604FF000037B6186
:10BDA0004FF00003FB6049F28073C0F601031A688C
:10BDB00007F1040310461946F6F720FE49F288738E
:10BDC000C0F601039B887B604FF002033B614FF09C
:10BDD0000103BB604FF000037B614FF00003FB6089
:10BDE00049F28873C0F601031A6807F1040310468C
:10BDF0001946F6F703FE49F29873C0F601039B88D3
:10BE00007B604FF000033B614FF01103BB604FF0CC
:10BE100000037B614FF00003FB6049F29873C0F6AA
:10BE200001031A6807F1040310461946F6F7E6FD08
:10BE300049F29873C0F601031A6849F29873C0F684
:10BE400001039B88104619464FF00002F7F7B0F93E
:10BE500049F27873C0F601039B887B604FF00203C0
:10BE60003B614FF00303BB604FF00003FB604FF0FA
:10BE700000037B6149F27873C0F601031A6807F189
:10BE8000040310461946F6F7B9FD49F2F873C0F6F7
:10BE900001039B887B604FF002033B614FF000037E
:10BEA000BB604FF00103FB604FF000037B6149F280
:10BEB000F873C0F601031A6807F104031046194627
:10BEC000F6F79CFD49F60003C0F601039B887B60F2
:10BED0004FF002033B614FF00003BB604FF00103E2
:10BEE000FB604FF000037B6149F60003C0F60103DD
:10BEF0001A6807F1040310461946F6F77FFD49F664
:10BF00000803C0F601039B887B604FF002033B618E
:10BF10004FF00003BB604FF00103FB604FF00003E4
:10BF20007B6149F60803C0F601031A6807F10403B0
:10BF300010461946F6F762FD49F61003C0F60103F4
:10BF40009B887B604FF002033B614FF00303BB60B3
:10BF50004FF00003FB604FF000037B6149F61003D4
:10BF6000C0F601031A6807F1040310461946F6F7F4
:10BF700045FD49F61803C0F601039B887B604FF02E
:10BF800002033B614FF00303BB604FF00003FB6013
:10BF90004FF000037B6149F61803C0F601031A68ED
:10BFA00007F1040310461946F6F728FD49F2A0737D
:10BFB000C0F601039B887B604FF00103BB604FF02C
:10BFC00002033B614FF00103FB6049F2A073C0F62E
:10BFD00001031A6807F1040310461946F6F70EFD2F
:10BFE00049F2A073C0F601031A6849F2A073C0F6C3
:10BFF00001039B88104619464FF00002F7F7D8F866
:10C0000049F2A873C0F601039B887B604FF00103DF
:10C01000BB604FF002033B614FF00103FB6049F24C
:10C02000A873C0F601031A6807F104031046194605
:10C03000F6F7E4FC49F2A873C0F601031A6849F266
:10C04000A873C0F601039B88104619464FF0000202
:10C05000F7F7AEF849F2B073C0F601039B887B6036
:10C060004FF00103BB604FF002033B614FF001034F
:10C07000FB6049F2B073C0F601031A6807F10403CC
:10C0800010461946F6F7BAFC49F2B073C0F6010340
:10C090001A6849F2B073C0F601039B88104619462E
:10C0A0004FF00002F7F784F849F2C073C0F60103BD
:10C0B0009B887B604FF00103BB604FF002033B6144
:10C0C0004FF00103FB6049F2C073C0F601031A6828
:10C0D00007F1040310461946F6F790FC49F2C073C5
:10C0E000C0F601031A6849F2C073C0F601039B88C9
:10C0F000104619464FF00102F7F75AF849F2B873A3
:10C10000C0F601039B887B604FF00103BB604FF0DA
:10C1100002033B614FF00103FB6049F2B873C0F6C4
:10C1200001031A6807F1040310461946F6F766FC86
:10C1300049F2B873C0F601031A6849F2B873C0F641
:10C1400001039B88104619464FF00102F7F730F8BB
:10C1500049F2C873C0F601039B887B604FF001036E
:10C16000BB604FF002033B614FF00103FB6049F2FB
:10C17000C873C0F601031A6807F104031046194694
:10C18000F6F73CFC49F2C873C0F601031A6849F29D
:10C19000C873C0F601039B88104619464FF0000291
:10C1A000F7F706F849F2D873C0F601039B887B6065
:10C1B0004FF00103BB604FF002033B614FF00103FE
:10C1C000FB6049F2D873C0F601031A6807F1040353
:10C1D00010461946F6F712FC49F2D873C0F601036F
:10C1E0001A6849F2D873C0F601039B8810461946B5
:10C1F0004FF00102F6F7DCFF49F2D073C0F60103FD
:10C200009B887B604FF00103BB604FF002033B61F2
:10C210004FF00103FB6049F2D073C0F601031A68C6
:10C2200007F1040310461946F6F7E8FB49F2D0730C
:10C23000C0F601031A6849F2D073C0F601039B8867
:10C24000104619464FF00102F6F7B2FF49F62003F7
:10C25000C0F601039A8849F62803C0F601039B88BB
:10C2600013439BB27B604FF00303BB604FF00003AE
:10C27000FB6049F62003C0F601031A6807F10403C6
:10C2800010461946F6F7BAFB49F63003C0F601032B
:10C290009B887B604FF00103BB604FF000033B6164
:10C2A0004FF00003FB6049F63003C0F601031A6843
:10C2B00007F1040310461946F6F7A0FB49F63003D0
:10C2C000C0F601031A6849F63003C0F601039B88E3
:10C2D000104619464FF00102F6F76AFF49F6380397
:10C2E000C0F601039B887B604FF00103BB604FF0F9
:10C2F00000033B614FF00003FB6049F63803C0F6D2
:10C3000001031A6807F1040310461946F6F776FB95
:10C3100049F63803C0F601031A6849F63803C0F637
:10C3200001039B88104619464FF00002F6F740FFC4
:10C3300049F64003C0F601039B887B604FF0010380
:10C34000BB604FF000033B614FF00003FB6049F618
:10C350004003C0F601031A6807F1040310461946AA
:10C36000F6F74CFB49F64003C0F601031A6849F69C
:10C370004003C0F601039B88104619464FF00002A7
:10C38000F6F716FF49F64803C0F601039B887B6069
:10C390004FF00103BB604FF000033B614FF000031F
:10C3A000FB6049F64803C0F601031A6807F104036D
:10C3B00010461946F6F722FB49F64803C0F601037A
:10C3C0001A6849F64803C0F601039B8810461946CF
:10C3D0004FF00102F6F7ECFE49F65003C0F60103F8
:10C3E0009B887B604FF00103BB604FF000033B6113
:10C3F0004FF00003FB6049F65003C0F601031A68D2
:10C4000007F1040310461946F6F7F8FA49F6500307
:10C41000C0F601031A6849F65003C0F601039B8871
:10C42000104619464FF00002F6F7C2FE49F688039F
:10C43000C0F601039B887B604FF00103BB604FF0A7
:10C4400000033B614FF00003FB6049F68803C0F630
:10C4500001031A6807F1040310461946F6F7CEFAED
:10C4600049F68803C0F601031A6849F68803C0F646
:10C4700001039B88104619464FF00102F6F798FE1B
:10C4800049F69003C0F601039B887B604FF00103DF
:10C49000BB604FF000033B614FF00003FB6049F6C7
:10C4A0009003C0F601031A6807F104031046194609
:10C4B000F6F7A4FA49F69003C0F601031A6849F6A4
:10C4C0009003C0F601039B88104619464FF0000206
:10C4D000F6F76EFE49F67803C0F601039B887B6091
:10C4E0004FF00103BB604FF000033B614FF00003CE
:10C4F000FB6049F67803C0F601031A6807F10403EC
:10C5000010461946F6F77AFA49F67803C0F60103A1
:10C510001A6849F67803C0F601039B88104619464D
:10C520004FF00002F6F744FE49F68003C0F601031F
:10C530009B887B604FF00103BB604FF000033B61C1
:10C540004FF00003FB6049F68003C0F601031A6850
:10C5500007F1040310461946F6F750FA49F680032E
:10C56000C0F601031A6849F68003C0F601039B88F0
:10C57000104619464FF00102F6F71AFE49F6680315
:10C58000C0F601039B887B604FF00103BB604FF056
:10C5900000033B614FF00003FB6049F66803C0F6FF
:10C5A00001031A6807F1040310461946F6F726FA44
:10C5B00049F66803C0F601031A6849F66803C0F635
:10C5C00001039B88104619464FF00002F6F7F0FD74
:10C5D00049F67003C0F601039B887B604FF00103AE
:10C5E000BB604FF000033B614FF00003FB6049F676
:10C5F0007003C0F601031A6807F1040310461946D8
:10C60000F6F7FCF949F67003C0F601031A6849F61B
:10C610007003C0F601039B88104619464FF00102D3
:10C62000F6F7C6FD49F65803C0F601039B887B6008
:10C630004FF00103BB604FF000033B614FF000037C
:10C64000FB6049F65803C0F601031A6807F10403BA
:10C6500010461946F6F7D2F949F65803C0F6010319
:10C660001A6849F65803C0F601039B88104619461C
:10C670004FF00002F6F79CFD49F66003C0F6010397
:10C680009B887B604FF00103BB604FF000033B6170
:10C690004FF00003FB6049F66003C0F601031A681F
:10C6A00007F1040310461946F6F7A8F949F66003A6
:10C6B000C0F601031A6849F66003C0F601039B88BF
:10C6C000104619464FF00102F6F772FD49F6A00335
:10C6D000C0F601039B887B604FF01103BB604FF0F5
:10C6E00000033B614FF00103FB6049F6A003C0F675
:10C6F00001031A6807F1040310461946F6F77EF99C
:10C7000049F6A003C0F601031A6849F6A003C0F673
:10C7100001039B88104619464FF00102F6F748FDC9
:10C7200049F69803C0F601039B887B604FF0110324
:10C73000BB604FF000033B614FF00103FB6049F623
:10C740009803C0F601031A6807F10403104619465E
:10C75000F6F754F949F69803C0F601031A6849F64A
:10C760009803C0F601039B88104619464FF001025A
:10C77000F6F71EFD49F6B003C0F601039B887B6007
:10C780004FF00103BB604FF000033B614FF000032B
:10C79000FB6049F6B003C0F601031A6807F1040311
:10C7A00010461946F6F72AF949F6B003C0F6010318
:10C7B0001A6849F6B003C0F601039B881046194673
:10C7C0004FF00102F6F7F4FC49F6A803C0F60103A6
:10C7D0009B887B604FF00103BB604FF000033B611F
:10C7E0004FF00003FB6049F6A803C0F601031A6886
:10C7F00007F1040310461946F6F700F949F6A803B5
:10C80000C0F601031A6849F6A803C0F601039B8825
:10C81000104619464FF00102F6F7CAFC49F6B80374
:10C82000C0F601039B887B604FF00103BB604FF0B3
:10C8300000033B614FF00003FB6049F6B803C0F60C
:10C8400001031A6807F1040310461946F6F7D6F8F3
:10C8500049F6B803C0F601031A6849F6B803C0F6F2
:10C8600001039B88104619464FF00102F6F7A0FC21
:10C8700049F6C003C0F601039B887B604FF00103BB
:10C88000BB604FF000033B614FF00003FB6049F6D3
:10C89000C003C0F601031A6807F1040310461946E5
:10C8A000F6F7ACF849F6C003C0F601031A6849F67A
:10C8B000C003C0F601039B88104619464FF00102E1
:10C8C000F6F776FC49F6D003C0F601039B887B603F
:10C8D0004FF00103BB604FF000033B614FF00003DA
:10C8E000FB6049F6D003C0F601031A6807F10403A0
:10C8F00010461946F6F782F849F6D003C0F6010350
:10C900001A6849F6D003C0F601039B881046194601
:10C910004FF00102F6F74CFC49F6C803C0F60103DC
:10C920009B887B604FF00103BB604FF000033B61CD
:10C930004FF00003FB6049F6C803C0F601031A6814
:10C9400007F1040310461946F6F758F849F6C803EC
:10C95000C0F601031A6849F6C803C0F601039B88B4
:10C96000104619464FF00102F6F722FC49F6D803AB
:10C97000C0F601039B887B604FF00303BB604FF060
:10C9800000033B614FF00003FB6049F6D803C0F69B
:10C9900001031A6807F1040310461946F6F72EF84A
:10C9A00049F6D803C0F601031A6849F6D803C0F661
:10C9B00001039B88104619464FF00002F6F7F8FB7A
:10C9C00049F6E003C0F601039B887B604FF0030348
:10C9D000BB604FF000033B614FF00003FB6049F682
:10C9E000E003C0F601031A6807F104031046194674
:10C9F000F6F704F849F6E803C0F601039B887B606C
:10CA00004FF00103BB604FF000033B614FF00003A8
:10CA1000FB6049F6E803C0F601031A6807F1040356
:10CA200010461946F5F7EAFF49F6E803C0F6010398
:10CA30001A6849F6E803C0F601039B8810461946B8
:10CA40004FF00102F6F7B4FB49F6F003C0F601031C
:10CA50009B887B604FF00103BB604FF000033B619C
:10CA60004FF00003FB6049F6F003C0F601031A68BB
:10CA700007F1040310461946F5F7C0FF49F6F00325
:10CA8000C0F601031A6849F6F003C0F601039B885B
:10CA9000104619464FF00102F6F78AFB49F60813D3
:10CAA000C0F601039B887B604FF00003BB604FF032
:10CAB00000033B614FF00103FB6049F60813C0F629
:10CAC00001031A6807F1040310461946F5F796FFAB
:10CAD00049F61013C0F601039B887B604FF00003FA
:10CAE000BB604FF000033B614FF00103FB6049F670
:10CAF0001013C0F601031A6807F104031046194623
:10CB0000F5F77CFF49F6F803C0F601039B887B60CC
:10CB10004FF00003BB604FF000033B614FF0000398
:10CB2000FB6049F6F803C0F601031A6807F1040335
:10CB300010461946F5F762FF49F60013C0F60103E7
:10CB40009B887B604FF00003BB604FF000033B61AC
:10CB50004FF00003FB6049F60013C0F601031A68AA
:10CB600007F1040310461946F5F748FF49F630135C
:10CB7000C0F601039B887B604FF000033B614FF0E0
:10CB80000103BB604FF00103FB6049F63013C0F6B0
:10CB900001031A6807F1040310461946F5F72EFF42
:10CBA00049F63013C0F601031A6849F63013C0F68F
:10CBB00001039B88104619464FF00002F6F7F8FA79
:10CBC00049F61813C0F601039B887B604FF0000301
:10CBD0003B614FF00103BB604FF00003FB6049F67F
:10CBE0001813C0F601031A6807F10403104619462A
:10CBF000F5F704FF49F63013C0F601031A6849F649
:10CC00003013C0F601039B88104619464FF000020E
:10CC1000F6F7CEFA49F62013C0F601039B887B6035
:10CC20004FF000033B614FF00003BB604FF0000387
:10CC3000FB6049F62013C0F601031A6807F10403EC
:10CC400010461946F5F7DAFE49F62813C0F6010337
:10CC50009B887B604FF000033B614FF00003BB609B
:10CC60004FF00003FB6049F62813C0F601031A6871
:10CC700007F1040310461946F5F7C0FE07F118073F
:10CC8000BD4680BD80B500AF40F62C23C2F2000344
:10CC90004FF000021A8040F6CC23C2F200034FF09E
:10CCA00000021A8040F68133C2F200034FF0000206
:10CCB0001A7040F68A33C2F200034FF064021A8001
:10CCC00040F62133C2F200034FF000021A7040F622
:10CCD0002033C2F200034FF000021A704FF4605389
:10CCE000C4F202034FF46052C4F20202526C42F4E6
:10CCF00080725A644FF46053C4F202034FF46052DE
:10CD0000C4F20202526C42F400725A644FF460534F
:10CD1000C4F202034FF46052C4F20202526C42F4B5
:10CD200080625A644FF46053C4F202034FF46052BD
:10CD3000C4F20202126B42F001021A634FF4605314
:10CD4000C4F202034FF46052C4F20202126B42F0CA
:10CD500002021A634FF46053C4F202034FF46052AC
:10CD6000C4F20202126B42F004021A634FF46053E1
:10CD7000C4F202034FF46052C4F20202526A42F457
:10CD800080725A624FF46053C4F202034FF460524F
:10CD9000C4F20202526A22F480725A6240F64423BC
:10CDA000C2F200034FF40052C4F201021A6040F6CE
:10CDB0004423C2F200034FF000025A6040F64423BD
:10CDC000C2F200034FF000029A6040F64423C2F220
:10CDD00000034FF000021A6140F64423C2F2000340
:10CDE0004FF001029A6140F64423C2F200034FF073
:10CDF00000025A6240F64423C2F200034FF00002E0
:10CE00009A6240F64423C2F200034FF00002DA6255
:10CE100040F64423C2F200034FF000021A6340F6CA
:10CE20004423C2F200034FF00002DA6040F64423CC
:10CE3000C2F200034FF001021A6240F64423C2F22C
:10CE400000034FF00002DA6140F64423C2F200030F
:10CE50004FF000025A6140F64420C2F20000FAF797
:10CE60001DFE0346002B0CD040F62033C2F2000317
:10CE70001B7803F10103DAB240F62033C2F200035B
:10CE80001A7040F68823C2F200034FF40452C4F231
:10CE900001021A6040F68823C2F200034FF000023C
:10CEA0005A6040F68823C2F200034FF000029A60F5
:10CEB00040F68823C2F200034FF000021A6140F6E8
:10CEC0008823C2F200034FF001029A6140F68823E2
:10CED000C2F200034FF000025A6240F68823C2F209
:10CEE00000034FF000029A6240F68823C2F200036A
:10CEF0004FF00002DA6240F68823C2F200034FF0DE
:10CF000000021A6340F68823C2F200034FF00002C9
:10CF1000DA6040F68823C2F200034FF001021A6281
:10CF200040F68823C2F200034FF00002DA6140F6B7
:10CF30008823C2F200034FF000025A6140F68820B5
:10CF4000C2F20000FAF7AAFD0346002B0CD040F60F
:10CF50002033C2F200031B7803F10103DAB240F67A
:10CF60002033C2F200031A7040F6C833C2F2000345
:10CF70004FF40852C4F201021A6040F6C833C2F2FC
:10CF800000034FF000025A6040F6C833C2F20003BB
:10CF90004FF000029A6040F6C833C2F200034FF02F
:10CFA00000021A6140F6C833C2F200034FF00102DA
:10CFB0009A6140F6C833C2F200034FF000025A6291
:10CFC00040F6C833C2F200034FF000029A6240F606
:10CFD000C833C2F200034FF00002DA6240F6C833F1
:10CFE000C2F200034FF000021A6340F6C833C2F2E7
:10CFF00000034FF00002DA6040F6C833C2F20003CB
:10D000004FF001021A6240F6C833C2F200034FF03B
:10D010000002DA6140F6C833C2F200034FF00002AA
:10D020005A6140F6C830C2F20000FAF737FD0346F5
:10D03000002B0CD040F62033C2F200031B7803F122
:10D040000103DAB240F62033C2F200031A7040F650
:10D050003023C2F200034FF009021A6040F6302379
:10D06000C2F200034FF001025A6040F63023C2F2D0
:10D0700000034FF000029A6040F63023C2F2000332
:10D080004FF00002DA6040F60C43C2F200034FF0AA
:10D0900006021A6040F60C43C2F200034FF0010290
:10D0A0005A6040F60C43C2F200034FF000029A604F
:10D0B00040F60C43C2F200034FF00002DA6040F683
:10D0C0001033C2F200034FF003021A6040F610332F
:10D0D000C2F200034FF001025A6040F61033C2F270
:10D0E00000034FF000029A6040F61033C2F20003D2
:10D0F0004FF00002DA6040F64420C2F2000040F631
:10D100003021C2F20001FAF731FF0346002B0CD0A8
:10D1100040F62033C2F200031B7803F10103DAB2B8
:10D1200040F62033C2F200031A7040F68820C2F2A3
:10D13000000040F60C41C2F20001FAF717FF034667
:10D14000002B0CD040F62033C2F200031B7803F111
:10D150000103DAB240F62033C2F200031A7040F63F
:10D16000C830C2F2000040F61031C2F20001FAF7F6
:10D17000FDFE0346002B0CD040F62033C2F2000324
:10D180001B7803F10103DAB240F62033C2F2000348
:10D190001A7080BD80B500AF40F64420C2F2000096
:10D1A0004FF00A01FAF792FE40F68820C2F2000022
:10D1B0004FF00A01FAF78AFE40F6C830C2F20000CA
:10D1C0004FF00A01FAF782FE40F64420C2F2000056
:10D1D000FBF788F80346152B38D140F68820C2F2B9
:10D1E0000000FBF77FF80346152B2FD140F6C8301F
:10D1F000C2F20000FBF776F80346152B26D140F665
:10D200004420C2F20000FAF7A3FE03469AB240F6A9
:10D210002C23C2F200031A8040F68820C2F20000DC
:10D22000FAF796FE03469AB240F6CC23C2F2000308
:10D230001A8040F6C830C2F20000FAF789FE0346B1
:10D240009AB240F67E33C2F200031A8080BD00BF5E
:10D2500080B500AF40F64420C2F20000FAF796FD18
:10D260000346002B0CD040F62033C2F200031B789B
:10D2700003F10103DAB240F62033C2F200031A7060
:10D2800040F68820C2F20000FAF780FD0346002B2A
:10D290000CD040F62033C2F200031B7803F10103E7
:10D2A000DAB240F62033C2F200031A7040F6C830FA
:10D2B000C2F20000FAF76AFD0346002B0CD040F6DC
:10D2C0002033C2F200031B7803F10103DAB240F607
:10D2D0002033C2F200031A7080BD00BF80B500AFDA
:10D2E000FBF7DAF94FF46D43CEF200034FF46D42D1
:10D2F000CEF20002D2F8882042F47002C3F88820EF
:10D30000FBF70AF900F002F880BD00BF80B592B0CB
:10D3100000AF4FF46053C4F202034FF46052C4F202
:10D320000202126C42F080521A644FF4E043C4F2DD
:10D3300000034FF4E042C4F20002126842F440429B
:10D340001A604FF001037B604FF00103BB604FF0A8
:10D350000203FB614FF480033B624FF018037B62D2
:10D360004FF4A873BB624FF00203FB624FF0070358
:10D370003B6307F104031846F4F7B2FB4FF00F03C9
:10D380007B634FF00203BB634FF00003FB634FF47A
:10D39000A0533B644FF480537B6407F13403184679
:10D3A0004FF00501F4F754FF07F14807BD4680BD73
:10D3B00080B483B000AF03463960FB7197F9073042
:10D3C000002B10DA4FF46D43CEF20003FA7902F02D
:10D3D0000F02A2F104013A68D2B24FEA0212D2B2AD
:10D3E0005B181A760DE04FF46143CEF2000397F913
:10D3F00007103A68D2B24FEA0212D2B25B1883F831
:10D40000002307F10C07BD4680BC704780B582B091
:10D4100000AF78607B6803F1FF326FF07F439A4280
:10D4200002D94FF001031DE04EF21003CEF20003CB
:10D430007A6802F1FF325A604FF0FF304FF00F016F
:10D44000FFF7B6FF4EF21003CEF200034FF00002DA
:10D450009A604EF21003CEF200034FF007021A60FA
:10D460004FF00003184607F10807BD4680BD00BF16
:10D4700080B500AF40F20C03C2F200031A6844F614
:10D48000D353C1F26203A3FB02134FEA931318466E
:10D49000FFF7BCFF80BD00BF80B400AF44F6580367
:10D4A000C2F200031B68002B0BD044F65803C2F2F3
:10D4B00000031B6803F1FF3244F65803C2F2000375
:10D4C0001A60BD4680BC704780B586B000AF4FF48F
:10D4D0006053C4F202034FF46052C4F20202126BB2
:10D4E00042F001021A634FF480737B604FF0010336
:10D4F000BB604FF002033B614FF00103FB6007F19B
:10D5000004034FF00000C4F202001946F5F776FA62
:10D510004FF00000C4F202004FF480714FF000029F
:10D52000F5F746FE07F11807BD4680BD80B582B00D
:10D5300000AF0346FB8049F28073C0F601031A680E
:10D5400049F28073C0F601039B88104619464FF0DC
:10D550000002F5F72DFE49F2F073C0F601031A68D8
:10D5600049F2F073C0F601039B88104619464FF04C
:10D570000002F5F71DFE49F29073C0F601031A6828
:10D5800049F29073C0F601039B88104619464FF08C
:10D590000002F5F70DFE44F65C03C2F20003FA88C0
:10D5A0001A8040F62830C2F2000044F65C01C2F254
:10D5B00000014FF001024FF00103F4F721F849F2A6
:10D5C0009073C0F601031A6849F29073C0F6010324
:10D5D0009B88104619464FF00102F5F7E9FD07F167
:10D5E0000807BD4680BD00BF80B582B000AF0346CE
:10D5F000FB8049F28073C0F601031A6849F2807318
:10D60000C0F601039B88104619464FF00102F5F75A
:10D61000CFFD49F2F073C0F601031A6849F2F073C6
:10D62000C0F601039B88104619464FF00002F5F73B
:10D63000BFFD49F29073C0F601031A6849F2907376
:10D64000C0F601039B88104619464FF00002F5F71B
:10D65000AFFD44F65C03C2F20003FA881A8040F67C
:10D660002830C2F2000044F65C01C2F200014FF023
:10D6700001024FF00103F3F7C3FF49F29073C0F6C4
:10D6800001031A6849F29073C0F601039B881046A3
:10D6900019464FF00102F5F78BFD07F10807BD466B
:10D6A00080BD00BF80B500AF49F28873C0F60103AA
:10D6B0001A6849F28873C0F601039B881046194620
:10D6C0004FF00102F5F774FD4FF00500FEF704FB83
:10D6D00049F28873C0F601031A6849F28873C0F6EC
:10D6E00001039B88104619464FF00002F5F760FDD4
:10D6F0004FF01400FEF7F0FA49F28873C0F6010308
:10D700001A6849F28873C0F601039B8810461946CF
:10D710004FF00102F5F74CFD4FF09600FEF7DCFAF2
:10D7200049F29073C0F601031A6849F29073C0F68B
:10D7300001039B88104619464FF00002F5F738FDAB
:10D740004FF0EF00FFF7F2FE4FF00300FFF74CFF42
:10D750004FF08000FFF748FF4FF00200FFF744FF53
:10D760004FF0CF00FFF7E2FE4FF00000FFF73CFF65
:10D770004FF0C100FFF738FF4FF03000FFF734FFE4
:10D780004FF0ED00FFF7D2FE4FF06400FFF72CFFE3
:10D790004FF00300FFF728FF4FF01200FFF724FFC0
:10D7A0004FF08100FFF720FF4FF0E800FFF7BEFECB
:10D7B0004FF08500FFF718FF4FF00000FFF714FF50
:10D7C0004FF07800FFF710FF4FF0CB00FFF7AEFEF1
:10D7D0004FF03900FFF708FF4FF02C00FFF704FF70
:10D7E0004FF00000FFF700FF4FF03400FFF7FCFEA2
:10D7F0004FF00200FFF7F8FE4FF0F700FFF796FE3C
:10D800004FF02000FFF7F0FE4FF0EA00FFF78EFE2A
:10D810004FF00000FFF7E8FE4FF00000FFF7E4FED6
:10D820004FF0C000FFF782FE4FF02300FFF7DCFE51
:10D830004FF0C100FFF77AFE4FF01000FFF7D4FE63
:10D840004FF0C500FFF772FE4FF03E00FFF7CCFE31
:10D850004FF02800FFF7C8FE4FF0C700FFF766FE45
:10D860004FF08600FFF7C0FE4FF03600FFF75EFE78
:10D870004FF04800FFF7B8FE4FF03A00FFF756FEB2
:10D880004FF05500FFF7B0FE4FF0B100FFF74EFE2E
:10D890004FF00000FFF7A8FE4FF01800FFF7A4FEBE
:10D8A0004FF0B600FFF742FE4FF00800FFF79CFE76
:10D8B0004FF08200FFF798FE4FF02700FFF794FE2D
:10D8C0004FF0F200FFF732FE4FF00000FFF78CFE42
:10D8D0004FF02600FFF72AFE4FF00100FFF784FE0D
:10D8E0004FF0E000FFF722FE4FF00F00FFF77CFE45
:10D8F0004FF03100FFF778FE4FF02B00FFF774FE7A
:10D900004FF00C00FFF770FE4FF00E00FFF76CFEBB
:10D910004FF00800FFF768FE4FF04E00FFF764FE7F
:10D920004FF0F100FFF760FE4FF03700FFF75CFEAD
:10D930004FF00700FFF758FE4FF01000FFF754FEBE
:10D940004FF00300FFF750FE4FF00E00FFF74CFEC4
:10D950004FF00900FFF748FE4FF00000FFF744FECC
:10D960004FF0E100FFF7E2FD4FF00000FFF73CFE53
:10D970004FF00E00FFF738FE4FF01400FFF734FEB3
:10D980004FF00300FFF730FE4FF01100FFF72CFEC1
:10D990004FF00700FFF728FE4FF03100FFF724FE9D
:10D9A0004FF0C100FFF720FE4FF04800FFF71CFECC
:10D9B0004FF00800FFF718FE4FF00F00FFF714FEBE
:10D9C0004FF00C00FFF710FE4FF03100FFF70CFE98
:10D9D0004FF03600FFF708FE4FF00F00FFF704FE90
:10D9E0004FF01100FFF7A2FD4FF07800FEF774F939
:10D9F0004FF02900FFF79AFD80BD00BF80B582B0CF
:10DA000000AFF880B9807A803B804FF02A00FFF7A2
:10DA10008DFDFB884FEA13239BB21846FFF7E4FD08
:10DA2000FB88DBB29BB21846FFF7DEFD7B884FEA2E
:10DA300013239BB21846FFF7D7FD7B88DBB29BB25E
:10DA40001846FFF7D1FD4FF02B00FFF76FFDBB88A5
:10DA50004FEA13239BB21846FFF7C6FDBB88184652
:10DA6000FFF7C2FD3B884FEA13239BB21846FFF72E
:10DA7000BBFD3B881846FFF7B7FD4FF02C00FFF7C2
:10DA800055FD07F10807BD4680BD00BF90B597B0B2
:10DA900014AF13460246FA800A46BA807B80B7F973
:10DAA0000630002B79DB40F68233C2F200031B887C
:10DAB000B7F906201BB29A426FDAB7F90430002B8F
:10DAC0006BDB40F68833C2F200031B88B7F90420F1
:10DAD0001BB29A4261DAF888B988FB8803F1010326
:10DAE0009AB2BB8803F101039BB2FFF787FF49F2AB
:10DAF0008073C0F601031A6849F28073C0F601030F
:10DB00009B88104619464FF00102F5F751FB49F288
:10DB10009073C0F601031A6849F29073C0F60103CE
:10DB20009B88104619464FF00002F5F741FB44F67A
:10DB30005C03C2F200037A881A8040F62834C2F2ED
:10DB4000000444F66003C2F20003119344F65C0340
:10DB5000C2F2000312934FF001031393694604F1DC
:10DB600010024FF04403084611461A4603F0F0FD38
:10DB700094E80F00FAF72EFF49F29073C0F6010304
:10DB80001A6849F29073C0F601039B881046194643
:10DB90004FF00102F5F70CFB00E000BF07F10C07A6
:10DBA000BD4690BD90B597B014AFF880B9807A802B
:10DBB0003B8040F68233C2F200031B88B7F906208F
:10DBC0001BB29A4280F2948040F68833C2F200037E
:10DBD0001B88B7F904201BB29A4280F28980B7F9FA
:10DBE0000420B7F90230D31803F1FF3240F688332E
:10DBF000C2F200031B881BB29A4209DB40F688334D
:10DC0000C2F200031B889AB2BB88D31A9BB27B80F6
:10DC1000F888B988FA88BC887B88E3189BB203F13E
:10DC2000FF339BB2FFF7EAFE49F28073C0F60103AF
:10DC30001A6849F28073C0F601039B8810461946A2
:10DC40004FF00102F5F7B4FA49F29073C0F6010300
:10DC50001A6849F29073C0F601039B881046194672
:10DC60004FF00002F5F7A4FA24E044F65C03C2F298
:10DC700000033A881A8040F62834C2F2000444F6C1
:10DC80006003C2F20003119344F65C03C2F2000386
:10DC900012934FF001031393694604F110024FF001
:10DCA0004403084611461A4603F052FD94E80F005B
:10DCB000FAF790FEB7F90230002B0CBF00230123C6
:10DCC000DBB27A8802F1FF327A80002BCDD149F2A3
:10DCD0009073C0F601031A6849F29073C0F601030D
:10DCE0009B88104619464FF00102F5F761FA00E0F3
:10DCF00000BF07F10C07BD4690BD00BF90B597B0BF
:10DD000014AFF880B9807A803B8040F68233C2F24B
:10DD100000031B88B7F906201BB29A4280F2948058
:10DD200040F68833C2F200031B88B7F904201BB207
:10DD30009A4280F28980B7F90620B7F90230D318E9
:10DD400003F1FF3240F68233C2F200031B881BB29C
:10DD50009A4209DB40F68233C2F200031B889AB272
:10DD6000FB88D31A9BB27B80F888B988FA887B88B5
:10DD7000D3189BB203F1FF339AB2BB88FFF73EFE84
:10DD800049F28073C0F601031A6849F28073C0F645
:10DD900001039B88104619464FF00102F5F708FA77
:10DDA00049F29073C0F601031A6849F29073C0F605
:10DDB00001039B88104619464FF00002F5F7F8F969
:10DDC00024E044F65C03C2F200033A881A8040F66D
:10DDD0002834C2F2000444F66003C2F20003119337
:10DDE00044F65C03C2F2000312934FF00103139355
:10DDF000694604F110024FF04403084611461A46E2
:10DE000003F0A6FC94E80F00FAF7E4FDB7F902303E
:10DE1000002B0CBF00230123DBB27A8802F1FF3212
:10DE20007A80002BCDD149F29073C0F601031A68B5
:10DE300049F29073C0F601039B88104619464FF0D3
:10DE40000102F5F7B5F900E000BF07F10C07BD4688
:10DE500090BD00BF90B597B014AFF880B9807A80BC
:10DE60003B8040F68233C2F200031B88B7F90620DC
:10DE70001BB29A4280F2BB8040F68833C2F20003A4
:10DE80001B88B7F904201BB29A4280F2B080B7F920
:10DE90000620B7F90230D31803F1FF3240F682337F
:10DEA000C2F200031B881BB29A4209DB40F68233A0
:10DEB000C2F200031B889AB2FB88D31A9BB27B8004
:10DEC000B7F90420B7F90030D31803F1FF3240F658
:10DED0008833C2F200031B881BB29A4209DB40F66A
:10DEE0008833C2F200031B889AB2BB88D31A9BB254
:10DEF0003B80F888B988FA887B88D3189BB203F1F5
:10DF0000FF339AB2BC883B88E3189BB203F1FF331E
:10DF10009BB2FFF773FD49F28073C0F601031A68E4
:10DF200049F28073C0F601039B88104619464FF0F2
:10DF30000102F5F73DF949F29073C0F601031A6842
:10DF400049F29073C0F601039B88104619464FF0C2
:10DF50000002F5F72DF93B88BB8033E07B88FB801E
:10DF600028E044F65C03C2F200033A8B1A8040F6C4
:10DF70002834C2F2000444F66003C2F20003119395
:10DF800044F65C03C2F2000312934FF001031393B3
:10DF9000694604F110024FF04403084611461A4640
:10DFA00003F0D6FB94E80F00FAF714FDFB8803F1A9
:10DFB000FF33FB80B7F90630002BD2DCBB8803F1BE
:10DFC000FF33BB80B7F90430002BC7DC49F29073F4
:10DFD000C0F601031A6849F29073C0F601039B88EA
:10DFE000104619464FF00102F5F7E2F800E000BFD5
:10DFF00007F10C07BD4690BD80B582B000AF134657
:10E000000246FA800A46BA807B80FA88BB88D2181A
:10E010007B88D318B3F5A07F2BD14FF03300FFF7E7
:10E0200085FAFB884FEA13239BB21846FFF7DCFA08
:10E03000FB88DBB29BB21846FFF7D6FABB884FEAE3
:10E0400013239BB21846FFF7CFFABB88DBB29BB213
:10E050001846FFF7C9FA7B884FEA13239BB218468C
:10E06000FFF7C2FA7B88DBB29BB21846FFF7BCFA17
:10E0700000E000BF07F10807BD4680BD80B584B051
:10E0800000AF0346FB714FF03600FFF74FFAFB7904
:10E0900003F00303FB60FB68032B57D801A252F87F
:10E0A00023F000BFB5E00008DBE0000801E1000854
:10E0B00027E100084FF04800FFF796FA40F6823358
:10E0C000C2F200034FF0F0021A8040F68833C2F229
:10E0D00000034FF4A0721A8038E04FF02800FFF7D9
:10E0E00083FA40F68233C2F200034FF4A0721A8022
:10E0F00040F68833C2F200034FF0F0021A8025E0A8
:10E100004FF08800FFF770FA40F68233C2F2000346
:10E110004FF0F0021A8040F68833C2F200034FF449
:10E12000A0721A8012E04FF0E800FFF75DFA40F6A7
:10E130008233C2F200034FF4A0721A8040F6883393
:10E14000C2F200034FF0F0021A8000BF07F110077F
:10E15000BD4680BD80B584B000AFF880B9807A80BC
:10E160003B80FB88FB810CE0B7F90E00B7F9041087
:10E17000B7F900203B8BFFF715FDFB8903F1010385
:10E18000FB81B7F90E20B7F90610B7F90230CB18AA
:10E190009A42E9DB07F11007BD4680BD80B584B027
:10E1A00002AF0346FB8040F68233C2F200031A88B6
:10E1B00040F68833C2F200031B8812B21BB2F98802
:10E1C00000914FF000004FF00001FFF743FE07F110
:10E1D0000807BD4680BD00BF80B58CB000AFF88099
:10E1E000B9807A803B80B7F90420B7F900309A42B1
:10E1F0000BDDBB887B843B88BB807B8C3B80FB88B2
:10E200003B847B88FB803B8C7B80B7F90020B7F98F
:10E210003C309A420BDDBB8FFB833B88BB87FB8B7B
:10E220003B803B8FBB837B883B87BB8B7B80B7F975
:10E230000420B7F900309A420BDDBB887B833B8812
:10E24000BB807B8B3B80FB883B837B88FB803B8B4D
:10E250007B80B7F90420B7F93C309A4237D1FB886C
:10E26000BB85BB8DFB85B7F90220B7F92E309A42EA
:10E2700002DA7B88FB8507E0B7F90220B7F92C307A
:10E280009A4201DD7B88BB85B7F93820B7F92E307B
:10E290009A4202DA3B8FFB8507E0B7F93820B7F9DD
:10E2A0002C309A4201DD3B8FBB85BA8DFB8DD31A92
:10E2B0009BB203F101039BB29BB2B7F92E00B7F9F1
:10E2C00004101AB2B7F84030FFF718FDD9E07A8889
:10E2D000FB88D31A9BB2FB823A88BB88D31A9BB2C5
:10E2E000BB823A8FFB88D31A9BB27B82BA8FBB88E2
:10E2F000D31A9BB23B823A8F7B88D31A9BB2FB81A5
:10E30000BA8F3B88D31A9BB2BB814FF00003FB84CA
:10E310004FF00003BB84B7F90020B7F93C309A42B4
:10E3200002D13B883B8504E03B8803F1FF339BB27D
:10E330003B85BB887B8540E0B7F92620B7F91430D0
:10E3400092FBF3F39AB2FB88D3189BB2FB85B7F923
:10E350002420B7F9103092FBF3F39AB2FB88D3185C
:10E360009BB2BB85FA8CFB8AD3189BB2FB84BA8C18
:10E370007B8AD3189BB2BB84B7F92E20B7F92C3017
:10E380009A4205DDFB8D7B81BB8DFB857B89BB853F
:10E39000BA8DFB8DD31A9BB203F101039BB29BB2E2
:10E3A000B7F92E00B7F92A101AB2B7F84030FFF7C4
:10E3B000A5FC7B8D03F101037B85B7F92A20B7F912
:10E3C00028309A42B8DDB7F92A20B7F90030D31ABD
:10E3D0009BB2FA8902FB03F39BB2FB84B7F92A20B4
:10E3E000B7F90430D31A9BB27A8A02FB03F39BB2CB
:10E3F000BB8440E0B7F92620B7F90C3092FBF3F369
:10E400009AB27B88D3189BB2FB85B7F92420B7F961
:10E41000103092FBF3F39AB2FB88D3189BB2BB8502
:10E42000FA8CFB89D3189BB2FB84BA8C7B8AD318F5
:10E430009BB2BB84B7F92E20B7F92C309A4205DD88
:10E44000FB8D3B81BB8DFB853B89BB85BA8DFB8DED
:10E45000D31A9BB203F101039BB29BB2B7F92E0012
:10E46000B7F92A101AB2B7F84030FFF747FC7B8D96
:10E4700003F101037B85B7F92A20B7F93C309A42B2
:10E48000B8DD07F13007BD4680BD00BF90B589B04B
:10E4900000AFBA600246FA810A46BA81FB80F88969
:10E4A000B989FA89FB88D3189BB203F1FF339AB27A
:10E4B000BC893B8EE3189BB203F1FF339BB2FFF79D
:10E4C0009DFA49F28073C0F601031A6849F280731D
:10E4D000C0F601039B88104619464FF00102F4F77D
:10E4E00067FE49F29073C0F601031A6849F290730F
:10E4F000C0F601039B88104619464FF00002F4F75E
:10E5000057FE4FF00003FB832CE0B7F91E304FEAB3
:10E510004303BA68D3181A88BB8E13409BB24FEAE4
:10E5200013239BB2DBB23B75B7F91E304FEA4303AE
:10E53000BA68D3181B88DAB2BB8EDBB21340DBB2E9
:10E540007B7507F1140340F62830C2F2000019462B
:10E550004FF002024FF00103F3F752F8FB8B03F187
:10E560000103FB83B7F91E20B7F90630B7F9301065
:10E5700001FB03F39A42C8DB49F29073C0F6010332
:10E580001A6849F29073C0F601039B881046194639
:10E590004FF00102F4F70CFE07F12407BD4690BDD1
:10E5A000B0B584B002AF0346FB71FB790A2B1DD1D5
:10E5B00040F68733C2F200031B784FEAC3039AB2D6
:10E5C00040F64023C2F200031B889BB2D3189BB2D3
:10E5D0009AB240F64023C2F200031A8040F6843318
:10E5E000C2F200034FF000021A807FE0FB790D2B8E
:10E5F0007CD040F68433C2F20003198840F64023F1
:10E60000C2F200031A8840F61E43C2F200031C88BF
:10E6100040F61C43C2F200031D8840F68733C2F265
:10E620000003187809B212B2FB79009501900846F0
:10E6300011461A46234600F05DF840F68733C2F2D1
:10E6400000031B781A464FEA4202D3184FEA4303ED
:10E650009AB240F68433C2F200031B889BB2D318EF
:10E660009BB29AB240F68433C2F200031A8040F69D
:10E670008633C2F200031B78002B37D040F6843378
:10E68000C2F200031B8819B240F68233C2F20003C3
:10E690001B8818B240F68733C2F200031B781A4673
:10E6A00013464FEA82029B1A4FEA4303C31899426A
:10E6B0001CDD40F68733C2F200031B784FEAC30328
:10E6C0009AB240F64023C2F200031B889BB2D318D3
:10E6D0009BB29AB240F64023C2F200031A8040F681
:10E6E0008433C2F200034FF000021A8007F10807DA
:10E6F000BD46B0BD90B587B002AFF880B980FA7062
:10E700003B804FF00003FB73BDE097F90F30052B02
:10E7100003D14FF00003BB730FE0FA7813464FEAC2
:10E7200083039B181A4697F90F30D21849F638130D
:10E73000C0F60103D3181B78BB734FF000037B7343
:10E7400098E0BB7B03F00103DBB2002B43D097F8CA
:10E750002430012B16D197F90F309AB2FB88D318C9
:10E760009BB29AB297F90D3099B2BB88CB189BB285
:10E770009BB211B21AB23B88084611461A46FFF7FF
:10E7800085F96FE097F90F309BB297F8242092B289
:10E7900002FB03F39AB2FB88D3189BB298B297F9A5
:10E7A0000D309BB297F8242092B202FB03F39AB289
:10E7B000BB88D3189BB299B297F824309AB297F8D5
:10E7C00024309BB200B209B212B21BB23C88009452
:10E7D000FFF7C0FC46E03A8C3B889A4242D097F85B
:10E7E0002430012B16D197F90F309AB2FB88D31839
:10E7F0009BB29AB297F90D3099B2BB88CB189BB2F5
:10E800009BB211B21AB23B8C084611461A46FFF76A
:10E810003DF927E097F90F309BB297F8242092B288
:10E8200002FB03F39AB2FB88D3189BB298B297F914
:10E830000D309BB297F8242092B202FB03F39AB2F8
:10E84000BB88D3189BB299B297F824309AB297F844
:10E8500024309BB200B209B212B21BB23C8C0094BD
:10E86000FFF778FCBB7B4FEA5303BB737B7B03F161
:10E8700001037B7397F90D30072B7FF762AFFB7BAA
:10E8800003F10103FB7397F90F30052B7FF73DAFC1
:10E8900007F11407BD4690BD80B483B000AF0246B7
:10E8A0000B46FA80BB8040F68433C2F20003FA883C
:10E8B0001A8040F64023C2F20003BA881A8007F19A
:10E8C0000C07BD4680BC704780B483B000AF0346E0
:10E8D000FB71FB79002B01D0FA7901E04FF00102C6
:10E8E00040F68733C2F200031A7007F10C07BD46E9
:10E8F00080BC704780B483B000AF02460B46FA80FC
:10E90000BB8040F61E43C2F20003FA881A8040F62C
:10E910001C43C2F20003BA881A8007F10C07BD46F7
:10E9200080BC704780B483B000AF0346FB7140F6F3
:10E930008633C2F20003FA791A7007F10C07BD465C
:10E9400080BC704780B485B000AF786079807A7001
:10E950003B704FF00003FB737B687A881A807A68FB
:10E960004AF23463C0F6010353607B687A789A7088
:10E970007B683A78DA707B681B88B3F5807F2ED08D
:10E98000B3F5807F04DC102B47D0402B36D053E00A
:10E99000B3F5806F14D0B3F5805F4DD17B684FF035
:10E9A00001029A817B684FF00102DA817A6849F6A8
:10E9B0003463C0F6010393607B68294A1A613FE023
:10E9C0007B684FF004029A817B684FF00402DA8181
:10E9D0007B681F4A9A607B68224A1A6130E07B6834
:10E9E0004FF010029A817B684FF01002DA817B6849
:10E9F000184A9A607B681C4A1A6121E07B684FF0D4
:10EA000040029A817B684FF04002DA817B68124AAB
:10EA10009A607B68154A1A6112E07B684FF4807235
:10EA20009A817B684FF48072DA817B680B4A9A6026
:10EA30007B680F4A1A6103E04FF0FF03FB7300BFCE
:10EA4000FB7B5BB2184607F11407BD4680BC7047DC
:10EA50003A9E0108529E0108B29E010832A00108A8
:10EA6000000080390000803A0000803B0000803CBC
:10EA70000000803D80B4C1B000AFF8607A600A4603
:10EA80007A813B817B89C7F8F430D7F8F430C7F836
:10EA9000E430D7F8F4304FEA9303C7F8F4304FF07E
:10EAA0000003C7F8F8304FF00003C7F8FC30D7F880
:10EAB000F430C7F8F030D7F8F820D7F8F430D3188E
:10EAC000C7F8E030D7F8E020D7F8F430D318C7F80B
:10EAD000DC30D7F8DC20D7F8F430D318C7F8D830BA
:10EAE000D7F8F8304FEAC303FA68D3181B68C7F8A1
:10EAF000D430D7F8F8304FEAC30303F10403FA68BF
:10EB0000D3181B68C7F8D030D7F8E0304FEAC303FA
:10EB1000FA68D3181B68C7F8CC30D7F8E0304FEA52
:10EB2000C30303F10403FA68D3181B68C7F8C8309D
:10EB3000D7F8DC304FEAC303FA68D3181B68C7F86C
:10EB4000C430D7F8DC304FEAC30303F10403FA689A
:10EB5000D3181B68C7F8C030D7F8D8304FEAC303C2
:10EB6000FA68D3181B68C7F8BC30D7F8D8304FEA1A
:10EB7000C30303F10403FA68D3181B68C7F8B8305D
:10EB800097ED357AD7ED317A77EE277AC7ED2D7A82
:10EB900097ED337AD7ED2F7A77EE277AC7ED2C7A77
:10EBA00097ED347AD7ED307A77EE277AC7ED2B7A66
:10EBB00097ED327AD7ED2E7A77EE277AC7ED2A7A5B
:10EBC000D7F8FC20D7F8FC30D318C7F8A430D7F812
:10EBD000A4304FEAC3037A68D3181B68C7F8A03083
:10EBE000D7F8A4304FEAC30303F104037A68D318BB
:10EBF0001B68C7F89C3097ED357AD7ED317A77EE00
:10EC0000677AC7ED267A97ED337AD7ED2F7A77EECC
:10EC1000677AC7ED257A97ED347AD7ED307A77EEBB
:10EC2000677AC7ED247A97ED327AD7ED2E7A77EEB0
:10EC3000677AC7ED237AD7F8F8304FEAC303FA684A
:10EC4000D31897ED2D7AD7ED2C7A77EE277AC3ED8E
:10EC5000007AD7F8F8304FEAC30303F10403FA68E7
:10EC6000D31897ED2B7AD7ED2A7A77EE277AC3ED72
:10EC7000007A97ED267AD7ED237A77EE277AC7EDDB
:10EC8000227A97ED247AD7ED257A77EE677AC7ED69
:10EC9000217A97ED2D7AD7ED2C7A77EE677AC7ED4A
:10ECA000207A97ED2B7AD7ED2A7A77EE677AC7ED3F
:10ECB0001F7A97ED267AD7ED237A77EE677AC7ED3C
:10ECC0001E7A97ED257AD7ED247A77EE277AC7ED6D
:10ECD0001D7AD7F8FC304FEAC3037A68D3181B6853
:10ECE0003B67D7F8FC304FEAC30303F104037A68AB
:10ECF000D3181B68FB66D7F8A420D7F8FC30D318CC
:10ED0000BB66BB6E4FEAC3037A68D3181B687B6689
:10ED1000BB6E4FEAC30303F104037A68D3181B6880
:10ED20003B6697ED227AD7ED1C7A67EE277AC7ED1E
:10ED3000177A97ED217AD7ED1C7A67EE277AC7ED1F
:10ED4000167A97ED207AD7ED287A67EE277AC7ED05
:10ED5000157A97ED1F7AD7ED287A67EE277AC7EDF7
:10ED6000147A97ED1E7AD7ED197A67EE277AC7EDF8
:10ED7000137A97ED1D7AD7ED197A67EE277AC7EDEA
:10ED8000127A97ED217AD7ED1B7A67EE277AC7EDD5
:10ED9000117A97ED227AD7ED1B7A67EE277AC7EDC5
:10EDA000107A97ED1F7AD7ED277A67EE277AC7EDAD
:10EDB0000F7A97ED207AD7ED277A67EE277AC7ED9D
:10EDC0000E7A97ED1D7AD7ED187A67EE277AC7EDA0
:10EDD0000D7A97ED1E7AD7ED187A67EE277AC7ED90
:10EDE0000C7A97ED177AD7ED117A77EE277AC7ED7F
:10EDF000177A97ED167AD7ED107A77EE677AC7ED26
:10EE0000167A97ED157AD7ED0F7A77EE277AC7ED58
:10EE1000157A97ED147AD7ED0E7A77EE677AC7ED0B
:10EE2000147A97ED137AD7ED0D7A77EE277AC7ED3E
:10EE3000137A97ED127AD7ED0C7A77EE677AC7EDF1
:10EE4000127AD7F8E0304FEAC303FA68D3187A6D24
:10EE50001A60D7F8E0304FEAC30303F10403FA68FD
:10EE6000D3183A6D1A60D7F8DC304FEAC303FA685A
:10EE7000D318FA6D1A60D7F8DC304FEAC30303F1F8
:10EE80000403FA68D318BA6D1A60D7F8D8304FEA7D
:10EE9000C303FA68D318FA6C1A60D7F8D8304FEA6F
:10EEA000C30303F10403FA68D318BA6C1A603B89F0
:10EEB000D7F8FC20D318C7F8FC30D7F8F83003F1A6
:10EEC0000103C7F8F830D7F8F03003F1FF33C7F883
:10EED000F030D7F8F030002B7FF4EDAD3B894FEAEE
:10EEE00083033B817B894FEA93039BB2C7F8EC30E5
:10EEF0003DE2D7F8F430C7F8E430D7F8F4304FEA01
:10EF00009303C7F8F4304FF00003C7F8FC304FF01C
:10EF10000003C7F8F030D7F8FC20D7F8FC30D3183E
:10EF2000C7F8A430D7F8A420D7F8FC30D318BB66B4
:10EF3000D7F8FC304FEAC3037A68D3181B683B67E5
:10EF4000D7F8FC304FEAC30303F104037A68D318FF
:10EF50001B68FB66D7F8A4304FEAC3037A68D3185E
:10EF60001B68C7F8A030D7F8A4304FEAC30303F1F9
:10EF700004037A68D3181B68C7F89C30BB6E4FEA4D
:10EF8000C3037A68D3181B687B66BB6E4FEAC30362
:10EF900003F104037A68D3181B683B663B89D7F8F2
:10EFA000FC20D318C7F8FC30D7F8F030C7F8F83099
:10EFB000D7F8F820D7F8F430D318C7F8E030D7F8EE
:10EFC000E020D7F8F430D318C7F8DC30D7F8DC20CD
:10EFD000D7F8F430D318C7F8D830D7F8F8304FEA5C
:10EFE000C303FA68D3181B68C7F8D430D7F8F830D1
:10EFF0004FEAC30303F10403FA68D3181B68C7F888
:10F00000D030D7F8E0304FEAC303FA68D3181B6852
:10F01000C7F8CC30D7F8E0304FEAC30303F104035C
:10F02000FA68D3181B68C7F8C830D7F8DC304FEA45
:10F03000C303FA68D3181B68C7F8C430D7F8DC30AC
:10F040004FEAC30303F10403FA68D3181B68C7F837
:10F05000C030D7F8D8304FEAC303FA68D3181B681A
:10F06000C7F8BC30D7F8D8304FEAC30303F1040324
:10F07000FA68D3181B68C7F8B83097ED357AD7ED22
:10F08000317A77EE677AC7ED267A97ED337AD7ED46
:10F090002F7A77EE677AC7ED257A97ED347AD7ED38
:10F0A000307A77EE677AC7ED247A97ED327AD7ED2A
:10F0B0002E7A77EE677AC7ED237A97ED357AD7ED1A
:10F0C000317A77EE277AC7ED2D7A97ED337AD7ED3F
:10F0D0002F7A77EE277AC7ED2C7A97ED347AD7ED31
:10F0E000307A77EE277AC7ED2B7A97ED327AD7ED23
:10F0F0002E7A77EE277AC7ED2A7A97ED267AD7ED22
:10F10000237A77EE277AC7ED227A97ED247AD7ED26
:10F11000257A77EE677AC7ED217A97ED2D7AD7EDCC
:10F120002C7A77EE677AC7ED207A97ED2B7AD7EDB8
:10F130002A7A77EE677AC7ED1F7A97ED267AD7EDB0
:10F14000237A77EE677AC7ED1E7A97ED257AD7EDA9
:10F15000247A77EE277AC7ED1D7AD7F8F8304FEA90
:10F16000C303FA68D31897ED2D7AD7ED2C7A77EE92
:10F17000277AC3ED007AD7F8F8304FEAC30303F1DA
:10F180000403FA68D31897ED2B7AD7ED2A7A77EE35
:10F19000277AC3ED007A97ED227AD7ED1C7A67EED5
:10F1A000277AC7ED177A97ED217AD7ED1C7A67EEAB
:10F1B000277AC7ED167A97ED207AD7ED287A67EE91
:10F1C000277AC7ED157A97ED1F7AD7ED287A67EE83
:10F1D000277AC7ED147A97ED1E7AD7ED197A67EE84
:10F1E000277AC7ED137A97ED1D7AD7ED197A67EE76
:10F1F000277AC7ED127A97ED217AD7ED1B7A67EE61
:10F20000277AC7ED117A97ED227AD7ED1B7A67EE50
:10F21000277AC7ED107A97ED1F7AD7ED277A67EE38
:10F22000277AC7ED0F7A97ED207AD7ED277A67EE28
:10F23000277AC7ED0E7A97ED1D7AD7ED187A67EE2B
:10F24000277AC7ED0D7A97ED1E7AD7ED187A67EE1B
:10F25000277AC7ED0C7A97ED177AD7ED117A77EE0A
:10F26000277AC7ED177A97ED167AD7ED107A77EEF1
:10F27000677AC7ED167A97ED157AD7ED0F7A77EEA4
:10F28000277AC7ED157A97ED147AD7ED0E7A77EED7
:10F29000677AC7ED147A97ED137AD7ED0D7A77EE8A
:10F2A000277AC7ED137A97ED127AD7ED0C7A77EEBD
:10F2B000677AC7ED127AD7F8E0304FEAC303FA68ED
:10F2C000D3187A6D1A60D7F8E0304FEAC30303F120
:10F2D0000403FA68D3183A6D1A60D7F8DC304FEAA5
:10F2E000C303FA68D318FA6D1A60D7F8DC304FEA16
:10F2F000C30303F10403FA68D318BA6D1A60D7F890
:10F30000D8304FEAC303FA68D318FA6C1A60D7F8FA
:10F31000D8304FEAC30303F10403FA68D318BA6C78
:10F320001A60D7F8F820D7F8E430D318C7F8F830C7
:10F330007A89D7F8F8309A423FF63AAED7F8F030EB
:10F3400003F10103C7F8F030D7F8F43003F1FF32CE
:10F35000D7F8F0309A42BFF4DEAD3B894FEA830321
:10F360003B81D7F8EC304FEA9303C7F8EC30D7F87D
:10F37000EC30042B3FF6BDAD7B894FEA93039BB283
:10F38000C7F8F030FB68C7F8E830D7F8E8301B68FA
:10F39000C7F8D430D7F8E8305B68C7F8D030D7F872
:10F3A000E8309B68C7F8CC30D7F8E830DB68C7F89E
:10F3B000C830D7F8E8301B69C7F8C430D7F8E83050
:10F3C0005B69C7F8C030D7F8E8309B69C7F8BC3034
:10F3D000D7F8E830DB69C7F8B83097ED357AD7ED64
:10F3E000317A77EE277AC7ED2D7A97ED357AD7ED1A
:10F3F000317A77EE677AC7ED267A97ED347AD7EDD2
:10F40000307A77EE277AC7ED2B7A97ED347AD7EDFD
:10F41000307A77EE677AC7ED247A97ED337AD7EDB5
:10F420002F7A77EE277AC7ED2C7A97ED327AD7EDDF
:10F430002E7A77EE277AC7ED2A7A97ED337AD7EDD1
:10F440002F7A77EE677AC7ED257A97ED327AD7ED86
:10F450002E7A77EE677AC7ED237A97ED2D7AD7ED7E
:10F460002C7A77EE277AC7ED0B7A97ED2B7AD7EDCA
:10F470002A7A77EE277AC7ED0A7A97ED2D7AD7EDBB
:10F480002C7A77EE677AC7ED097A97ED2B7AD7ED6C
:10F490002A7A77EE677AC7ED087A97ED267AD7ED64
:10F4A000237A77EE277AC7ED077A97ED247AD7ED9E
:10F4B000257A77EE677AC7ED067A97ED267AD7ED4B
:10F4C000237A77EE677AC7ED057A97ED257AD7ED3F
:10F4D000247A77EE277AC7ED047AD7F8E830FA6A0B
:10F4E0001A60D7F8E83003F10403BA6A1A60D7F853
:10F4F000E83003F108037A6A1A60D7F8E83003F1BC
:10F500000C033A6A1A60D7F8E83003F11003FA697D
:10F510001A60D7F8E83003F11403BA691A60D7F813
:10F52000E83003F118037A691A60D7F8E83003F17C
:10F530001C033A691A60D7F8E83003F12003C7F8D2
:10F54000E830D7F8F03003F1FF33C7F8F030D7F8E0
:10F55000F030002B7FF419AF07F58277BD4680BCF1
:10F56000704700BF80B4C3B000AFF86007F104007B
:10F5700002601A463B4683ED000A0B467B8107F189
:10F5800008031A807B89C7F8FC30D7F8FC30C7F82D
:10F59000EC30D7F8FC304FEA9303C7F8FC304FF05B
:10F5A0000003C7F800314FF00003C7F80431D7F863
:10F5B000FC30C7F8F830D7F80021D7F8FC30D31862
:10F5C000C7F8E830D7F8E820D7F8FC30D318C7F8E8
:10F5D000E430D7F8E420D7F8FC30D318C7F8E0308F
:10F5E000D7F800314FEAC303FA68D3181B68C7F88D
:10F5F000DC30D7F800314FEAC30303F10403FA68A3
:10F60000D3181B68C7F8D830D7F8E4304FEAC303E3
:10F61000FA68D3181B68C7F8D430D7F8E4304FEA3B
:10F62000C30303F10403FA68D3181B68C7F8D0308A
:10F63000D7F8E8304FEAC303FA68D3181B68C7F855
:10F64000CC30D7F8E8304FEAC30303F10403FA687B
:10F65000D3181B68C7F8C830D7F8E0304FEAC303A7
:10F66000FA68D3181B68C7F8C430D7F8E0304FEAFF
:10F67000C30303F10403FA68D3181B68C7F8C0304A
:10F6800097ED377AD7ED357A77EE277AC7ED2F7A6F
:10F6900097ED337AD7ED317A77EE277AC7ED2E7A68
:10F6A00097ED367AD7ED347A77EE277AC7ED2D7A53
:10F6B00097ED327AD7ED307A77EE277AC7ED2C7A4C
:10F6C000D7F80421D7F80431D318C7F8AC30D7F8ED
:10F6D000AC304FEAC30307F104021268D3181B6869
:10F6E000C7F8A830D7F8AC304FEAC30303F10403DE
:10F6F00007F104021268D3181B68C7F8A43097ED0D
:10F70000377AD7ED357A77EE677AC7ED287A97EDB5
:10F71000337AD7ED317A77EE677AC7ED277A97EDAE
:10F72000367AD7ED347A77EE677AC7ED267A97ED99
:10F73000327AD7ED307A77EE677AC7ED257AD7F847
:10F7400000314FEAC303FA68D31897ED2F7AD7ED4B
:10F750002E7A77EE277AC3ED007AD7F800314FEA98
:10F76000C30303F10403FA68D31897ED2D7AD7ED9C
:10F770002C7A77EE277AC3ED007A97ED287AD7EDC9
:10F78000257A77EE677AC7ED247A97ED267AD7ED5A
:10F79000277A77EE277AC7ED237A97ED2F7AD7ED80
:10F7A0002E7A77EE677AC7ED227A97ED2D7AD7ED2C
:10F7B0002C7A77EE677AC7ED217A97ED287AD7ED24
:10F7C000257A77EE277AC7ED207A97ED267AD7ED5E
:10F7D000277A77EE677AC7ED1F7AD7F804314FEAB8
:10F7E000C30307F104021268D3181B68BB67D7F87C
:10F7F00004314FEAC30303F1040307F10402126862
:10F80000D3181B687B67D7F8AC20D7F80431D3181E
:10F810003B673B6F4FEAC30307F104021268D3183A
:10F820001B68FB663B6F4FEAC30303F1040307F158
:10F8300004021268D3181B68BB6697ED247AD7EDD3
:10F840001E7A67EE277AC7ED197A97ED237AD7EDFE
:10F850001E7A67EE277AC7ED187A97ED227AD7EDF0
:10F860002A7A67EE277AC7ED177A97ED217AD7EDD6
:10F870002A7A67EE277AC7ED167A97ED207AD7EDC8
:10F880001B7A67EE277AC7ED157A97ED1F7AD7EDC9
:10F890001B7A67EE277AC7ED147A97ED237AD7EDB6
:10F8A0001D7A67EE277AC7ED137A97ED247AD7EDA4
:10F8B0001D7A67EE277AC7ED127A97ED217AD7ED98
:10F8C000297A67EE277AC7ED117A97ED227AD7ED7C
:10F8D000297A67EE277AC7ED107A97ED1F7AD7ED70
:10F8E0001A7A67EE277AC7ED0F7A97ED207AD7ED6F
:10F8F0001A7A67EE277AC7ED0E7A97ED197AD7ED67
:10F90000137A77EE677AC7ED197A97ED187AD7ED03
:10F91000127A77EE277AC7ED187A97ED177AD7ED36
:10F92000117A77EE677AC7ED177A97ED167AD7EDE9
:10F93000107A77EE277AC7ED167A97ED157AD7ED1C
:10F940000F7A77EE677AC7ED157A97ED147AD7EDCF
:10F950000E7A77EE277AC7ED147AD7F8E8304FEAB7
:10F96000C303FA68D318FA6D1A60D7F8E8304FEA83
:10F97000C30303F10403FA68D318BA6D1A60D7F809
:10F98000E4304FEAC303FA68D3187A6E1A60D7F8E6
:10F99000E4304FEAC30303F10403FA68D3183A6E64
:10F9A0001A60D7F8E0304FEAC303FA68D3187A6DCB
:10F9B0001A60D7F8E0304FEAC30303F10403FA6892
:10F9C000D3183A6D1A6007F108031B88D7F8042191
:10F9D000D318C7F80431D7F8003103F10103C7F891
:10F9E0000031D7F8F83003F1FF33C7F8F830D7F813
:10F9F000F830002B7FF4DFAD07F1080307F10802B0
:10FA000012884FEA82021A807B894FEA93039BB2E5
:10FA1000C7F8F4304FE2D7F8FC30C7F8EC30D7F82D
:10FA2000FC304FEA9303C7F8FC304FF00003C7F8EF
:10FA300004314FF00003C7F8F830D7F80421D7F8A5
:10FA40000431D318C7F8AC30D7F8AC20D7F804315C
:10FA5000D3183B67D7F804314FEAC30307F1040218
:10FA60001268D3181B68BB67D7F804314FEAC30389
:10FA700003F1040307F104021268D3181B687B67C3
:10FA8000D7F8AC304FEAC30307F104021268D31869
:10FA90001B68C7F8A830D7F8AC304FEAC30303F1AE
:10FAA000040307F104021268D3181B68C7F8A430D6
:10FAB0003B6F4FEAC30307F104021268D3181B68B7
:10FAC000FB663B6F4FEAC30303F1040307F1040233
:10FAD0001268D3181B68BB6607F108031B88D7F8A8
:10FAE0000421D318C7F80431D7F8F830C7F800312B
:10FAF000D7F80021D7F8FC30D318C7F8E830D7F88A
:10FB0000E820D7F8FC30D318C7F8E430D7F8E42061
:10FB1000D7F8FC30D318C7F8E030D7F800314FEAF7
:10FB2000C303FA68D3181B68C7F8DC30D7F8003174
:10FB30004FEAC30303F10403FA68D3181B68C7F83C
:10FB4000D830D7F8E8304FEAC303FA68D3181B68F7
:10FB5000C7F8CC30D7F8E8304FEAC30303F1040309
:10FB6000FA68D3181B68C7F8C830D7F8E4304FEAF2
:10FB7000C303FA68D3181B68C7F8D430D7F8E43049
:10FB80004FEAC30303F10403FA68D3181B68C7F8EC
:10FB9000D030D7F8E0304FEAC303FA68D3181B68B7
:10FBA000C7F8C430D7F8E0304FEAC30303F10403C9
:10FBB000FA68D3181B68C7F8C03097ED377AD7EDCD
:10FBC000357A77EE677AC7ED287A97ED337AD7EDF5
:10FBD000317A77EE677AC7ED277A97ED367AD7EDE7
:10FBE000347A77EE677AC7ED267A97ED327AD7EDD9
:10FBF000307A77EE677AC7ED257A97ED377AD7EDC9
:10FC0000357A77EE277AC7ED2F7A97ED337AD7EDED
:10FC1000317A77EE277AC7ED2E7A97ED367AD7EDDF
:10FC2000347A77EE277AC7ED2D7A97ED327AD7EDD1
:10FC3000307A77EE277AC7ED2C7A97ED287AD7EDD0
:10FC4000257A77EE677AC7ED247A97ED267AD7ED95
:10FC5000277A77EE277AC7ED237A97ED2F7AD7EDBB
:10FC60002E7A77EE677AC7ED227A97ED2D7AD7ED67
:10FC70002C7A77EE677AC7ED217A97ED287AD7ED5F
:10FC8000257A77EE277AC7ED207A97ED267AD7ED99
:10FC9000277A77EE677AC7ED1F7AD7F800314FEAF7
:10FCA000C303FA68D31897ED2F7AD7ED2E7A77EE43
:10FCB000277AC3ED007AD7F800314FEAC30303F186
:10FCC0000403FA68D31897ED2D7AD7ED2C7A77EEE6
:10FCD000277AC3ED007A97ED247AD7ED1E7A67EE86
:10FCE000277AC7ED197A97ED237AD7ED1E7A67EE5A
:10FCF000277AC7ED187A97ED227AD7ED2A7A67EE40
:10FD0000277AC7ED177A97ED217AD7ED2A7A67EE31
:10FD1000277AC7ED167A97ED207AD7ED1B7A67EE32
:10FD2000277AC7ED157A97ED1F7AD7ED1B7A67EE24
:10FD3000277AC7ED147A97ED237AD7ED1D7A67EE0F
:10FD4000277AC7ED137A97ED247AD7ED1D7A67EEFF
:10FD5000277AC7ED127A97ED217AD7ED297A67EEE7
:10FD6000277AC7ED117A97ED227AD7ED297A67EED7
:10FD7000277AC7ED107A97ED1F7AD7ED1A7A67EEDA
:10FD8000277AC7ED0F7A97ED207AD7ED1A7A67EECA
:10FD9000277AC7ED0E7A97ED197AD7ED137A77EEB9
:10FDA000677AC7ED197A97ED187AD7ED127A77EE60
:10FDB000277AC7ED187A97ED177AD7ED117A77EE93
:10FDC000677AC7ED177A97ED167AD7ED107A77EE46
:10FDD000277AC7ED167A97ED157AD7ED0F7A77EE79
:10FDE000677AC7ED157A97ED147AD7ED0E7A77EE2C
:10FDF000277AC7ED147AD7F8E8304FEAC303FA68D8
:10FE0000D318FA6D1A60D7F8E8304FEAC30303F14C
:10FE10000403FA68D318BA6D1A60D7F8E4304FEAD1
:10FE2000C303FA68D3187A6E1A60D7F8E4304FEA41
:10FE3000C30303F10403FA68D3183A6E1A60D7F8C3
:10FE4000E0304FEAC303FA68D3187A6D1A60D7F826
:10FE5000E0304FEAC30303F10403FA68D3183A6DA4
:10FE60001A60D7F80021D7F8EC30D318C7F8003162
:10FE70007A89D7F800319A423FF63AAED7F8F8308F
:10FE800003F10103C7F8F830D7F8FC3003F1FF3273
:10FE9000D7F8F8309A42BFF4D0AD07F1080307F164
:10FEA000080212884FEA82021A80D7F8F4304FEA2B
:10FEB0009303C7F8F430D7F8F430042B3FF6ABAD1A
:10FEC0007B894FEA93039BB2C7F8F830FB68C7F809
:10FED000F030D7F8F0301B68C7F8DC30D7F8F030D6
:10FEE0005B68C7F8D830D7F8F0309B68C7F8CC30DB
:10FEF000D7F8F030DB68C7F8C830D7F8F0301B69A6
:10FF0000C7F8D430D7F8F0305B69C7F8D030D7F8ED
:10FF1000F0309B69C7F8C430D7F8F030DB69C7F818
:10FF2000C03097ED377AD7ED357A77EE277AC7ED7F
:10FF30002F7A97ED377AD7ED357A77EE677AC7ED76
:10FF4000287A97ED367AD7ED347A77EE277AC7EDAF
:10FF50002D7A97ED367AD7ED347A77EE677AC7ED5A
:10FF6000267A97ED337AD7ED317A77EE277AC7ED97
:10FF70002E7A97ED327AD7ED307A77EE277AC7ED81
:10FF80002C7A97ED337AD7ED317A77EE677AC7ED31
:10FF9000277A97ED327AD7ED307A77EE677AC7ED28
:10FFA000257A97ED2F7AD7ED2E7A77EE277AC7ED5F
:10FFB0000D7A97ED2D7AD7ED2C7A77EE277AC7ED6B
:10FFC0000C7A97ED2F7AD7ED2E7A77EE677AC7ED18
:10FFD0000B7A97ED2D7AD7ED2C7A77EE677AC7ED0D
:10FFE0000A7A97ED287AD7ED257A77EE677AC7ED0A
:10FFF000097A97ED267AD7ED277A77EE277AC7ED3B
:020000040801F1
:10000000087A97ED287AD7ED257A77EE277AC7ED2B
:10001000077A97ED267AD7ED277A77EE677AC7EDDC
:10002000067A3B4697ED0D7AD3ED007A67EE277A94
:10003000C7ED137A3B4697ED0C7AD3ED007A67EE65
:10004000277AC7ED127A3B4697ED0B7AD3ED007A0B
:1000500067EE277AC7ED117A3B4697ED0A7AD3ED22
:10006000007A67EE277AC7ED107A3B4697ED097A5A
:10007000D3ED007A67EE277AC7ED0F7A3B4697ED0E
:10008000087AD3ED007A67EE277AC7ED0E7A3B4601
:1000900097ED077AD3ED007A67EE277AC7ED057AF8
:1000A0003B4697ED067AD3ED007A67EE277AC7EDE7
:1000B000047AD7F8F030FA6C1A60D7F8F03003F110
:1000C0000403BA6C1A60D7F8F03003F108037A6CB5
:1000D0001A60D7F8F03003F10C033A6C1A60D7F8C5
:1000E000F03003F11003FA6B1A60D7F8F03003F127
:1000F0001403BA6B1A60D7F8F03003F118037A6969
:100100001A60D7F8F03003F11C033A691A60D7F887
:10011000F03003F12003C7F8F030D7F8F83003F1DE
:10012000FF33C7F8F830D7F8F830002B7FF4D1AEA2
:1001300007F58677BD4680BC704700BF80B582B0AA
:1001400000AF786039607B689B78012B0ED17B68AB
:1001500019887B685A687B689B897868D0ED047A37
:100160003868B0EE670AFFF7FDF908E07B68198888
:100170007B685A687B689B893868FEF77BFC7B68E4
:10018000DB78012B08D17B6819887B68DA897B686A
:100190009B68386800F004F807F10807BD4680BD89
:1001A00080B489B000AFF8607B600B467B8113465A
:1001B0003B814FF00003BB837B894FEA53037B8372
:1001C0007B894FEA53039BB203F101033B834FF05A
:1001D0000003FB83E5E0FA8BBB8B9A4280F08880BA
:1001E000FB8B4FEAC303FA68D3181B687B61FB8B58
:1001F0004FEAC303FA68D318BA8B4FEAC202F96810
:100200008A1812681A60BB8B4FEAC303FA68D318C6
:100210007A691A60FB8B4FEAC30303F10403FA689F
:10022000D3181B687B61FB8B4FEAC30303F1040304
:10023000FA68D318BA8B4FEAC20202F10402F968D5
:100240008A1812681A60BB8B4FEAC30303F10403D8
:10025000FA68D3187A691A60FA8B3B8BD3184FEA85
:10026000C303FA68D3181B687B61FA8B3B8BD318E6
:100270004FEAC303FA68D318B98B3A8B8A184FEA4E
:10028000C202F9688A1812681A60BA8B3B8BD318BD
:100290004FEAC303FA68D3187A691A60FA8B3B8B6A
:1002A000D3184FEAC30303F10403FA68D3181B6899
:1002B0007B61FA8B3B8BD3184FEAC30303F1040332
:1002C000FA68D318B98B3A8B8A184FEAC20202F146
:1002D0000402F9688A1812681A60BA8B3B8BD3182B
:1002E0004FEAC30303F10403FA68D3187A691A606A
:1002F000FB8B03F101034FEAC303FA68D3181B68B1
:100300007B61FB8B03F101034FEAC303FA68D31847
:10031000B98B7A8B8A184FEAC202F9688A18126878
:100320001A60BA8B7B8BD3184FEAC303FA68D318D1
:100330007A691A60FB8B03F101034FEAC30303F1EF
:100340000403FA68D3181B687B61FB8B03F101037C
:100350004FEAC30303F10403FA68D318B98B7A8B0D
:100360008A184FEAC20202F10402F9688A18126878
:100370001A60BA8B7B8BD3184FEAC30303F10403D3
:10038000FA68D3187A691A607B681B88BB833B893B
:100390004FEA43037A68D3187B60FB8B03F10203B7
:1003A000FB83FA8B7B8BA3F102039A427FF613AF98
:1003B00007F12407BD4680BC704700BF80B582B0FE
:1003C00000AF87ED010A3860D7ED017AF5EEC07A0B
:1003D000F1EE10FAD4BF00230123DBB2002B0BD0C7
:1003E00097ED010A00F0F8F8F0EE407A3B68C3EDB3
:1003F000007A4FF0000304E03B68054A1A604FF0B2
:10040000FF035BB2184607F10807BD4680BD00BF79
:100410000000000080B588B000AFF860B9607A6075
:100420007B684FEA9303FB619BE0FB681B68BB6141
:10043000FB6803F10403FB60FB681B687B61FB68DE
:1004400003F10403FB6097ED067AD7ED067A27EEF9
:10045000277AD7ED056AD7ED057A66EEA77A77EEAB
:10046000277ABB68BA6802F10402BA60B0EE670A84
:100470001846FFF7A3FFFB681B68BB61FB6803F12D
:100480000403FB60FB681B687B61FB6803F10403EA
:10049000FB6097ED067AD7ED067A27EE277AD7ED3F
:1004A000056AD7ED057A66EEA77A77EE277ABB68FC
:1004B000BA6802F10402BA60B0EE670A1846FFF7A4
:1004C0007DFFFB681B68BB61FB6803F10403FB60F5
:1004D000FB681B687B61FB6803F10403FB6097ED1D
:1004E000067AD7ED067A27EE277AD7ED056AD7ED9B
:1004F000057A66EEA77A77EE277ABB68BA6802F1CA
:100500000402BA60B0EE670A1846FFF757FFFB68AF
:100510001B68BB61FB6803F10403FB60FB681B689D
:100520007B61FB6803F10403FB6097ED067AD7ED6E
:10053000067A27EE277AD7ED056AD7ED057A66EEBB
:10054000A77A77EE277ABB68BA6802F10402BA602C
:10055000B0EE670A1846FFF731FFFB6903F1FF337E
:10056000FB61FB69002B7FF460AF7B6803F0030342
:10057000FB6129E0FB681B68BB61FB6803F10403B6
:10058000FB60FB681B687B61FB6803F10403FB6095
:1005900097ED067AD7ED067A27EE277AD7ED056A2A
:1005A000D7ED057A66EEA77A77EE277ABB68BA6848
:1005B00002F10402BA60B0EE670A1846FFF7FEFEC9
:1005C000FB6903F1FF33FB61FB69002BD2D107F11B
:1005D0002007BD4680BD00BF10B52DED028B294C14
:1005E0008AB0B0EE408A00F051F894F9003001333F
:1005F000F0EE408A2FD0B0EE480A00F0CFF850B3AA
:10060000B5EEC08AF1EE10FA25D5012300931E4BFA
:1006100018EE100A01930023089300F051FA247891
:10062000CDE90401CDE90201DCB100200021024640
:100630000B4600F0C3FB022CCDE9060117D101F0F7
:1006400081F821230360089BBBB9DDE9060100F0B6
:100650004DFD08EE900AB0EE680A0AB0BDEC028BC0
:1006600010BD0022002343EC172B8DED067B68465E
:1006700000F092F80028E6D1E1E701F063F8089B6A
:100680000360E2E7580000203426020810EE103A1A
:1006900023F00042B2F1FF4F70B42FD262B3002BAF
:1006A0003ADBD915B2F5000F2BD323F07F43A1F12C
:1006B0007F0223F40003D10743F4000348BF5B002B
:1006C000002556105B0019212C464FF08072A018AF
:1006D000984202DC84181B1AAD185B0052080139DD
:1006E000F5D113B105F001035D196D1005F17C55CD
:1006F00005EBC65500EE105A70BC704700EE000ABC
:10070000FAE713F400020CD15B0001321802FBD5AA
:10071000C2F101028918C8E730EE400A80EE000AF3
:10072000EAE701228918C0E753EC102B10461A465D
:1007300063B1B3F1004F09D04FF6FF73A2F58011FA
:10074000C7F6DF73994205D8042070470028F3D11B
:100750000220704702F1FE4101F570019942F3D980
:100760004FF6FF73C0F20F039A4201D8032070477F
:1007700002F100419942F9D90023C7F6F0739A4279
:1007800004D012F5801F01D000207047D0F1010085
:1007900038BF0020704700BF0020704710EE103AAD
:1007A0000BB902207047B3F1004FFAD0A3F5000156
:1007B0006FF00142914201D80420704703F1FF41DC
:1007C0009142F9D94FF6FE72591EC0F27F02914252
:1007D00001D80320704703F1004101399142F8D953
:1007E000B3F1FF4F05D013F5000F14BF0020012017
:1007F00070470120704700BF81F0004102E000BF58
:1008000083F0004330B54FEA41044FEA430594EAD0
:10081000050F08BF90EA020F1FBF54EA000C55EA0B
:10082000020C7FEA645C7FEA655C00F0E2804FEADC
:100830005454D4EB5555B8BF6D420CDD2C4480EABE
:10084000020281EA030382EA000083EA010180EAEE
:10085000020281EA0303362D88BF30BD11F0004F3C
:100860004FEA01314FF4801C4CEA113102D0404272
:1008700061EB410113F0004F4FEA03334CEA1333AD
:1008800002D0524263EB430394EA050F00F0A780C5
:10089000A4F10104D5F1200E0DDB02FA0EFC22FAC0
:1008A00005F2801841F1000103FA0EF2801843FAB4
:1008B00005F359410EE0A5F120050EF1200E012AA5
:1008C00003FA0EFC28BF4CF0020C43FA05F3C018E3
:1008D00051EBE37101F0004507D54FF0000EDCF15C
:1008E000000C7EEB00006EEB0101B1F5801F1BD305
:1008F000B1F5001F0CD349085FEA30004FEA3C0C09
:1009000004F101044FEA445212F5800F80F09A80FE
:10091000BCF1004F08BF5FEA500C50F1000041EB02
:10092000045141EA050130BD5FEA4C0C404141EB06
:10093000010111F4801FA4F10104E9D191F0000F2D
:1009400004BF01460020B1FA81F308BF2033A3F1B0
:100950000B03B3F120020CDA0C3208DD02F1140CA7
:10096000C2F10C0201FA0CF021FA02F10CE002F1E2
:100970001402D8BFC2F1200C01FA02F120FA0CFCDB
:10098000DCBF41EA0C019040E41AA2BF01EB045124
:10099000294330BD6FEA04041F3C1CDA0C340EDC22
:1009A00004F11404C4F1200220FA04F001FA02F365
:1009B00040EA030021FA04F345EA030130BDC4F123
:1009C0000C04C4F1200220FA02F001FA04F340EA18
:1009D0000300294630BD21FA04F0294630BD94F0C9
:1009E000000F83F4801306BF81F480110134013DB0
:1009F0004EE77FEA645C18BF7FEA655C29D094EA21
:100A0000050F08BF90EA020F05D054EA000C04BF9E
:100A10001946104630BD91EA030F1EBF0021002089
:100A200030BD5FEA545C05D14000494128BF41F028
:100A3000004130BD14F580043CBF01F5801130BD8C
:100A400001F0004545F0FE4141F470014FF0000017
:100A500030BD7FEA645C1ABF194610467FEA655CC8
:100A60001CBF0B46024650EA013406BF52EA03356A
:100A700091EA030F41F4002130BD00BF90F0000F58
:100A800004BF0021704730B54FF4806404F1320494
:100A90004FF000054FF0000150E700BF90F0000F4D
:100AA00004BF0021704730B54FF4806404F1320474
:100AB00010F0004548BF40424FF000013EE700BF44
:100AC00042004FEAE2014FEA31014FEA02701FBFD4
:100AD00012F07F4393F07F4F81F06051704792F0A6
:100AE000000F14BF93F07F4F704730B54FF4607420
:100AF00001F0004521F0004120E700BF50EA01026B
:100B000008BF704730B54FF000050AE050EA010217
:100B100008BF704730B511F0004502D5404261EB87
:100B200041014FF4806404F132045FEA915C3FF4C8
:100B3000DCAE4FF003025FEADC0C18BF03325FEA61
:100B4000DC0C18BF033202EBDC02C2F1200300FA16
:100B500003FC20FA02F001FA03FE40EA0E0021FA3B
:100B600002F11444C1E600BF70B54FF0FF0C4CF425
:100B7000E06C1CEA11541DBF1CEA135594EA0C0FDB
:100B800095EA0C0F00F0DEF82C4481EA030621EA16
:100B90004C5123EA4C5350EA013518BF52EA033551
:100BA00041F4801143F4801338D0A0FB02CE4FF003
:100BB0000005E1FB02E506F00042E0FB03E54FF033
:100BC0000006E1FB03569CF0000F18BF4EF0010E2B
:100BD000A4F1FF04B6F5007F64F5407404D25FEA27
:100BE0004E0E6D4146EB060642EAC62141EA5551DA
:100BF0004FEAC52040EA5E504FEACE2EB4F1FD0C1C
:100C000088BFBCF5E06F1ED8BEF1004F08BF5FEA99
:100C1000500E50F1000041EB045170BD06F000464B
:100C200046EA010140EA020081EA0301B4EB5C04F8
:100C3000C2BFD4EB0C0541EA045170BD41F48011F0
:100C40004FF0000E013C00F3AB8014F1360FDEBF15
:100C5000002001F0004170BDC4F10004203C35DAF1
:100C60000C341BDC04F11404C4F1200500FA05F374
:100C700020FA04F001FA05F240EA020001F0004215
:100C800021F0004110EBD37021FA04F642EB06018B
:100C90005EEA430E08BF20EAD37070BDC4F10C04B5
:100CA000C4F1200500FA04F320FA05F001FA04F279
:100CB00040EA020001F0004110EBD37041F1000165
:100CC0005EEA430E08BF20EAD37070BDC4F1200570
:100CD00000FA05F24EEA020E20FA04F301FA05F2D8
:100CE00043EA020321FA04F001F0004121FA04F280
:100CF00020EA020000EBD3705EEA430E08BF20EA50
:100D0000D37070BD94F0000F0FD101F00046400089
:100D100041EB010111F4801F08BF013CF7D041EA0B
:100D2000060195F0000F18BF704703F0004652000F
:100D300043EB030313F4801F08BF013DF7D043EAE0
:100D40000603704794EA0C0F0CEA135518BF95EA96
:100D50000C0F0CD050EA410618BF52EA4306D1D11D
:100D600081EA030101F000414FF0000070BD50EA3C
:100D7000410606BF1046194652EA430619D094EAC6
:100D80000C0F02D150EA013613D195EA0C0F05D1B0
:100D900052EA03361CBF104619460AD181EA030104
:100DA00001F0004141F0FE4141F470014FF00000BC
:100DB00070BD41F0FE4141F4780170BD70B54FF057
:100DC000FF0C4CF4E06C1CEA11541DBF1CEA1355D7
:100DD00094EA0C0F95EA0C0F00F0A7F8A4EB0504B9
:100DE00081EA030E52EA03354FEA013100F08880B0
:100DF0004FEA03334FF0805545EA131343EA126379
:100E00004FEA022245EA111545EA10654FEA00262D
:100E10000EF000419D4208BF964244F1FD0404F5E6
:100E2000407402D25B084FEA3202B61A65EB030542
:100E30005B084FEA32024FF480104FF4002CB6EBFF
:100E4000020E75EB030E22BFB61A754640EA0C007F
:100E50005B084FEA3202B6EB020E75EB030E22BFBF
:100E6000B61A754640EA5C005B084FEA3202B6EB00
:100E7000020E75EB030E22BFB61A754640EA9C00BF
:100E80005B084FEA3202B6EB020E75EB030E22BF8F
:100E9000B61A754640EADC0055EA060E18D04FEA4D
:100EA000051545EA16754FEA06164FEAC30343EAED
:100EB00052734FEAC2025FEA1C1CC0D111F4801FBA
:100EC0000BD141EA00014FF000004FF0004CB6E7B3
:100ED00011F4801F04BF01430020B4F1FD0C88BF52
:100EE000BCF5E06F3FF6AFAEB5EB030C04BFB6EB5D
:100EF000020C5FEA500C50F1000041EB045170BD50
:100F00000EF0004E4EEA113114EB5C04C2BFD4EB7C
:100F10000C0541EA045170BD41F480114FF0000E00
:100F2000013C90E645EA060E8DE60CEA135594EA7C
:100F30000C0F08BF95EA0C0F3FF43BAF94EA0C0F7F
:100F40000AD150EA01347FF434AF95EA0C0F7FF4F4
:100F500025AF104619462CE795EA0C0F06D152EA48
:100F600003353FF4FDAE1046194622E750EA41062C
:100F700018BF52EA43067FF4C5AE50EA41047FF43D
:100F80000DAF52EA43057FF4EBAE12E74FF0FF3CA2
:100F900006E000BF4FF0010C02E000BF4FF0010C73
:100FA0004DF804CD4FEA410C7FEA6C5C4FEA430CEC
:100FB00018BF7FEA6C5C1BD001B050EA410C0CBF3B
:100FC00052EA430C91EA030F02BF90EA020F00209D
:100FD000704710F1000F91EA030F58BF994208BF04
:100FE00090422CBFD8176FEAE37040F001007047C1
:100FF0004FEA410C7FEA6C5C02D150EA013C07D118
:101000004FEA430C7FEA6C5CD6D152EA033CD3D062
:101010005DF8040B704700BF8446104662468C465C
:101020001946634600E000BF01B5FFF7B7FF00288F
:1010300048BF10F1000F01BD4DF808EDFFF7F4FFB8
:101040000CBF012000205DF808FB00BF4DF808ED43
:10105000FFF7EAFF34BF012000205DF808FB00BF66
:101060004DF808EDFFF7E0FF94BF012000205DF888
:1010700008FB00BF4DF808EDFFF7CEFF94BF01203D
:1010800000205DF808FB00BF4DF808EDFFF7C4FF36
:1010900034BF012000205DF808FB00BF4FEA410289
:1010A00012F5001215D211D56FF47873B3EB6252BA
:1010B00012D94FEAC12343F0004343EA505311F0E1
:1010C000004F23FA02F018BF404270474FF0000073
:1010D000704750EA013005D111F0004008BF6FF0B1
:1010E000004070474FF00000704700BF4FEA4102D8
:1010F000B2F1E04324BFB3F5001CDCF1FE5C0DD976
:1011000001F0004C4FEAC0024CEA5070B2F1004FBF
:1011100040EB830008BF20F00100704711F0804FC2
:1011200021D113F13872BCBF01F00040704741F487
:1011300080114FEA5252C2F11802C2F1200C10FA8B
:101140000CF320FA02F018BF40F001004FEAC1236F
:101150004FEAD32303FA0CFC40EA0C0023FA02F313
:101160004FEA4303CCE77FEA625307D150EA0133E9
:101170001EBF4FF0FE4040F44000704701F00040B9
:1011800040F0FE4040F40000704700BFF8B5144640
:1011900006460F461D4600F027F804FB01F300FB4E
:1011A0000535A4FB0023EB18069CB21A67EB03037A
:1011B000C4E90023F8BD00BFF8B5144606460F4643
:1011C0001D4600F075F900FB05F5A0FB042304FBA8
:1011D0000155EB18069CB21A67EB0303C4E9002320
:1011E000F8BD00BF704700BF00292DE9F0071D467C
:1011F000C0F29E800024002DC0F2958007460D4667
:1012000016469C46002B3ED18A4254D9B2FA82F34C
:1012100043B1C3F1200620FA06F501FA03F19A4022
:1012200029439840160CB1FBF6F597B206FB151151
:101230004FEA104C07FB05F34CEA01418B4209D9F8
:10124000891805F1FF3C80F015818B4240F2128134
:10125000023D8918C3EB010CBCFBF6F306FB13C17E
:1012600080B207FB03F740EA0140874207D9591EC5
:10127000821880F00581974240F20281023B43EAE6
:101280000542002303E08B420AD900231A46104688
:10129000194614B1404261EB4101BDE8F0077047C7
:1012A000B3FA83F3002B40F087808C4501D3824250
:1012B000ECD80122EBE712B90123B3FBF2F2B2FA48
:1012C00082F6002E3AD1891A150C1FFA82FC0123EE
:1012D000B1FBF5F705FB17114FEA10480CFB07F6B9
:1012E00048EA01418E4207D9891807F1FF3802D236
:1012F0008E4200F2DA804746891BB1FBF5F605FB0A
:10130000161180B20CFB06FC40EA0140844507D967
:10131000711E821880F0B080944540F2AD80023E8C
:1013200046EA0742B3E7E443524263EB430365E70F
:10133000404261EB41014FF0FF345CE7B240C6F13F
:10134000200521FA05F320FA05F701FA06F9150C34
:10135000B3FBF5F847EA09091FFA82FC05FB1837C9
:101360004FEA19410CFB08F341EA0747B040BB4282
:101370000AD9BF1808F1FF3180F09580BB4240F2D6
:101380009280A8F10208BF18FE1AB6FBF5F305FB20
:1013900013611FFA89F90CFB03F649EA01418E42F9
:1013A00006D95F1E891878D28E4276D9023B8918F9
:1013B000891B43EA08438BE7C3F1200726FA07F8A5
:1013C0000CFA03F248EA020C21FA07F105FA03FAD3
:1013D0004FEA1C4920FA07F5B1FBF9F845EA0A057E
:1013E00009FB18172A0C1FFA8CFA0AFB08F142EACB
:1013F0000747B94206FA03F609D917EB0C0708F1BB
:10140000FF324ED2B9424CD9A8F1020867447F1A84
:10141000B7FBF9F209FB1271ADB20AFB02FA45EA19
:1014200001418A4507D9551E11EB0C0137D28A4577
:1014300035D9023A614442EA08424FEA124C1FFA97
:1014400086F808FB0CF7360C95B208FB05F806FB8E
:10145000057505EB184506FB0CFCAF4288BF0CF583
:10146000803CCAEB01010CEB1546B14212D309D006
:1014700000230CE76546EDE60E4646EA074206E71E
:101480000B46FCE61FFA88F800FA03F308EB054563
:10149000AB42EDD2013A0023F9E63B4688E72A4603
:1014A000C9E79046B3E788466EE7023F891823E70D
:1014B0002DE9F00F144605460E46002B3FD18A4217
:1014C0004AD9B2FA82F343B1C3F1200025FA00F2FF
:1014D00001FA03F69C4016439D40210CB6FBF1F245
:1014E0002F0CA0B201FB126C00FB02F347EA0C4682
:1014F000B34208D9571E361980F0FF80B34240F23C
:10150000FC80023A3619F61AB6FBF1F301FB1361BF
:10151000ADB200FB03F045EA0141884207D95E1EE7
:10152000091980F0EC80884240F2E980023B43EAEE
:101530000242002310461946BDE8F00F70478B4267
:1015400043D8B3FA83F4002C42D18B42234601D313
:1015500082423BD80122EDE712B90123B3FBF2F43A
:10156000B4FA84F2002A40F08A80091B260CA7B244
:101570000123B1FBF6F006FB10114FEA154C07FBF7
:1015800000F24CEA01418A4207D9091900F1FF3CF7
:1015900002D28A4200F2D3806046C2EB010CBCFB4F
:1015A000F6F206FB12C1ADB207FB02F745EA0145B0
:1015B000AF4207D9511E2C1980F0A380A74240F2F8
:1015C000A080023A42EA0042B4E700231A46B1E79B
:1015D000C4F1200722FA07F603FA04F3334321FA91
:1015E00007FA4FEA134C01FA04FB20FA07F141EA2B
:1015F0000B0BBAFBFCF70CFB17A61FFA83F84FEA9C
:101600001B4508FB07F945EA0645A94502FA04FA15
:1016100004D97A1EED18C0F088801746C9EB05057D
:10162000B5FBFCF60CFB16521FFA8BFB08FB06F809
:101630004BEA0241884503D9721EC91870D3164679
:1016400046EA0742170C1FFA8AFC0CFB07F695B214
:101650004FEA1A430CFB05FC03FB056505EB1C4533
:1016600003FB07F3AE4288BF03F58033C8EB0101EB
:1016700003EB1543994250D347D000235AE79440D7
:10168000C2F12008260C20FA08F721FA08F501FA21
:1016900002F9B5FBF6F847EA090906FB1855A7B2A7
:1016A0004FEA194C4CEA054C07FB08F3634500FA76
:1016B00002F509D91CEB040C08F1FF323DD2634559
:1016C0003BD9A8F10208A444C3EB0C02B2FBF6F329
:1016D00006FB13201FFA89F907FB03F249EA0041D0
:1016E0008A4206D9581E091925D28A4223D9023BBB
:1016F0000919891A43EA08433BE73A4603E73346A8
:1017000015E70A4642EA004214E71FFA8CF100FA94
:1017100004F001EB0545A842AFD2013A002309E7E6
:1017200088458CD9023EC9188AE7A9457FF675AF6E
:10173000023FED1872E70346DBE79046C4E7023844
:1017400009192AE740F28843C2F20003186870477B
:101750000F2AF0B43AD941EA00039B0738D10C466E
:101760000346154626681E6066685E60A6689E6031
:10177000E668103DDE60103410330F2DF2D8A2F170
:10178000100424F00F0402F00F021034032A00EBBF
:101790000403214411D90E461D46144656F8047B15
:1017A000043C032C45F8047BF8D8141F24F00304F0
:1017B000043402F0030209191B192AB111F8014B74
:1017C000013A03F8014BF9D1F0BC70470346F4E746
:1017D0000346F3E70EB470B540F288419DB0C2F203
:1017E000000121AB096853F8042B6FF00044054653
:1017F0000394069408464FF4027601A94FF6FF744D
:101800001B93ADF8106001950595ADF8124000F0FE
:1018100067F8019B00221A701DB0BDE8704003B04C
:10182000704700BF80EA0102844612F0030F4FD1D7
:1018300011F0030F32D14DF8044D11F0040F51F89F
:10184000043B0BD0A3F101329A4312F0803F04BF56
:101850004CF8043B51F8043B16D100BF51F8044B3F
:10186000A3F101329A4312F0803FA4F101320BD16F
:101870004CF8043BA24312F0803F04BF51F8043BF4
:101880004CF8044BEAD023460CF8013B13F0FF0F51
:101890004FEA3323F8D15DF8044B704711F0010F84
:1018A00006D011F8012B0CF8012B002A08BF704755
:1018B00011F0020FBFD031F8022B12F0FF0F16BF4C
:1018C0002CF8022B8CF8002012F47F4FB3D1704714
:1018D00011F8012B0CF8012B002AF9D1704700BF39
:1018E0002DE9F04FBFB0934605910B93089002F09D
:1018F000E7F9006800230022CDE91423109002F0DC
:10190000E1FF1290059883891B0603D50369002B1C
:1019100001F03F8046F26761002319AAC6F26661B2
:101920000A9333923593349316931793079316467D
:1019300013919BF80030002B00F0BC80252B00F0A9
:10194000B9805A465F4601E0252B04D012F8013FCA
:101950000137002BF8D1CBEB07037BB1349C359DCD
:10196000C6F800B00134ED18072C73603595349437
:1019700000F3828008360798C01807903B78002B48
:1019800000F084800021002207F1010B7B78069192
:101990008DF8F7204FF0FF37039120242B200BF117
:1019A000010BA3F12002582A00F21782DFE812F09F
:1019B000C10215021502AE0215021502150215022A
:1019C00015021502B502840015025D00890015029A
:1019D000A300AA00AA00AA00AA00AA00AA00AA00BE
:1019E000AA00AA0015021502150215021502150219
:1019F0001502150215021502BB0049011502490125
:101A000015021502150215028401150215028B013B
:101A100015021502150215021502A3011502150281
:101A2000B70115021502150215021502150215025D
:101A30001502150215024F02270249014901490109
:101A400048022702150215020A0215028A026002E4
:101A50007302DA011502E10115029802150215025E
:101A6000D602069B0B915B420693039941F0040159
:101A700003919BF8003092E708980599029333AAE6
:101A800002F050FF029B40B919AE74E7359B23B1B9
:101A90000898059933AA02F045FF0599079A8B89A2
:101AA00013F0400F18BF4FF0FF32079207983FB076
:101AB000BDE8F08F5F4661E78DF8F7009BF80030D6
:101AC0006DE75A4612F8013B2A2B01F0FB80A3F187
:101AD0003001092901F2AA80002712F8013B07EB27
:101AE000870701EB4707A3F1300109299346F4D991
:101AF00047EAE77755E7039941F0800103919BF8A6
:101B000000304CE759460022A3F1300C11F8013B9C
:101B1000A3F1300502EB8202092D0CEB42028B4649
:101B2000F2D906923DE70F93039B43F01003039312
:101B30000398850640F168810B99CB1D23F00703BC
:101B4000D3E9000108330B93002871F100038046AC
:101B50008946C0F26C810123002F03DB039921F039
:101B60008001039158EA090240F0E882002F40F01A
:101B7000E582002B40F03784039AD10740F133848B
:101B800030238DF8CB30012309930DF1CB0A09984E
:101B90009DF8F7300C97B842B8BF38460021049042
:101BA000119113B1049801300490039B13F00203C8
:101BB0000D9302D0049802300490039B13F0840329
:101BC0000E9340F0E28106980499471A002F40F3E3
:101BD000DC81102F359D349CDFF87C8325DD234686
:101BE0002A4644464FF01009059DDDF8208003E0A9
:101BF000103F0836102F15DD01331032072B86E811
